:100000000C9466000C9487000C9487000C94870075
:100010000C9487000C9487000C9487000C94870044
:100020000C9487000C9487000C9487000C94870034
:100030000C9487000C941A0F0C9487000C94870082
:100040000C9487000C94A1000C9487000C948700FA
:100050000C9487000C9487000C9487000C94870004
:100060000C9487000C94A3160C9487000C948700C2
:100070000C9487000C9487000C9487000C948700E4
:100080000C9487000C9487000C9487000C948700D4
:100090000C942C300C9487000C9487000C948700EF
:1000A0000C9487000C9487000C9487000C948700B4
:1000B0000C9487000C9487000C9487000C948700A4
:1000C0000C9487000C9487000C94870011241FBEA9
:1000D000CFEFD1E2DEBFCDBF00E00CBF15E0A0E066
:1000E000B2E0E4E2FFE001E00BBF02C007900D9236
:1000F000AC39B107D9F718E0ACE9B5E001C01D9201
:10010000A13EB107E1F70E9485100C9490870C94F2
:10011000000081E08093AD051092A2058091A205B8
:100120008093A1058091A1058093A0058091A005F1
:1001300080939F051092A3051092B0051092B1050F
:1001400008951F920F920FB60F9211242F933F9391
:100150004F935F938F939F93AF93BF938091390693
:1001600090913A068F5F9F4F49F0809139069091A8
:100170003A06019690933A068093390680919C0541
:10018000823009F474C0813009F460C0882309F01A
:1001900050C08091010290910202A0910302B0919F
:1001A00004028093050290930602A0930702B09385
:1001B0000802209101023091020240910302509105
:1001C000040280914B0690914C06A0914D06B0918F
:1001D0004E06820F931FA41FB51F809301029093B8
:1001E0000202A0930302B093040220910102309115
:1001F0000202409103025091040280910502909105
:100200000602A0910702B0910802281739074A0791
:100210005B0778F48091AD058F5F8093AD05809189
:10022000AD0581708093AD058091AC058F5F8093A3
:10023000AC05BF91AF919F918F915F914F913F918D
:100240002F910F900FBE0F901F90189599B1929516
:1002500091708091D505981761F39093AD059093B7
:10026000D5058091AC058F5F8093AC05E2CF80917E
:10027000D1059091D205892BE1F28091D105909121
:10028000D20501979093D2058093D1058091D10535
:100290009091D205892B69F6C7CFE0E7F0E0808125
:1002A0008260808383E08093B0008093B1008AEF06
:1002B0008093B30008951092800089E080938100BC
:1002C00085E09DE0909389008093880010928500DE
:1002D0001092840082E080936F000895089508953D
:1002E000BC0181E06D327807C0F16CE271E09B01E6
:1002F00040E050E080913E0690913F0686179707B8
:1003000019F081E08093C00570933F0660933E062C
:100310007093500660934F066091090270910A0233
:1003200080910B0290910C020E946E876FEF7FEF1D
:100330008FEF9FEF0E946E87CA01B90128EE33E06C
:1003400040E050E00E941C8760934B0670934C067F
:1003500080934D0690934E0608956431710538F6EA
:1003600064E170E024E130E040E050E0C3CF9B0165
:10037000AC01CA01AA27BB27BC01892B79F0687F91
:10038000672B59F483E056954795379527958A95BD
:10039000D1F73093540620935306089530935406B2
:1003A00020935306089580915106982F9295969523
:1003B00096959370282F221F2227221F9227282FDD
:1003C00022952F709227282F269526959227917097
:1003D000880F892B8093510608959093430680934C
:1003E000420685EB9BE390935B0680935A0683E37A
:1003F00093E1909361068093600685E694ED909377
:1004000056068093550608958091420690914306C2
:10041000AC01440F452F441F550B519548275927D0
:1004200060915A0670915B06709343066093420692
:10043000809160069091610690935B0680935A06C6
:100440002091550630915606309361062093600640
:10045000C9010024969587950794969587950794EA
:10046000982F802D8227932784279527542F442760
:100470005295550F507E842795279093560680936A
:100480005506660F771F6F5F7F4F869F9001879F8E
:10049000300D969F300D1124C9010895FC01908103
:1004A000992351F08091C80085FFFCCF9093CE0036
:1004B000319690819923B1F708951F93CF93DF93DD
:1004C000182F492FE0E1F7E2C0E0D0E0812F942F10
:1004D000BF010E9447879B016115710589F5812F36
:1004E000942FBF010E944787182F492FCF016AE040
:1004F00070E00E944787FB012196C430D10531F797
:100500003097A1F18091C80085FFFCCF812F942FF7
:10051000BF010E944787605D6093CE00CF016AE013
:1005200070E00E9447879B0161157105F9F0812FEA
:10053000942FBF010E944787182F492FF901E2CF5E
:100540008091C80085FFFCCF822F805D8093CE0014
:10055000812F942FBF010E944787182F492FCF0169
:100560006AE070E00E944787FB01CACFDF91CF911C
:100570001F910895982F9F709A3040F48091C80081
:1005800085FFFCCF905D9093CE0008958091C800C8
:1005900085FFFCCF995C9093CE000895982F8091B1
:1005A000C80085FFFCCF9093CE0080E090E00895D6
:1005B0002091C800332727FD30952227330F221FB3
:1005C0003327C90108958091C80087FFFCCF80912F
:1005D000CE0090E008959C018FEF8093470693E052
:1005E000283E390768F580934406809345062436F3
:1005F0003105D8F0C90164E670E00E944787609336
:100600004406C9016AE070E00E944787CB016AE0B6
:1006100070E00E94478780934506C9016AE070E058
:100620000E9447878093460608952A30310548F78F
:10063000C9016AE070E00E944787809346060895EA
:100640001092440610924506109246060895909125
:10065000A40593609093A4058093A50508958091C7
:10066000A40583608093A4050895F999FECF92BDF7
:1006700081BDF89A30B5F999FECF019692BD81BD42
:10068000F89A20B5932F80E030E0282B392BC90150
:100690000895F999FECF92BD81BDF89A80B508956D
:1006A000F999FECF92BD81BD60BDF894FA9AF99A8E
:1006B000789408958091C90088618093C90083E38C
:1006C0008093CC001092CD008091C80087FD3AC085
:1006D0008091C90080688093C9008091C1008869B9
:1006E0008093C1008FE18093C4001092C50090EC0C
:1006F00091B98CE382B987E384B995B99FEF97B933
:1007000088EF8AB98BE08BB982E08DB99EB910BAB7
:1007100091BB88E183BB87EE84BB80E58CBD8DB542
:1007200081608DBD8CB581608CBD8CB58D7F8CBD9D
:1007300008958091CE008AE00E9478168091C800CA
:1007400087FFC6CF8091C80087FDF3CF8091C80096
:1007500087FFF8CFEECFAF92BF92CF92DF92EF92AA
:10076000FF920F931F93DF93CF930F92CDB7DEB716
:10077000F89420919C05223009F42AC38091330615
:10078000882309F0EFC1CC2480913406813009F42C
:100790000CC380919F058C3060F010929F05809172
:1007A000A0058F5F8093A0058091A1058F5F809346
:1007B000A1058091A105882341F08091A10590E0D9
:1007C00083709070892B09F4E1C28091A205883072
:1007D00028F01092A20581E08093BF058091A105C9
:1007E0008F708093A1059091A005809100029817C9
:1007F000C0F01092A0058091A3058F5F8093A305A0
:100800009091A30580915F06981708F0BCC2809173
:10081000A40582608093A4058091A80581608093DF
:10082000A80580913406823009F44AC380919D0660
:100830008C3009F434C3DC2CC4FC29C0C0FE1CC0BD
:100840008091BE05882309F428C481E08093AD051A
:100850001092A2058091A2058093A1058091A10527
:100860008093A0058091A00580939F051092A30519
:100870001092B0051092B105D1FC9DC3D2FE05C007
:100880008091BE05882309F4E5C4D3FC9BC3209165
:100890009C05222309F056C18091AD05882309F0FB
:1008A0004BC15C989091B00580915906981710F053
:1008B0001092B0058091DB08882329F08091B00563
:1008C000882309F45BC28091350620915705409139
:1008D000570590E030E0240F311D8217930714F084
:1008E00010923506E0915705E695E695E69520913C
:1008F000B20590913506E150F0E0EE0FFF1FEE0FCC
:10090000FF1FE20FF11DE35FFD4F8081891709F49E
:10091000FEC2BB2480915705869590915206899F0F
:10092000902D11248091B105891710F01092B10516
:100930008091DB08882349F08091B105882309F470
:10094000A39A9695891709F43BC380919D06873039
:1009500009F437C1883008F42CC18B3009F431C157
:100960008C3008F435C38C3009F487C48D3009F419
:1009700028C180913406823009F447C58091DB0894
:10098000882321F022E0B21609F44DC68091DB08DD
:10099000882309F4CDC28091EF058F708093EF0515
:1009A0008091BE05882309F0F7C18091A10590E0F0
:1009B00083709070892B09F452C580919C0588231F
:1009C00009F0BAC285E20E941B248091EF0590E0F5
:1009D0008370907002970CF4A6C28FEF8093E305AA
:1009E0008091F805882309F02AC28091B2058130F0
:1009F00009F4FDC1809133068823B1F08091A505EB
:100A0000882391F080915C06813009F426C480919E
:100A10005C06882321F48091A40580FD22C6809184
:100A20005C06833009F414C38091A605813009F473
:100A3000C4C48250823008F4CCC48091AB058823B2
:100A400051F08091B305823009F4E6C480919C0591
:100A5000882309F475C20E94A724BB2031F080913D
:100A60009D058F5F817080939D05809135068F5F16
:100A7000809335068091CF088F5F8093CF08809157
:100A80009F058F5F80939F058091B0058F5F809356
:100A9000B0058091B1058F5F8093B1052091CF089B
:100AA0008091570530E086958695869548E1849F2C
:100AB000C00111242817390714F01092CF08D4FE72
:100AC0002EC010E11C25012F10FF1CC08091BE0517
:100AD000882309F4B5C281E08093AD051092A20588
:100AE0008091A2058093A1058091A1058093A00526
:100AF0008091A00580939F051092A3051092B005E8
:100B00001092B10501FD85C402FF05C08091BE05AC
:100B1000882309F49AC203FF02C00E9415657894E5
:100B20000F90CF91DF911F910F91FF90EF90DF9089
:100B3000CF90BF90AF9008955C9A88EF0E942618DE
:100B400020919C05213009F4D7C1223009F0AACEAA
:100B50008091AD05882309F4A4CE5C9A88EF0E94A9
:100B60002618A0CE213009F456C2CC24223009F038
:100B70000BCE8091C60580FF08C081E0C82A809115
:100B8000C60591E089278093C6058091C60581FF3F
:100B900008C0E4E0CE2A8091C60592E089278093C0
:100BA000C6058091AD05882309F0EECDF0E1CF2A8E
:100BB000EBCD813008F4DDCE843018F0853009F0BB
:100BC000D8CE21E0B21609F46EC232E0B31609F0B5
:100BD000D0CE8091EF058F5F8093EF058091DB0889
:100BE000882309F4C5C0809162078823F1F58091BC
:100BF00032088823A1F480919D06853009F47AC7D4
:100C0000809177088D3010F01092770880917708E6
:100C100080937C088091BB05823009F493C71092C1
:100C2000CF0880916607882349F48091D1088823F2
:100C300029F08091F805882309F08BC78091EA0795
:100C400060913208680F80917508909176080E9433
:100C5000C55D1092EF0580916E02882309F080C671
:100C600081E08093B2051092350680916207E09191
:100C70007508F0917608E80FF11D808180933D069C
:100C80008091B805882341F08091FF05882321F4E5
:100C90008091B50580933D0680914A068093480671
:100CA00080913D06807480934A068091F8058823E0
:100CB00009F0BDC580913D068F708F3009F439C6AB
:100CC00080913D068F708F3029F180913D060E9402
:100CD000185900917C08080F10913D06107860911A
:100CE0004806802F412F0E94FB43112309F02FC695
:100CF00080E0902F935F982B8091A905981751F071
:100D00008091A9058093AA059093A9058091A905D2
:100D10000E94DA1780919D06833009F4A8C580915E
:100D20009D06873029F58091A605882349F08330F8
:100D300039F08091490790914A0701960E94EB0291
:100D40008091490790914A07E0915B07F0E0EE0F30
:100D5000FF1FED58FD4F6081718182959295907FC4
:100D60009827807F98270E944787862F0E944428D3
:100D70008091A40581608093A405FBCDA49A85E0B1
:100D80008093AE05A0CD1092A30541CD8091A20520
:100D90008F5F8093A20519CD8091A10580FFC6C009
:100DA00063E085E20E94D72310CE8091AD058823B1
:100DB00009F4EFCC8091DB08882329F48091330675
:100DC000882309F05FC4E8E0CE2A10923406E1CC13
:100DD0008091C80581508093C8058091C8058170B5
:100DE0008093C8058091C8058093AD05C7CC8091DC
:100DF0003506882309F0FECDA0916902AA0FAA0F3B
:100E0000EA2FF0E0EB5EFD4F808180930D02AF5F33
:100E1000EA2FF0E0EB5EFD4F808180930E02AF5F22
:100E2000EA2FF0E0EB5EFD4F808180930F02AF5F11
:100E3000B0E0AB5EBD4F8C9180931002DBCD8CE2B5
:100E40000E941859982F8091EF058111945F80912D
:100E5000CF08882341F48091F905882309F49CC4C4
:100E600083E20E9485238091CF08843009F0BDCDB4
:100E70008091F905882379F48091F605823008F491
:100E8000B4C48091EE070E9418594091EE07407853
:100E900060E00E94FB4383E20E941B24A6CD809168
:100EA000A80580FF0AC08091DB08882309F0ECC206
:100EB0008091CB05882309F01EC41092A805BBCCF5
:100EC0008091A005882309F0B1CC80919F058823EB
:100ED00009F0ACCC80913306882359F08091DB086F
:100EE000882309F079C4F2E0CF2A222311F421E00B
:100EF000C22A109234069ACC8091AD05882309F459
:100F0000D1CC88EF0E94261820919C051ECE2F5F21
:100F100023702093B20580919D05882309F455C064
:100F2000BB24B394F7CC1092E3055ACD60E039CFDF
:100F300081E20E941B242FCD85E20E94BD2345CD76
:100F400080915605882309F486CD0E94F22760918E
:100F50003E0670913F06603A710508F49BC3603A03
:100F6000710509F47BC480E090E02EE030E040E0C1
:100F700050E00E941C87685E7E4F8F4F9F4F28E194
:100F800031E040E050E00E946E87022F293008F4E3
:100F9000B4C518E0812F0E9442271F5F1017D0F3BD
:100FA000003108F058CD102F812F0E94112B1F5FA8
:100FB0001031D0F350CD0E94015ED2FE66CC60CCE1
:100FC000A398C3CC0E94156562CCB2E0BB2EA2CC24
:100FD000883009F0CECC81E0B81609F4E3C3E2E032
:100FE000BE1609F0C6CC80913C0680939E05809188
:100FF0003B0680933C060E94D30180933B06809180
:101000003C068F7360E040E00E94FB4380913C0609
:101010000E94DA17AECC0E94E31E882309F01FC39A
:10102000C82E0E94F51E882311F024E0C22A809168
:10103000AD05882311F430E1C32A20919C0596CD9B
:101040000E94015E1D7F012F46CD0E94156563CD74
:101050008091A40590E083709070892B09F4E4CC12
:101060008091A4058C7F8093A4050E94F227809133
:10107000DB08882359F0809162070E9442279091F3
:1010800062078091A305981709F4CECC8091A3053F
:101090008F7063E00E94B826C7CC0E94015EFDEF0E
:1010A000CF22DC2CD2CB809166078F5F80936607BE
:1010B0008091DB08882309F45CCC809162078F5F04
:1010C000809362079091620780915805981710F0FD
:1010D0001092620780916207882309F07FC0809197
:1010E0009D06873009F4E9C3809132088F5F8093B1
:1010F0003208A0903208909132088091F00798173A
:1011000008F451C08091F305882319F481E080939D
:10111000320680919D06813009F48CC480919D0631
:10112000823009F483C480919D06833009F419C389
:1011300090E0109266078091F805882369F080910D
:10114000F6058093D1088091D108882329F0109268
:10115000F60581E0809360071092320880919D0629
:10116000833009F46AC480919D06873009F41BC45A
:1011700080919D068D3009F4EBC220E080919D06A0
:10118000833009F402C480919D068D3009F4DBC3DD
:1011900080919D06833009F4D6C31092B905109250
:1011A000BA050E94735C8091320890E08295929516
:1011B000907F9827807F98278C5C974F9093760834
:1011C0008093750880913E0280930E0280913F02C9
:1011D00080930F0280914002809310020E94895AEE
:1011E0008091F805882399F580916207E091750850
:1011F000F0917608E80FF11D808180933D06809183
:101200003D068093B6058091B805882341F0809112
:10121000FF05882321F48091B50580933D068091D8
:101220003D068F708F3009F445C380914A060E94B5
:1012300012448091AA05882309F035C380914A069B
:10124000882329F48091A905882309F0E8C30E9426
:10125000C6578FCB0E94156518CB8091A40581FFDE
:10126000D6CB8091A4058D7F8093A4050E94F227A0
:101270008091A3050E944227CACB0E94F227809149
:10128000A80580FD52C18091CB05882309F047C194
:10129000F1E0BF1609F44DC1F2E0BF1609F069CBC9
:1012A0008091EF058F5F8093EF058091DB088823A5
:1012B00009F45FCBE0913208F0E0E858F74F808105
:1012C00084FD97C28CE08093570580916207E0917E
:1012D0007508F0917608E80FF11D808180933D0636
:1012E00080914A068093480680913D0680748093E1
:1012F0004A0680913D068F708F3009F4A7C2809115
:101300003D068F708F3029F180913D060E9418595B
:1013100000917C08080F10913D06107860914806F6
:10132000802F412F0E94FB43112309F0B3C280E0BC
:10133000902F935F982B8091A905981751F0809179
:10134000A9058093AA059093A9058091A9050E94FB
:10135000DA178091A705982F92959F7090938D082A
:10136000982F97709093EA07869586958695817059
:101370008093CE088091BB05823009F4EAC2809147
:10138000CE08882309F046C288E00E948523809118
:101390006107882309F4D5C263E081E00E94D72366
:1013A0000E9407298091EA078F5F0E94AB278091F6
:1013B000DB0881708093DB08DCCA0E941B288091C7
:1013C000A10580FF34C18091A6058250823008F0CB
:1013D00034CB0E941B2890914406892F8150823083
:1013E00008F4EEC19091450680914606981709F4DD
:1013F0002AC1992309F0DEC18091A10580FD1DCB92
:10140000809146060E94CF2718CB81E20E94BD231F
:10141000C2CA0E94015E78CB009169020A3018F1BD
:10142000B6EFFB2EF00E10E0812F63E00E94B8268D
:101430001F5FF116C8F7102F1950103130F4812FAB
:101440000E94112B1F5F1031D0F3FF2009F003CB56
:101450008FE00E94422780E00E944227FCCA85E27A
:101460000E948523B2CA0B5F10E0812F0E94112BCE
:101470001F5F1017D0F3102F812F63E00E94B82652
:101480001F5F1031C8F3E7CA8091DB08823008F48F
:1014900014CD8091CB05882329F480914D078823B2
:1014A00009F40BCD8091CC058093A705909132086B
:1014B0009F5F909332089091320891709093320818
:1014C0006091320870E062957295707F7627607F38
:1014D00076276C5C774F70937608609375089091CF
:1014E0003208092F10E00E942E5B0858174FF801B0
:1014F0008083E0913208F0E0E858F74F80818F70E8
:101500008F5F80935805E0913208F0E0E858F74F7C
:10151000808184FD53C18CE080935705CECC8091AF
:10152000CB0581500E944227B3CE8FE00E94422714
:10153000AACE8091DB08882309F41BCA8091620738
:101540008F5F809362078091CB05882309F43CC1AB
:101550009091CC058091A705891789F19091320867
:101560009F5F9170092F10E07801E294F29480EF70
:10157000F822FE24E822FE2424E338E0E20EF31EE3
:101580008091CC05B70199830E942E5B0858174FB4
:10159000F80180838091CC058093A7059981909371
:1015A0003208E0913208F0E0E858F74F80818F7000
:1015B0008F5F80935805F0927608E09275088091CD
:1015C0006207609158050E943B8790936207809163
:1015D0006207E0917508F0917608E80FF11D8081AF
:1015E00080933D0680913D068F708F3009F40AC1CB
:1015F00080914A060E9412448091AA05882309F02E
:10160000FAC080914A06882329F48091A90588238D
:1016100009F042C180916207882309F0AAC981E0DC
:1016200080933206A6C981E20E948523B4C9E09165
:10163000A105E695F0E0E370F070EC5BF94F808176
:101640000E94CF27C0CE8091A10582FD04C0809169
:10165000A10580FDF2C9892F0E94CF27EEC981E044
:10166000DFCC8091A4058E7F8093A4050E94F22791
:101670008091DB08882309F4D2C9809162070E9417
:101680004227CDC932E0C32A222309F09ECB81E054
:10169000C82A9BCB80E090E02EE030E040E050E0B4
:1016A0000E941C876E5070408040904028E131E0DD
:1016B00040E050E00E946E87022F222309F418C2F6
:1016C00010E0812F0E94112B1F5F1017D0F30830FC
:1016D00008F00CC2102F812F0E9442271F5F183084
:1016E000D0F3103108F0B7C9812F0E94112B1F5F72
:1016F0001031D0F3B0C98091CC058093A7050E942A
:10170000015E80919C05882309F4C1C01092B20546
:10171000809132088F5F8093320880913208817007
:10172000809332086091320870E062957295707F04
:101730007627607F76276C5C774F7093760860938E
:10174000750880913208082F10E08091A705CBCE54
:101750002091FD0521FFD3C181E08093B90520E0F0
:101760000DCD8091490790914A07019690934A07C1
:10177000809349072091490730914A078091540787
:10178000909155072817390708F4D2CC10924A07D0
:101790001092490791E0CDCC892F60E040E00E9493
:1017A000FB435ECB80E00E94124480913C060E9485
:1017B0000018DFC8892F0E94CF271ECE80E1ACCE53
:1017C000865F0E94CF270ECE80914D07882309F0B7
:1017D000F6CE0E941565F3CE1092B2051092350632
:1017E00010929D051092620784CB80E00E94124403
:1017F00052CB80E168CD8091AA050E94001810921A
:10180000AA05FFCE80914A06882309F0B8C010923D
:101810004A06EECE81E00E948523809161078130E7
:1018200009F4B1C063E088E00E94D723B9CD80916C
:10183000EA076091F007409163072091F10700915A
:101840006707E09061070E945B2B64CA80913D06A8
:101850008F7080933D0610924A0651CD0E94F22768
:1018600087E00E94422788E00E944227F4C88091C6
:10187000A605882309F453CA833009F450CA80911D
:10188000490790914A0701960E94EB0248CA0E94BC
:1018900089003CCF80E84CCD8091A9050E940018BA
:1018A0001092A905B7CE8091AA050E940018109247
:1018B000AA05C4CC10924A06B8CC8091EE058130BE
:1018C00009F012CC6091CE088091EA07409132086D
:1018D00020917C08480F81E597E00E94F9458091AE
:1018E0005B076091490770914A07409151070E9438
:1018F0005F468091490790914A07019690934A0765
:1019000080934907E0915B072091490730914A078E
:10191000F0E0EE0FFF1FED58FD4F808191812817F9
:10192000390708F4E1CB1092EE0583E20E941B24F4
:10193000DBCB80913D068F7080933D0610924A0666
:10194000BFC960E02ACD222309F42BCC26CC80E845
:10195000D0C90E94302980917C080E94652727CD3C
:101960008091EA076091F007409163072091F107A9
:1019700000916707E09061070E945B2B71C981E0CD
:101980000E94124444CF60E04ECF8091FD0581FF5C
:10199000CDC09091BA0591FFF6CB82E09827909345
:1019A000BA0521E0F0CB8091EE05813009F0E0CB63
:1019B00080914D078823B9F01092EE0510924D07E3
:1019C00080915B076091490770914A070E943646F3
:1019D00080915B070E94C2469093550780935407FD
:1019E00083E20E941B2480914E07882309F4C0CB18
:1019F00010924E0780915B076091490770914A07EA
:101A00006A190E94264680915B070E94B94690930E
:101A10005D0780935C0780E00E941B24A9CB809126
:101A2000A9050E9400181092A90511CC81E08093AD
:101A3000320679CB8093320671CB80914D07882393
:101A400009F0A2C080914E07882309F46BC0109260
:101A50004A07109249078091980680935B0780910E
:101A60005B070E94C246909355078093540780916C
:101A70005B070E94B94690935D0780935C072091B5
:101A80005C0730915D0780915407909155072817A6
:101A9000390720F010925D0710925C078091BA051B
:101AA00082608093BA0580914E07882309F077C041
:101AB00080915B076091490770914A070E94DC465C
:101AC0008093510780915B076091510749EA57E085
:101AD00021E637E003E617E077E7E72E78E0F72E18
:101AE0000E94D94581E08093F1073DCB102FF9CDBD
:101AF00010E0F1CD1092770883C818E055CA20FF96
:101B00003CCB8091F107882339F49091CE088091E5
:101B10006107981709F431CB81E028272093FD0550
:101B200021E02CCB992309F4BECF91CF80FF2BCBA2
:101B30009091BA0590FF27CB81E098279093BA0542
:101B400021E021CB0E943029809177080E946527EF
:101B500066C881E00E94124480E00E9412446091B5
:101B6000F00784E398E04EE858E028E637E00E946A
:101B700042591092F8058AE00E94345910924A06A0
:101B800082E00E9478165AC810924D0710924A07B8
:101B90001092490783E20E941B2491E053CF1092D8
:101BA0004E0780915C0790915D0790934A07809360
:101BB000490780E00E941B248091BA0582608093CF
:101BC000BA0576CFF999FECF92BD81BD70BDF8946C
:101BD000FA9AF99A7894F999FECF019692BD81BD4F
:101BE00060BDF894FA9AF99A78940895AC019C0132
:101BF000232F332722952F702115310509F04BC073
:101C0000252F33272115310591F59A01329522951B
:101C10002F7023273F70232721153105A1F4942F1E
:101C20009F709A3040F48091C80085FFFCCF905D92
:101C30009093CE0008958091C80085FFFCCF995CF9
:101C40009093CE000895922F9F709A3040F4809127
:101C5000C80085FFFCCF905D9093CE00E0CF8091CF
:101C6000C80085FFFCCF995C9093CE00D8CF922F0F
:101C70009F709A3040F48091C80085FFFCCF905D42
:101C80009093CE00C2CF8091C80085FFFCCF995CB5
:101C90009093CE00BACF922F9F709A3040F48091EB
:101CA000C80085FFFCCF905D9093CE00A9CF8091B6
:101CB000C80085FFFCCF995C9093CE00A1CF07C0F0
:101CC0008091AC0581508093AC050E94AB0380915C
:101CD000AC058823A9F78091BF058823B9F110923C
:101CE000BF0580919C058823F1F420913E06309138
:101CF0003F0680915706909158062817390799F0AA
:101D00008091DB08882379F485E20E948523609125
:101D10003E0670913F06709358066093570685E023
:101D200090E00E94E20D2091690280916A02821780
:101D300069F020936A02F999FECF80E190E092BDAC
:101D400081BD20BDF894FA9AF99A78948091C005E3
:101D5000882309F408951092C005F894789480912E
:101D60003E0690913F060E94BA2E0895CF93DF93CE
:101D7000F999FECF85E090E092BD81BDF89A30B52B
:101D8000F999FECF86E090E092BD81BDF89A20B52A
:101D9000932F80E0C22FD0E0C82BD92B81E0CD3229
:101DA000D807F0F1CCE2D1E09E0140E050E0809114
:101DB0003E0690913F068C179D0719F081E08093B5
:101DC000C005D0933F06C0933E06D0935006C09303
:101DD0004F066091090270910A0280910B02909166
:101DE0000C020E946E876FEF7FEF8FEF9FEF0E94D4
:101DF0006E87CA01B90128EE33E040E050E00E944E
:101E00001C8760934B0670934C0680934D0690930D
:101E10004E06D0935806C0935706DF91CF91089590
:101E2000C431D10508F6C4E1D0E024E130E040E05F
:101E300050E0BDCF1F920F920FB60F920BB60F92CC
:101E400011242F933F934F935F936F937F938F93BF
:101E50009F93AF93BF93EF93FF9340B1427090B1C4
:101E60001092C30580915E06481709F40AC1892FB4
:101E70008170442391F1882309F408C19FEF809178
:101E8000B305823091F180915605882309F44AC048
:101E90008091AB05882309F00CC18091C305992777
:101EA00087FD909520914F0630915006280F391FDD
:101EB0003093500620934F0681E02D32380708F00A
:101EC00009C12431310590F584E190E090935006EA
:101ED00080934F0624E130E029C0882309F4E0C054
:101EE00091E08091B305823071F68091C305181698
:101EF00074F49091690280916C02981798F49F5F36
:101F00009093690220914F06309150060FC08823AC
:101F100049F09091690280916B02891718F49150F1
:101F20009093690220914F063091500640935E06CF
:101F30008091D7058F3F29F08091D7058F5F8093DF
:101F4000D7058091D8058F3F29F08091D8058F5F04
:101F50008093D8058091E7059091E8058F5F9F4FAA
:101F600049F08091E7059091E80501969093E80586
:101F70008093E7058091AE05882351F08091AE05EE
:101F800081508093AE058091AE05882309F4A49812
:101F9000B90181E02D32380708F456C06CE271E0D7
:101FA0009B0140E050E080913E0690913F068617ED
:101FB000970719F081E08093C00570933F06609306
:101FC0003E067093500660934F066091090270912F
:101FD0000A0280910B0290910C020E946E876FEFB3
:101FE0007FEF8FEF9FEF0E946E87CA01B90128EE45
:101FF00033E040E050E00E941C8760934B067093F2
:102000004C0680934D0690934E069091C5059923FA
:1020100031F180917202981769F19F5F9F719093DF
:10202000C505FF91EF91BF91AF919F918F917F91E6
:102030006F915F914F913F912F910F900BBE0F9039
:102040000FBE0F901F9018952431310508F0A8CFCE
:1020500064E170E024E130E040E050E0A4CF8FEF95
:102060008093E4050E94A7249091C5058091720297
:10207000981799F61092E4050E94A7249091C5053F
:10208000CCCF20914F063091500652CF81E0809303
:10209000C3058091C4058F5F8093C40591E0EFCEA6
:1020A0008FEF8093C3058091C40581508093C40550
:1020B000E5CE9130C1F420914F0630915006295F52
:1020C0003F4F3093500620934F0681E02D32380762
:1020D00008F42CCF8CE291E09093500680934F0649
:1020E0002CE231E023CF9F3F09F01CCF20914F0617
:1020F00030915006275030403093500620934F06C1
:102100002431310508F012CFDFCE8F929F92AF922B
:10211000BF92CF92DF92EF92FF920F931F93DF93C4
:10212000CF93CDB7DEB760970FB6F894DEBF0FBE82
:10213000CDBF8091C90088618093C90083E38093FB
:10214000CC001092CD008091C80087FD33C28091F1
:10215000C90080688093C9008091C100886980931C
:10216000C1008FE18093C4001092C50090EC91B93A
:102170008CE382B987E384B995B99FEF97B988EF6B
:102180008AB98BE08BB982E08DB99EB910BA91BB48
:1021900088E183BB87EE84BB80E58CBD8DB5816013
:1021A0008DBD8CB581608CBD8CB58D7F8CBDF99952
:1021B000FECF85E090E092BD81BDF89A30B5F999E7
:1021C000FECF86E090E092BD81BDF89A20B5932FB6
:1021D00080E0022F10E0082B192B21E00D321207AE
:1021E00008F46CC40CE211E0980140E050E08091EA
:1021F0003E0690913F068017910719F081E0809389
:10220000C00510933F0600933E06109350060093BE
:102210004F066091090270910A0280910B02909121
:102220000C020E946E876FEF7FEF8FEF9FEF0E948F
:102230006E87CA01B90128EE33E040E050E00E9409
:102240001C8760934B0670934C0680934D069093C9
:102250004E0610935806009357061092800089E0AE
:102260008093810085E09DE09093890080938800B1
:10227000109285001092840082E080936F0080911C
:10228000700082608093700083E08093B000809340
:10229000B1008AEF8093B30084E398E090937608CE
:1022A00080937508F999FECF82E090E092BD81BDE0
:1022B000F89A80B5982F937090939C0582958170C1
:1022C0008093F905F999FECF87E090E092BD81BD3A
:1022D000F89A80B5882311F0813208F080E180936C
:1022E0000002F999FECF83E090E092BD81BDF89A9B
:1022F00080B58F7080937506F999FECF84E090E0E9
:1023000092BD81BDF89A80B58F7080936206F9996D
:10231000FECF88E090E092BD81BDF89A30B5F99982
:10232000FECF89E090E092BD81BDF89A20B5932F51
:1023300080E030E0282B392B2093510680913E0617
:1023400090913F06820F931F9C01220F232F221F83
:10235000330B31952827392745E25DEC4227532777
:10236000322F22273295330F307E42275327CA015E
:102370000024969587950794969587950794982FAE
:10238000802D8427952722EC3BE72827392785E6EF
:1023900094ED909343068093420650935B064093DE
:1023A0005A063093610620936006C9010024969571
:1023B00087950794969587950794982F802D822767
:1023C000932725E133EB28273927309356062093AE
:1023D00055068BEC98EA289FA001299F500D389F45
:1023E000500D1124F999FECF88E090E092BD81BD97
:1023F00050BDF894FA9AF99A7894F999FECF89E049
:1024000090E092BD81BD40BDF894FA9AF99A789413
:10241000F999FECF8AE090E092BD81BDF89A90B51F
:10242000892F8F7080935C0680915C06843010F059
:1024300010925C0692959F709F5F90935F068091CB
:102440005F06823018F482E080935F06F999FECF30
:102450008DE090E092BD81BDF89A60B5862F8C59D1
:10246000893C08F41BC360E87DE88BE590E0F894B4
:102470006093090270930A0280930B0290930C02FE
:10248000F999FECF8EE090E092BD81BDF89A40B5FB
:10249000493008F4FAC242E08CE080935906409338
:1024A0005206F999FECF8FE090E092BD81BDF89A77
:1024B00080B5853008F080E08093B405F999FECFAF
:1024C00080E190E092BD81BDF89A80B5853108F039
:1024D0008AE08093690280936A02F999FECF81E1D4
:1024E00090E092BD81BDF89A80B5982F9F7090932F
:1024F0006B0282958F70865F80936C029B3010F424
:10250000853130F084E080936B0280E180936C022F
:10251000F999FECF82E190E092BD81BDF89A80B535
:10252000823008F4D6C281E08093C105F999FECFCC
:1025300083E190E092BD81BDF89A90B5892F8150DA
:102540008F3008F096E0909372020E94525C78946B
:1025500000E010E01DC08091A2060E9442270E9468
:10256000A724C801849668E270E00E945B870E94FD
:10257000FA240E941B2480E10E947816C80187700B
:102580009070892B01F10F5F1F4F0C32110511F173
:10259000083208F7802F0E94FA240E948523DBCF9F
:1025A0008091CE008AE00E9478168091C80088232E
:1025B0000CF0CDCD8091C80087FDF2CF8091C8008E
:1025C00087FFF8CFEDCF0E9445220F5F1F4F0C32DF
:1025D0001105F1F60E9492240E94A7240E94452230
:1025E00080E00E945C1F882331F083E00E945C1F22
:1025F000882309F072C283E00E945C1F882309F4DB
:1026000030C28CE00E945C1F882309F42AC26E014C
:102610000894C11CD11CFF2421E1A22EB12CAC0EC8
:10262000BD1E9FE0E92E8601A0914206B0914306AF
:1026300040915A0650915B0680906006909061062A
:1026400060915506709156069D01220F232F221F7F
:10265000330B31952A273B27DA01509343064093E9
:102660004206A40180925A0650935B064B01709378
:1026700061066093600600247695679507947695C9
:1026800067950794762F602D682579256227732733
:10269000322F22273295330F307E622773277093B3
:1026A000560660935506CD01880F991F0196FC01CF
:1026B0006E9FC0016F9F900D7E9F900D1124F801B9
:1026C000908381830E5F1F4F0A151B0509F0BCCF55
:1026D000F60104C031960E171F0791F02081822F5A
:1026E00090E08F7090700D9724F0822F8F70808310
:1026F000282F2D3079F78E2F8C198F3009F0AFC12C
:1027000080E060E04F2D21E086010E94C95B85E5F5
:102710000E9406250E94A724F394F0E8FF1609F012
:1027200082CF0E9492248091C105882349F08DB503
:102730008E7F8DBD8CB58E7F8CBD8CB58D7F8CBD15
:102740008091A20680938D081092CE0810926107A6
:102750001092EA0781E08093F0071092F1078091D0
:102760008D086091CE084091EA072091F00704E3BC
:1027700018E00E94715B6091EA07C8010E94C55D84
:102780000E94545711E002E0F0E1CF2ED12CE5E099
:10279000AE2EB12C76E0E72EF12C0E9445228091DE
:1027A000A40583608093A4051092A5051092B3053B
:1027B00010936F0210937102009370021092BB0588
:1027C00080919D06873009F4BFC0883008F073C03F
:1027D000823009F4BFC0833008F087C0882309F431
:1027E000BFC0813009F4B9C00E9445228091AC0578
:1027F000882359F08091AC0581508093AC050E94EC
:10280000AB038091AC058823A9F78091BF0588238D
:1028100039F11092BF0580919C05882381F42091A5
:102820003E0630913F068091570690915806281732
:10283000390729F08091DB08882309F460C0909162
:10284000690280916A02891759F090936A02F99996
:10285000FECFD2BCC1BC90BDF894FA9AF99A789494
:102860008091C005882351F01092C005F8947894A7
:1028700080913E0690913F060E94BA2E0E945457C6
:10288000882309F08ACF80919D06863009F0ACCF6D
:1028900081E00E94881F882309F4A6CF80E00E946F
:1028A0005C1F882309F4A0CF0E9492240E94A724D1
:1028B000E0E0F0EF19948C3009F4ACC08D3048F4AE
:1028C000883009F456C08B3009F08ECF0E94A05298
:1028D00064CF8E3009F44AC08E3008F444C08F3083
:1028E00009F082CF0E94145F58CF843081F1843088
:1028F00040F1853009F078CF0E94EA674ECF85E23B
:102900000E94852380913E0690913F069093580641
:102910008093570690913E0680913F06F999FECF2D
:10292000B2BCA1BC80BDF894FA9AF99A7894F9994E
:10293000FECFF2BCE1BC90BDF894FA9AF99A789473
:102940007ECF0E945D4F29CF0E94144C26CF0E945B
:102950001A4423CF0E94CD7A20CF0E94AF7D1DCF95
:102960000E94F4181ACF0E94F07917CF0E94A0336A
:1029700014CF0E9492240E9445228091AC058823A6
:1029800059F08091AC0581508093AC050E94AB0357
:102990008091AC058823A9F78091BF05882331F188
:1029A0001092BF0580919C05882379F420913E0602
:1029B00030913F06809157069091580628173907A5
:1029C00021F08091DB08882341F190916902809188
:1029D0006A02891759F090936A02F999FECFD2BC26
:1029E000C1BC90BDF894FA9AF99A78948091C00588
:1029F000882351F01092C005F894789480913E0697
:102A000090913F060E94BA2E0E945457882309F4E1
:102A1000B2CFC3CE0E94F819C0CE85E20E948523B2
:102A200080913E0690913F069093580680935706FA
:102A300090913E0680913F06F999FECFB2BCA1BCB1
:102A400080BDF894FA9AF99A7894F999FECFF2BC7D
:102A5000E1BC90BDF894FA9AF99A7894B6CFE082E6
:102A600039CE87E10E945C1F882309F45CCE85E0A3
:102A70000E945C1F882309F456CE1092C10582E1A2
:102A800090E061E00E9450034ECE242F30E0C90157
:102A9000880F991F820F931F880FFFCC772767FD40
:102AA0007095872F972F20E737E140E050E00E9494
:102AB0001C8760587247844A9F4FD9CC0431110556
:102AC00008F092CB04E110E024E130E040E050E077
:102AD0008ECB882309F02ACD26CD10929C0510922A
:102AE000F9052091F905F999FECF82E090E092BDB9
:102AF00081BD822F90E08170907082959295907F39
:102B00009827807F982780BDF894FA9AF99A78944C
:102B10000E94525C1092750610926206F999FECFDF
:102B200083E090E092BD81BD10BCF894FA9AF99AC6
:102B30007894F999FECF84E090E092BD81BD10BCFD
:102B4000F894FA9AF99A789488E790E090933F067F
:102B500080933E06F999FECF85E090E092BD81BD5D
:102B600010BCF894FA9AF99A7894F999FECF86E015
:102B700090E092BD81BD88E780BDF894FA9AF99AF9
:102B8000789480E18093000220910002F999FECFB1
:102B900087E090E092BD81BD20BDF894FA9AF99A41
:102BA000789410925C0688E080935F0630915F060F
:102BB00020915C06F999FECF8AE090E092BD81BD3C
:102BC000832F90E0019782959295907F9827807F40
:102BD0009827282B20BDF894FA9AF99A7894F999B5
:102BE000FECF8DE090E092BD81BD10BCF894FA9AC2
:102BF000F99A7894F89480E89DE8ABE5B0E080938A
:102C0000090290930A02A0930B02B0930C027894ED
:102C10008CE08093590682E080935206F999FECFAA
:102C20008EE090E092BD81BD82E080BDF894FA9A7A
:102C3000F99A78941092B405F999FECF8FE090E05C
:102C400092BD81BD10BCF894FA9AF99A78948AE002
:102C50008093690280936A02F999FECF80E190E047
:102C600092BD81BD8AE080BDF894FA9AF99A789471
:102C700084E080936B0280E180936C02F999FECF2F
:102C800081E190E092BD81BD84E680BDF894FA9A1E
:102C9000F99A789481E08093C105F999FECF82E199
:102CA00090E092BD81BD10BCF894FA9AF99A78949C
:102CB00086E08093720220917202F999FECF83E13F
:102CC00090E092BD81BD20BDF894FA9AF99A78946B
:102CD00010E082E20E944F2483E20E944F240E946F
:102CE000A72482E30E9478161F5F183291F719CD4E
:102CF00020EA3FE0E22FF32F3197F1F78A95D1F7E1
:102D00000895882309F41EC09AEF20EA3FE0E22FDD
:102D1000F32F3197F1F79A95D1F7E22FF32F3197EF
:102D2000F1F79A95D1F7E22FF32F3197F1F79A95B2
:102D3000D1F7E22FF32F3197F1F79A95D1F7815020
:102D400009F0E5CF08951F920F920FB60F920BB6C0
:102D50000F9211242F933F938F939F93EF93FF93A1
:102D60009091C600892F8A5F823080F19C3FA1F14B
:102D7000983FC1F18091CF05E82FF0E0EA58F94F74
:102D800090838F5F8093CF058091CF058F71809363
:102D9000CF059091CF058091CE05981751F4809181
:102DA000CE058F5F8093CE058091CE058F71809385
:102DB000CE05FF91EF919F918F913F912F910F90B1
:102DC0000BBE0F900FBE0F901F9018958091C605F7
:102DD00081608093C605EDCF8091C60582608093A7
:102DE000C605E7CF8091390690913A0690939A05EF
:102DF0008093990510923A061092390680919C05AD
:102E00008230B9F68091D1059091D205892BE9F4F1
:102E1000109296021092C8058091B405882329F576
:102E20008091990590919A05969587959093D205F2
:102E30008093D1058091AC058F5F8093AC05809124
:102E4000C8058E5F8093C805B4CF5C988091AC05AF
:102E50008F5F8093AC058091C9059091CA0501965A
:102E60009093CA058093C905D7CF2091B40530E06F
:102E70002F5F3F4FC901880F991F880F991F820F3D
:102E8000931F9093D2058093D105D4CF10926B06F7
:102E90001092740608951F93CF93DF93EC01142FC3
:102EA0006F777885772309F44CC0462F50E08881EE
:102EB00090E08F7790704817590779F121E030E062
:102EC0000DC0D901FE01E20FF31F808190E08F77E2
:102ED00090702F5F3F4F8417950709F1271788F3EC
:102EE000272F2F5F293030F128E0922F822F915029
:102EF000FE01E80FF11DDE01A90FB11D8C91808349
:102F0000892F9923A1F71536C0F480E0862B88839A
:102F10002887DF91CF911F910895A0E0B0E015368A
:102F200070F480E0AC0FBD1F862B8C93DF91CF91A6
:102F30001F9108952223C9F6E6CF80E8E7CF80E805
:102F4000F1CF91E081E021E0D2CFCF93DF93EC018C
:102F500038853323B9F06F7770E0888190E08F7700
:102F600090706817790789F0FE0120E008C0818120
:102F700090E08F77907031966817790739F02F5F5E
:102F80002317A8F3DF91CF91089520E0323068F045
:102F9000922F9F5FFE01E20FF11DDE01A90FB11D0F
:102FA0008C918083292F9317A0F331503887DF91BC
:102FB000CF910895282F909162068091C00085FFDF
:102FC000FCCF90699093C6008091C00085FFFCCF34
:102FD000822F8F778093C60027FD09C090919502BC
:102FE0008091C00085FFFCCF9093C600089590911A
:102FF00093028091C00085FFFCCF9093C600089596
:10300000282F909162068091C00085FFFCCF9068C8
:103010009093C6008091C00085FFFCCF822F8F77F0
:103020008093C60027FD09C0909195028091C00051
:1030300085FFFCCF9093C6000895909193028091F4
:10304000C00085FFFCCF9093C6000895982F809113
:10305000C00085FFFCCF9093C60080E090E008950B
:103060009091CE058091CF0520E030E0981711F0C7
:1030700021E030E0C90108959091CE058091CF05FF
:103080009817D1F3F8949091CE05E92FF0E0EA5823
:10309000F94F80819F5F9093CE059091CE059F71EF
:1030A0009093CE05789490E0089590916206809177
:1030B000C00085FFFCCF906B9093C6008091C0004C
:1030C00085FFFCCF8BE78093C6008091C00085FF11
:1030D000FCCF1092C600089590919E058913089523
:1030E00080E00E9412448FEF80939E0508951F9305
:1030F000182F962F6623B9F060E080919E058F3FD0
:1031000009F061E0953648F4812F895140E00E9432
:10311000FB4310939E051F910895812F895141E033
:103120000E94FB43F6CF80919E051817A1F780E01F
:103130000E9412448FEF80939E05EDCF80919C05F5
:103140008230E9F08091C00085FFFCCF8CEF809346
:10315000C600909162068091C00085FFFCCF906B05
:103160009093C6008091C00085FFFCCF8BE78093D1
:10317000C6008091C00085FFFCCF1092C600089564
:103180009091CE058091CF059817C9F09091CE050A
:103190008091CF059817D1F3F8948091CE05E82F50
:1031A000F0E0EA58F94FE0818F5F8093CE0580917F
:1031B000CE058F718093CE057894E7FD03C0E0E0E3
:1031C0008E2F08954E2F42954F704F30C9F32E2FFA
:1031D00030E02F7030708091750690E02817390725
:1031E00071F74093C705ECCF0F931F930E94F2270E
:1031F000809175060E9442270E94452284E60E9423
:1032000078160E94452284E60E9478160E94452284
:103210008FEF80939E050FEF0E9445220E945F0E64
:103220000E945457882309F05BC09091CE0580918D
:10323000CF05981789F39091CE058091CF05981707
:10324000D1F3F8948091CE05E82FF0E0EA58F94FD9
:1032500010818F5F8093CE058091CE058F71809312
:10326000CE05789417FD91C08091C705883009F488
:1032700068C0893089F617FD4CC09091CE058091C9
:10328000CF059817D1F3F8948091CE05E82FF0E0A0
:10329000EA58F94FE0818F5F8093CE058091CE058B
:1032A0008F718093CE057894EE2309F463C060E0BB
:1032B00080919E058F3F09F061E0E53608F08FC0F0
:1032C000812F895140E00E94FB4310939E050E948C
:1032D00045220E945F0E0E945457882309F4A5CF0F
:1032E000909162068091C00085FFFCCF906B909317
:1032F000C6008091C00085FFFCCF8BE78093C6009D
:103300008091C00085FFFCCF1092C6001F910F91E5
:1033100008959091CE058091CF059817D1F3F89438
:103320008091CE05E82FF0E0EA58F94F10818F5FC9
:103330008093CE058091CE058F718093CE057894D1
:103340009CCF17FD34C09091CE058091CF05981782
:10335000D1F3F8948091CE05E82FF0E0EA58F94FC8
:10336000E0818F5F8093CE058091CE058F71809331
:10337000CE05789480919E05181709F04DCF80E016
:103380000E94124400939E0547CF412F42954F70F3
:103390004F3059F1212F30E02F7030708091750639
:1033A00090E02817390709F11092C70535CF9091A1
:1033B000CE058091CF059817D1F3F8948091CE0572
:1033C000E82FF0E0EA58F94F10818F5F8093CE0527
:1033D0008091CE058F718093CE057894B4CF812FE4
:1033E000895141E00E94FB4370CF4093C7053CCF19
:1033F000CF92DF92EF92FF920F931F9380914D0730
:10340000817080934D0780914D07809333060E9411
:10341000922480914D07882309F055C40E94A72467
:103420008BE090E00E944903809397028CE090E04B
:103430000E944903809398028091CE089091EA07F8
:10344000880F880F880F890F8093CC058091A20682
:103450009091CC058295807F890F8093CC058091D7
:10346000CE088093CD051092BB05EE2400E0DD244C
:10347000D394A2E0CA2E0E9445220E945F0E809142
:10348000DB08882309F0B5C0D09232060E94545759
:10349000882309F0B1C29091CE058091CF0598178D
:1034A00009F19091CE058091CF059817D1F3F8944A
:1034B0008091CE05E82FF0E0EA58F94F10818F5F38
:1034C0008093CE058091CE058F718093CE05789440
:1034D00017FD67C18091C705883009F476C189302E
:1034E00009F4E9C1002309F073C080916B068823B9
:1034F00049F480917406882329F48091DB0888239D
:1035000009F433C388E00E94721F882309F4D3C0F2
:103510008091BB05882309F4C7C0823009F0D0C070
:1035200010E0812F0E949320882309F46FC0712F2F
:103530007F7760917406662309F442C3472F50E0F9
:1035400080916C0690E08F7790704817590709F4C6
:10355000A1C021E030E00EC0D901F901E459F94FD2
:10356000808190E08F7790702F5F3F4F4817590709
:1035700009F492C0261780F3262F2F5F293008F414
:103580008FC028E0922FE22F01C0E92F9150F0E088
:10359000E459F94FA92FB0E0A459B94F8C91808319
:1035A000992399F770936C062093740680916C06AA
:1035B0008F7780937C081F5F1D3009F0B2CF88E0C1
:1035C0000E94881F882309F0E8C20E94625A00E026
:1035D00087E10E94B11F882309F042C00E94405A2F
:1035E0000E9445220E945F0E8091DB08882309F427
:1035F0004BCF0E946257882309F0FEC180913206AA
:10360000813009F4F4C11092320645CF812F0E9417
:103610002721882381F240917406442361F2812F8F
:103620008F77282F30E050916C06852F90E08F77B0
:1036300090702817390709F467C2ADE6B6E0E0E0FC
:1036400008C08D9190E08F7790708217930709F4EE
:103650005CC2EF5FE417A8F35F7750937C08ABCFB1
:1036600080914D078F5F80934D0780914D0781704A
:1036700080934D0780914D078093330680E00E9430
:103680001B2480914D07882309F4A8CF80E00E9475
:103690008523A4CFA0E0B0E0A459B94F7C9386CF96
:1036A000222309F06FCF7ECFC092BB050E949B29D9
:1036B00084E20E9485238091BB05823009F430CFDB
:1036C00084E10E945C1F882309F06FC200E085E15D
:1036D0000E945C1F882309F0C2C110E0812F0E9464
:1036E000AD20882309F4C6C15091CD05550F550F63
:1036F000550F510F5F7740916B06442309F464C264
:10370000652F70E08091630690E08F779070681766
:10371000790709F4EFC121E030E00EC0D901F901C9
:10372000ED59F94F808190E08F7790702F5F3F4F78
:103730008617970709F4E0C1241780F34F5F4930DB
:1037400008F4DEC148E0E42F942F01C0E42F41507B
:10375000F0E0ED59F94FA42FB0E0AD59B94F8C917D
:103760008083442399F7492F5093630640936B0657
:103770004093CB0501E01F5F183009F0AFCF002365
:1037800009F423CF809163068F778093CC058091D5
:10379000A2069091CC058295807F890F8093CC05FD
:1037A00014CF412F42954F704F3009F4CCC1212FD7
:1037B00030E02F7030708091750690E0281739073F
:1037C00009F4C1C11092C70556CE17FD5CC0909197
:1037D000CE058091CF059817D1F3F8948091CE054E
:1037E000E82FF0E0EA58F94FE0818F5F8093CE0533
:1037F0008091CE058F718093CE057894002309F0D7
:10380000A5C140919702141748F0842F90E00F96BD
:10381000212F30E0821793070CF0DAC14091980213
:10382000141708F462CE842F90E00C96212F30E01C
:10383000821793070CF459CE50917406552309F45E
:1038400054CE141B1F77212F30E080916C0690E03E
:103850008F7790702817390709F479C2ADE6B6E082
:1038600040E008C08D9190E08F779070281739075D
:1038700009F46EC24F5F4517A8F380916C068F77ED
:1038800080937C0832CE9091CE058091CF05981719
:10389000D1F3F8948091CE05E82FF0E0EA58F94F83
:1038A00010818F5F8093CE058091CE058F718093BC
:1038B000CE0578948CCF17FD82C09091CE05809173
:1038C000CF059817D1F3F8948091CE05E82FF0E05A
:1038D000EA58F94FF0808F5F8093CE058091CE0536
:1038E0008F718093CE057894002309F071CE4091BA
:1038F0009702141748F0842F90E00F96212F30E0A4
:10390000821793070CF095C140919802141708F4A0
:10391000ECCD842F90E00C96212F30E08217930796
:103920000CF4E3CD212F241B2F7710917406112363
:1039300009F43FC2622F70E080916C0690E08F77AF
:1039400090706817790709F41DC241E050E00EC07D
:10395000DA01FA01E459F94F808190E08F77907095
:103960004F5F5F4F6817790709F40EC2411780F364
:10397000E12FEF5FE93008F4CFC1E8E09E2F4E2F32
:1039800001C0E92F9150F0E0E459F94FA92FB0E0C0
:10399000A459B94F8C918083992399F7E42F84E639
:1039A0008F1508F4FCC180E0822B80936C06E093B5
:1039B000740680916C068F7780937C0896CD9091E9
:1039C000CE058091CF059817D1F3F8948091CE055C
:1039D000E82FF0E0EA58F94F10818F5F8093CE0511
:1039E0008091CE058F718093CE05789466CF0E942A
:1039F0005457882309F407CE80917C088093770878
:103A000081E08093F0078091CE0880936107109247
:103A1000F10780918D086091CE084091EA072091CE
:103A2000F00704E318E00E94715B6091EA07C801A7
:103A30000E94C55DEE2061F08BE090E060919702FE
:103A40000E9450038CE090E0609198020E94500325
:103A50001F910F91FF90EF90DF90CF900895D0923B
:103A60006107809161078093CD0581E00E94BD23AD
:103A700001E033CE812F0E940D21882309F47BCEF3
:103A80008091CD0540916B06442309F471CE880FD7
:103A9000880F880F810F8F77282F30E08091630681
:103AA00090E08F7790702817390709F423C1A4E6B6
:103AB000B6E0E0E0EF5FE41708F05ACE8D9190E0B9
:103AC0008F77907082179307A9F7423078F09E2F76
:103AD00001C0E92F9F5FF0E0ED59F94FA92FB0E049
:103AE000AD59B94F8C918083941798F3415040930E
:103AF0006B063ECEA0E0B0E0AD59B94F5C9338CE36
:103B0000442309F020CE30CEE0E0423078F09E2F02
:103B100001C0E92F9F5FF0E0E459F94FA92FB0E011
:103B2000A459B94F8C918083941798F3842F8150B6
:103B300080937406882309F43ECD50916C065F771C
:103B400050937C0838CD4093C705C4CC013009F4AC
:103B5000BEC08CE10E941B241093980280914D07F7
:103B600080933306EE24E394C0CC0E945C1F88232C
:103B700009F4C8CC89E00E94721F882309F0B3C001
:103B80008AE00E94721F882309F4BCCC109233068D
:103B90008CE10E94A12302E01BCD1092BB0584E2C0
:103BA0000E941B240E949B2910CD109261078091D6
:103BB00061078093CD0588E00E94BD2301E087CD99
:103BC00091E0E1E021E0E2CC41E0E1E091E0BFCD35
:103BD00050916B065523E1F0141B1F77212F30E025
:103BE0008091630690E08F7790702817390709F469
:103BF00097C0A4E6B6E040E008C08D9190E08F77D2
:103C000090708217930709F48CC04F5F4517A8F393
:103C10005093CB05809163068F778093CC0580917C
:103C2000A2069091CC058295807F890F8093CC0568
:103C30005CCC212F241B2F7760916B06662309F43F
:103C4000B4C0022F10E08091630690E08F779070EF
:103C50000817190709F450C041E050E00EC0DA011E
:103C6000FA01ED59F94F808190E08F7790704F5FA6
:103C70005F4F8017910709F441C0461780F36F5FCB
:103C8000693008F445C068E0962F462F01C0692FBF
:103C90009150E62FF0E0ED59F94FA92FB0E0AD5962
:103CA000B94F8C918083992391F7642F84E68F1507
:103CB00008F473C080E0822B8093630660936B06E8
:103CC0006093CB05A7CF80E00E948523A7CB8BE133
:103CD0000E941B241093970280914D078093330616
:103CE000EE24E39402CC109233068BE10E94A123D0
:103CF00001E06ECCE0E0E9CEA0E0B0E084E68F1514
:103D000008F44FC080E0AD59B94F822B8C93D8CFC7
:103D1000662309F0B9CFCACFEE2309F02FCE3FCEEC
:103D200040E0523080F0942F01C0492F9F5FE42F74
:103D3000F0E0ED59F94FA92FB0E0AD59B94F8C9192
:103D40008083951790F3515050936B0661CF40E0FC
:103D5000523080F0942F01C0492F9F5FE42FF0E094
:103D6000E459F94FA92FB0E0A459B94F8C91808341
:103D7000951790F3852F815080937406882309F45A
:103D8000B4CB7BCDA0E0B0E084E68F1560F080E09E
:103D9000A459B94F822B8C9370CD80E88CCF80E8EA
:103DA00003CE80E8B0CF80E8F3CF91E061E041E05E
:103DB0006FCF91E0E1E041E0E5CD80919C0581305D
:103DC00009F05F98089599B1991F9927991F8091DB
:103DD000D305882311F4992321F49093D30580E02F
:103DE00008959093D30581E0089599B1991F99277B
:103DF000991F8091D405882311F0992321F0909385
:103E0000D40580E008951092D40581E008958AB128
:103E1000806F8AB98BB18F708BB908958AB18F701A
:103E20008AB98BB18F708BB9089580919C058823D6
:103E300021F45C9881E00E9478165F9A0895AC01A5
:103E4000F89428980000000000000000289A20E064
:103E500030E01EBC0DB407FEFDCF8EB5FA01E20FB7
:103E6000F31F80832F5F3F4F2330310591F7789404
:103E7000089516980895169A089520B126952695C6
:103E80002F70822F90E02695322F3695369522702E
:103E9000322B880F991F282F2470322B880F991FDF
:103EA000880F991F8870382B8FE0831B089580B18D
:103EB000869586958F700895282F883188F4E82F8D
:103EC000E695E695E695F0E0ED55F94F808190E0B6
:103ED000277002C0959587952A95E2F7817008951D
:103EE00080E00895282F883188F4E82FE695E6953C
:103EF000E695F0E0E656F94F808190E0277002C029
:103F0000959587952A95E2F78170089580E0089548
:103F1000282F883188F4E82FE695E695E695F0E0BD
:103F2000E256F94F808190E0277002C09595879501
:103F30002A95E2F78170089580E008958091A306A4
:103F4000882321F48091A406882319F090E0892F1A
:103F5000089590E08091A5068823C9F791E0892F04
:103F60000895282F8831A0F4482F46954695469508
:103F7000277081E090E0382F01C0330F2A95EAF7CF
:103F8000A42FB0E0FD01E656F94F8081832319F498
:103F900020E0822F0895232F30E020953095AD55F5
:103FA000B94F8C9190E028233923232B89F7342FA4
:103FB0003F5F832F63E00E943B87E92FF0E0ED55E0
:103FC000F94F8081882321F720E0832F8F5F0E94A3
:103FD0003B87E92FF0E0ED55F94F80818823C9F642
:103FE00021E0D7CF8091D6051092D605089580E0C4
:103FF0000895382F883100F5282F277081E090E050
:10400000982F01C0990F2A95EAF7832F86958695F8
:104010008695A82FB0E0FD01E656F94F80818923EF
:1040200069F4FD01E256F94F8081892371F4AD55A1
:10403000B94F8C91982339F480E00895832F0E9422
:10404000022782E0089583E00895832F0E94592972
:1040500081E0089520E030E0F901EF55FD4F408107
:10406000483188F4E42FE695E695E695F0E0E656CB
:10407000F94F808190E0477002C0959587954A95E9
:10408000E2F780FD07C02F5F3F4F2A30310521F74F
:1040900080E00895822F8F5F089520E030E0F901DD
:1040A000E555FD4F4081483188F4E42FE695E695CB
:1040B000E695F0E0E656F94F808190E0477002C047
:1040C000959587954A95E2F780FD07C02F5F3F4F92
:1040D0002D30310521F780E00895822F8F5F0895FC
:1040E00020E030E0F901E756FD4F4081483188F487
:1040F000E42FE695E695E695F0E0E656F94F8081E7
:1041000090E0477002C0959587954A95E2F780FD4B
:1041100007C02F5F3F4F2830310521F780E0089519
:10412000822F8F5F0895E82FF0E0E555FD4F208145
:10413000283188F4E22FE695E695E695F0E0E6561C
:10414000F94F808190E0277002C0959587952A9558
:10415000E2F78170089580E00895E82FF0E0E756D7
:10416000FD4F2081283188F4E22FE695E695E6950B
:10417000F0E0E656F94F808190E0277002C09595F7
:1041800087952A95E2F78170089580E0089520E0F0
:1041900030E0F901E555FD4F4081483188F4E42FC6
:1041A000E695E695E695F0E0E256F94F808190E0DD
:1041B000477002C0959587954A95E2F780FD07C044
:1041C0002F5F3F4F2D30310521F780E00895822F7A
:1041D0008F5F089520E030E0F901E756FD4F408100
:1041E000483188F4E42FE695E695E695F0E0E2564E
:1041F000F94F808190E0477002C0959587954A9568
:10420000E2F780FD07C02F5F3F4F2830310521F7CF
:1042100080E00895822F8F5F0895E82FF0E0E75641
:10422000FD4F2081283188F4E22FE695E695E6954A
:10423000F0E0E256F94F808190E0277002C095953A
:1042400087952A95E2F78170089580E00895E82F18
:10425000F0E0E555FD4F2081283188F4E22FE69506
:10426000E695E695F0E0E256F94F808190E0277000
:1042700002C0959587952A95E2F78170089580E0B0
:10428000089520E030E0522FF901E555FD4F4081BF
:10429000483188F4E42FE695E695E695F0E0ED5593
:1042A000F94F808190E0477002C0959587954A95B7
:1042B000E2F780FD06C02F5F3F4F2D30310519F723
:1042C0005FEF852F089520E030E0F901E555FD4FBF
:1042D0004081483188F4E42FE695E695E695F0E0D4
:1042E000ED55F94F808190E0477002C09595879514
:1042F0004A95E2F780FD07C02F5F3F4F2D30310513
:1043000021F780E00895822F8F5F089520E030E04C
:10431000F901E756FD4F4081483188F4E42FE695D6
:10432000E695E695F0E0ED55F94F808190E0477015
:1043300002C0959587954A95E2F780FD07C02F5FEB
:104340003F4F2830310521F780E00895822F8F5F9D
:104350000895A9E9B2E02C91283188F4E22FE6957E
:10436000E695E695F0E0ED55F94F808190E02770F5
:1043700002C0959587952A95E2F780FD07C01196B2
:1043800082E0A13AB80739F780E0089581E0089506
:10439000CF93DF93A9E9B2E050E040E010C0C256ED
:1043A000D94F888190E002C0959587952A95E2F7CC
:1043B00080FD5F5F119682E0A13AB80701F19C9100
:1043C0009831C0F7892F869586958695C82FD0E0BD
:1043D000292F30E027703070FE01ED55F94F8081B4
:1043E00090E0022E02C0959587950A94E2F780FF2F
:1043F000D6CF4F5F119682E0A13AB80701F751304E
:1044000021F080E0DF91CF91089580E04730D1F72F
:1044100081E0F8CF382F3F5F3830D8F4E32FF0E059
:10442000E756FD4F20812831B0F7E22FE695E6955B
:10443000E695F0E0ED55F94F808190E0277002C0DD
:10444000959587952A95E2F780FFE5CF832F8F5FBB
:10445000089580E00895E82FF0E0E756FD4F2081B1
:10446000283188F4E22FE695E695E695F0E0ED55E3
:10447000F94F808190E0277002C0959587952A9525
:10448000E2F78170089580E00895CF92DF92EF9275
:10449000FF920F931F93DF93CF9300D000D0CDB73F
:1044A000DEB710929A0610929E0610929B0610920A
:1044B0009F0610929C061092A0068091D7058A3024
:1044C00078F426960FB6F894DEBF0FBECDBFCF911D
:1044D000DF911F910F91FF90EF90DF90CF900895A3
:1044E0001092D7051698F894289800000000000054
:1044F0000000289A7E010894E11CF11CF701A4E059
:10450000CA2ED12CCC0EDD1E1EBC0DB407FEFDCF75
:104510008EB58193EC15FD05B9F778948091A306CB
:104520008C838091A4068D838091A5068E8360E0A4
:1045300070E001E010E0E62FE695E695E695F0E004
:10454000CB0187709070980102C0220F331F8A95AB
:10455000E2F7C901AF014D55594FD701AE0FBF1F4B
:104560003C91EA55F94F2081232B28238095FA01AD
:1045700030818323282B20836F5F7F4F6831710543
:10458000D1F620B1269526952F70822F90E02695A2
:10459000322F369536952270322B880F991F282F8F
:1045A0002470322B880F991F880F991F8870382B21
:1045B0008FE0831B982F96959093A2068093980680
:1045C000169A40E050E0DA01AA55B94FF701E40F1E
:1045D000F51F80818C93F601E40FF51F2081FA010D
:1045E000ED55F94F9081FA01E656F94F822F8095EB
:1045F00089238083FA01E256F94F909592239083A4
:104600004F5F5F4F43305105F1F690B19695969507
:104610009F708091DB08882361F48091960689174A
:1046200021F01092D805909396068091D8058E3D82
:1046300030F090939706809197068093960680912C
:10464000A30690E0969587959695879581708093BF
:10465000AB050E94A72435CF482FE82FF0E0E7569E
:10466000FD4FE081E83120F58E2F86958695869561
:10467000A82FB0E02E2F30E027703070FD01E256F9
:10468000F94F808190E0022E02C0959587950A949B
:10469000E2F780FD0DC0AD55B94F8C9190E002C09E
:1046A000959587952A95E2F780FF02C080E00895EE
:1046B000641749F1E62FF0E0E756FD4F608168315D
:1046C00010F5862F869586958695A82FB0E070E028
:1046D00067707070FD01E256F94F808190E0062E00
:1046E00002C0959587950A94E2F780FD0CC0AD5500
:1046F000B94F8C9190E002C0959587956A95E2F745
:1047000080958170089581E00895282F8832C0F443
:10471000E82FE695E695E695F0E0277081E090E0D9
:1047200001C0880F2A95EAF7DF01A752BA4F2C91F2
:10473000282B2C93E252FA4F80952081822380838C
:104740000895282F8832C0F4E82FE695E695E6957F
:10475000F0E0277081E090E001C0880F2A95EAF729
:10476000DF01A252BA4F2C91282B2C93E752FA4F1B
:10477000809520818223808308958832B8F4E82FC1
:10478000E695E695E695F0E0877021E030E001C01F
:10479000220F8A95EAF7DF01A252BA4F8C91822B41
:1047A0008C93E752FA4F8081822B80830895282FC3
:1047B000883210F560FD21C0822F869586958695FA
:1047C000482F50E0277081E090E0382F01C0330F70
:1047D0002A95EAF7232FFA01E752FA4F832F8095A3
:1047E00090818923808361FD1FC0FA01E252FA4F54
:1047F00020958081822380830895822F86958695D7
:104800008695482F50E0277081E090E0382F01C056
:10481000330F2A95EAF7232FFA01E752FA4F8081E6
:10482000832B808361FFE1CFFA01E252FA4F80814E
:10483000822B80830895282F8832C8F4E82FE695CC
:10484000E695E695F0E0277081E090E002C0880FE1
:10485000991F2A95E2F78095DF01A752BA4F2C9154
:1048600028232C93E252FA4F2081822380830895DB
:10487000282F883298F4E82FE695E695E695F0E043
:10488000E252FA4F277081E090E002C0880F991F32
:104890002A95E2F780952081822380830895282F2E
:1048A000883290F4E82FE695E695E695F0E0E75239
:1048B000FA4F277081E090E002C0880F991F2A9577
:1048C000E2F72081282720830895E82F883298F482
:1048D000282F277081E090E002C0880F991F2A9549
:1048E000E2F7E695E695E695F0E0E252FA4F208190
:1048F0002823822F089520E0822F0895982F9695DF
:1049000096959695E9EDF5E0E90FF11D208130E0EF
:10491000877002C0359527958A95E2F7217030702F
:10492000C90108951092DD051092DC051092DB0597
:104930001092DA051092D9051092E2051092E10565
:104940001092E0051092DF051092DE050895F894AC
:10495000179860E070E0FB01E752FA4F5081FB01CD
:10496000E252FA4F3081232F25238091E3054091B5
:10497000E405922F90958323852B98232423922B53
:104980009EBD0DB407FEFDCF6F5F7F4F6530710593
:1049900011F7179A78940895E9EDF5E0AEEDB5E0DA
:1049A00080819D91892B819385E0EE3DF807C1F7C9
:1049B0000895E9EDF5E0AEEDB5E09D91909580812B
:1049C0008923819385E0EE3DF807B9F70895E9ED75
:1049D000F5E0AEEDB5E020819C91892F822319F09E
:1049E0009095922390831D92319685E0EE3DF807D5
:1049F00091F70895E8EBF2E0E80FF11D808108954A
:104A0000E0EEF2E0E80FF11D808108959091D90564
:104A100098279093D9059091DA0598279093DA0515
:104A20009091DB0598279093DB059091DC05982702
:104A30009093DC059091DD0598279093DD0508950E
:104A4000CF93DF93F8941798C0E0D0E0C0FF24C064
:104A50006093E405FE01E752FA4F5081FE01E252F5
:104A6000FA4F3081232F25238091E3054091E405FF
:104A7000922F90958323852B98232423922B9EBDE0
:104A80000DB407FEFDCF2196C530D105F9F6179A72
:104A90007894DF91CF9108950E940402692F80934A
:104AA000E405D8CFE82FF0E0E05DFC4FE081E8328C
:104AB00098F42E2F277081E090E002C0880F991F94
:104AC0002A95E2F7E695E695E695F0E0E252FA4F90
:104AD00020812823822F089520E0822F0895E82F37
:104AE0008150883010F080E00895F0E0E85BFC4FE2
:104AF0002081E22FE695E695E695F0E0E752FA4F41
:104B0000808190E0277002C0959587952A95E2F7FD
:104B100081700895803110F080E00895E82FF0E072
:104B2000E759FC4F2081E22FE695E695E695F0E007
:104B3000E752FA4F808190E0277002C095958795E3
:104B40002A95E2F781700895803118F020E0822FD5
:104B50000895E82FF0E0E759FC4FE081E832B0F724
:104B60002E2F277081E090E002C0880F991F2A95B0
:104B7000E2F7E695E695E695F0E0E252FA4F2081FD
:104B80002823822F0895E82F8150883018F020E0E4
:104B9000822F0895F0E0E85BFC4FE081E832B8F73F
:104BA0002E2F277081E090E002C0880F991F2A9570
:104BB000E2F7E695E695E695F0E0E252FA4F2081BD
:104BC0002823822F0895E82FF0E0E75BFC4F208137
:104BD000283210F560FD21C0822F86958695869536
:104BE000482F50E0277081E090E0382F01C0330F4C
:104BF0002A95EAF7232FFA01E752FA4F832F80957F
:104C000090818923808361FD1FC0FA01E252FA4F2F
:104C100020958081822380830895822F86958695B2
:104C20008695482F50E0277081E090E0382F01C032
:104C3000330F2A95EAF7232FFA01E752FA4F8081C2
:104C4000832B808361FFE1CFFA01E252FA4F80812A
:104C5000822B80830895803108F00895E82FF0E0DA
:104C6000E759FC4F20812832C0F7E22FE695E69500
:104C7000E695F0E0277081E090E001C0880F2A956A
:104C8000EAF7DF01A252BA4F2C91282B2C93E7525E
:104C9000FA4F80952081822380830895883108F01F
:104CA0000895E82FF0E0EF5AFC4F20812832C0F73A
:104CB000E22FE695E695E695F0E0277081E090E03A
:104CC00001C0880F2A95EAF7DF01A252BA4F2C9152
:104CD000282B2C93E752FA4F8095208182238083E2
:104CE0000895E82F8150883008F00895F0E0E85BDF
:104CF000FC4F20812832C8F7E22FE695E695E6952D
:104D0000F0E0277081E090E001C0880F2A95EAF773
:104D1000DF01A252BA4F2C91282B2C93E752FA4F65
:104D2000809520818223808308958D3008F0089536
:104D3000E82FF0E0E05DFC4F20812832C0F7E22F41
:104D4000E695E695E695F0E0277081E090E001C0F9
:104D5000880F2A95EAF7DF01A252BA4F2C91282B2F
:104D60002C93E752FA4F8095208182238083089507
:104D7000803108F00895E82FF0E0E759FC4F2081DA
:104D80002832C0F760FF1FC0822F869586958695D2
:104D9000482F50E0277081E090E0382F01C0330F9A
:104DA0002A95EAF7232FFA01E752FA4F8081832BE5
:104DB000808361FD20C0FA01E252FA4F2095808184
:104DC000822380830895822F869586958695482F25
:104DD00050E0277081E090E0382F01C0330F2A9512
:104DE000EAF7232FFA01E752FA4F832F809590813B
:104DF00089238083DECFFA01E252FA4F8081822B31
:104E000080830895E82FF0E0EF5AFC4F208128328C
:104E1000C0F4E22FE695E695E695F0E0277081E094
:104E200090E001C0880F2A95EAF7DF01A752BA4F38
:104E30002C91282B2C93E252FA4F809520818223CB
:104E400080830895E82FF0E0E75BFC4F2081283253
:104E5000C0F4E22FE695E695E695F0E0277081E054
:104E600090E001C0880F2A95EAF7DF01A752BA4FF8
:104E70002C91282B2C93E252FA4F8095208182238B
:104E800080830895803108F00895E82FF0E0E75915
:104E9000FC4F20812832C0F7E22FE695E695E69593
:104EA000F0E0277081E090E001C0880F2A95EAF7D2
:104EB000DF01A752BA4F2C91282B2C93E252FA4FC4
:104EC000809520818223808308958D3008F0089595
:104ED000E82FF0E0E05DFC4F20812832C0F7E22FA0
:104EE000E695E695E695F0E0277081E090E001C058
:104EF000880F2A95EAF7DF01A752BA4F2C91282B89
:104F00002C93E252FA4F809520818223808308956A
:104F1000883108F00895E82FF0E0EF5AFC4F208127
:104F20002832C0F7E22FE695E695E695F0E0277087
:104F300081E090E001C0880F2A95EAF7DF01A752CF
:104F4000BA4F2C91282B2C93E252FA4F8095208156
:104F5000822380830895E82F8150883008F00895D7
:104F6000F0E0E85BFC4F20812832C8F7E22FE6959D
:104F7000E695E695F0E0277081E090E001C0880FAB
:104F80002A95EAF7DF01A752BA4F2C91282B2C93D0
:104F9000E252FA4F809520818223808308958C30DD
:104FA00008F00895E82FF0E0E35CFC4F2081283200
:104FB000C0F7E22FE695E695E695F0E0277081E0F0
:104FC00090E001C0880F2A95EAF7DF01A752BA4F97
:104FD0002C91282B2C93E252FA4F8095208182232A
:104FE00080830895CF93DF93C9E6D3E041E050E09A
:104FF00088818832C0F4E82FE695E695E695F0E0E2
:1050000087709A0102C0220F331F8A95E2F720951C
:10501000DF01A752BA4F8C9182238C93E252FA4F50
:10502000808128232083219683E0C937D80701F7A0
:10503000DF91CF910895CF93DF93CDE3D3E041E0AB
:1050400050E088818832C0F4E82FE695E695E69531
:10505000F0E087709A0102C0220F331F8A95E2F7B1
:105060002095DF01A752BA4F8C9182238C93E25294
:10507000FA4F808128232083219683E0C934D80702
:1050800001F7DF91CF910895CF93DF93582FC9E6B1
:10509000D3E040E061E070E01EC088818832B8F45F
:1050A000E82FE695E695E695F0E08770962F01C02B
:1050B000990F8A95EAF7DF01A752BA4F8C91892B95
:1050C0008C93E252FA4F90958081982390834F5FA2
:1050D0002196403109F1451700F388818832B8F7ED
:1050E000E82FE695E695E695F0E087709B0102C013
:1050F000220F331F8A95E2F72095DF01A752BA4F9E
:105100008C9182238C93E252FA4F80812823208352
:105110004F5F21964031F9F6DF91CF910895CF93FB
:10512000DF93C1E5D3E041E050E088818832C0F4EC
:10513000E82FE695E695E695F0E087709A0102C0C3
:10514000220F331F8A95E2F72095DF01A752BA4F4D
:105150008C9182238C93E252FA4F80812823208302
:10516000219683E0C936D80701F7DF91CF910895E2
:10517000CF93DF93582FC9E4D3E041E061E070E0C2
:105180001FC088818832C0F4E82FE695E695E69541
:10519000F0E087709B0102C0220F331F8A95E2F76F
:1051A0002095DF01A752BA4F8C9182238C93E25253
:1051B000FA4F8081282320834F5F2196493021F1C7
:1051C0004517F9F6E42FF0E0E85BFC4F8081883268
:1051D00098F7E82FE695E695E695F0E08770962F2C
:1051E00001C0990F8A95EAF7DF01A752BA4F8C9157
:1051F000892B8C93E252FA4F90958081982390836B
:105200004F5F21964930E1F6DF91CF910895CF931A
:10521000DF93C9E4D3E041E050E088818832C0F4F4
:10522000E82FE695E695E695F0E087709A0102C0D2
:10523000220F331F8A95E2F72095DF01A752BA4F5C
:105240008C9182238C93E252FA4F80812823208311
:10525000219683E0C135D80701F7DF91CF910895FA
:10526000CF93DF93C0E3D3E041E050E08881883200
:10527000C0F4E82FE695E695E695F0E087709A0190
:1052800002C0220F331F8A95E2F72095DF01A75253
:10529000BA4F8C9182238C93E252FA4F808128235B
:1052A0002083219683E0CD33D80701F7DF91CF919A
:1052B0000895E82FF0E0EF5AFC4F20812832C8F41F
:1052C000E22FE695E695E695F0E0277081E090E024
:1052D00002C0880F991F2A95E2F78095DF01A75237
:1052E000BA4F2C9128232C93E252FA4F208182232B
:1052F00080830895E82FF0E0E75BFC4F208128329F
:10530000C8F4E22FE695E695E695F0E0277081E097
:1053100090E002C0880F991F2A95E2F78095DF017F
:10532000A752BA4F2C9128232C93E252FA4F208196
:10533000822380830895CF93DF93C0E3D3E041E0DD
:1053400050E088818832C0F4E82FE695E695E6952E
:10535000F0E087709A0102C0220F331F8A95E2F7AE
:105360002095DF01A752BA4F8C9182238C93E25291
:10537000FA4F808128232083219683E0CD33D807FC
:1053800001F72091DE059091D9058091DA058E7F95
:105390008093DA058091DF058E7F8093DF05957E0F
:1053A0009093D905257E2093DE05DF91CF91089556
:1053B000CF93DF93782F2091DE059091D9058091CE
:1053C000DA058E7F8093DA058091DF058E7F8093EA
:1053D000DF05957E9093D905257E2093DE05372F36
:1053E00074FD69C035FD50C077FD5AC036FD41C01F
:1053F000C0E3D3E041E050E088818832C0F4E82F78
:10540000E695E695E695F0E087709A0102C0220FD6
:10541000331F8A95E2F72095DF01A752BA4F8C918E
:1054200082238C93E252FA4F808128232083219695
:1054300083E0CD33D80701F76623C1F0872F8F7043
:105440008D30E8F19091E1058091DC0588618093D1
:10545000DC05977E9093E1059091DF058091DA0558
:10546000806E8093DA059F719093DF05DF91CF9175
:1054700008958091D90582608093D9058091DE05D9
:105480008D7F8093DE05B4CF8091D90588608093AD
:10549000D9058091DE05877F8093DE0577FFA6CF53
:1054A0008091DA0581608093DA058091DF058E7F37
:1054B0008093DF059BCF90619093D90593CFE82F20
:1054C000F0E0E05DFC4F80810E948523CFCFCF9339
:1054D000DF93C0E3D3E041E050E088818832C0F43C
:1054E000E82FE695E695E695F0E087709A0102C010
:1054F000220F331F8A95E2F72095DF01A752BA4F9A
:105500008C9182238C93E252FA4F8081282320834E
:10551000219683E0CD33D80701F72091DE059091E5
:10552000D9058091DA058E7F8093DA058091DF05B9
:105530008E7F8093DF05917E9093D905217E209305
:10554000DE05DF91CF910895883108F00895E82FA6
:10555000F0E0EF5AFC4F20812832C0F7E22FE695A9
:10556000E695E695F0E0277081E090E002C0880FB4
:10557000991F2A95E2F78095DF01A752BA4F2C9127
:1055800028232C93E252FA4F2081822380830895AE
:10559000E82F8150883008F00895F0E0E85BFC4F78
:1055A00020812832C8F7E22FE695E695E695F0E0EF
:1055B000277081E090E002C0880F991F2A95E2F7DA
:1055C0008095DF01A752BA4F2C9128232C93E252E9
:1055D000FA4F20818223808308958D3008F008954A
:1055E000E82FF0E0E05DFC4F20812832C0F7E22F89
:1055F000E695E695E695F0E0277081E090E002C040
:10560000880F991F2A95E2F78095DF01A752BA4FBC
:105610002C9128232C93E252FA4F208182238083FD
:105620000895803108F00895E82FF0E0E759FC4F25
:1056300020812832C0F7E22FE695E695E695F0E066
:10564000277081E090E002C0880F991F2A95E2F749
:105650008095DF01A752BA4F2C9128232C93E25258
:10566000FA4F20818223808308952091D9053091BB
:10567000DE05932F9F7E823069F0922F977E909364
:10568000D905232F277E2093DE05813081F08F3FBF
:1056900041F0089598609093DE05277E2093D90508
:1056A000089590619093D9052093DE050895986040
:1056B0009093D9050895EF920F931F93CF93DF93A3
:1056C0001E2D222309F473C0E22EE40EC9E4D3E0B8
:1056D00050E061E070E023C05E1518F5501709F442
:1056E00047C088818832B8F4E82FE695E695E695BC
:1056F000F0E08770962F01C0990F8A95EAF7DF01D5
:10570000A752BA4F8C91892B8C93E252FA4F909505
:105710008081982390835F5F2196583009F1541758
:10572000D8F688818832B8F7E82FE695E695E695B1
:10573000F0E087709B0102C0220F331F8A95E2F7C9
:105740002095DF01A752BA4F8C9182238C93E252AD
:10575000FA4F8081282320835F5F21965830F9F625
:10576000123048F1DF91CF911F910F91EF90089582
:10577000E52FF0E0E75BFC4F8081883260F6E82F90
:10578000E695E695E695F0E08770962F01C0990FB3
:105790008A95EAF7DF01A252BA4F8C91892B8C933C
:1057A000E752FA4F9095808198239083B4CFE62EEC
:1057B000E80E482F8BCF1123D1F08091DA058E7F30
:1057C0008093DA058091DF058E7F8093DF058091DD
:1057D000D90582608093D9058091DE058D7F809305
:1057E000DE05DF91CF911F910F91EF900895809189
:1057F000DA0581608093DA058091DF058E7F8093E2
:10580000DF058091D9058D7F8093D9058091DE05D4
:105810008D7F8093DE05DF91CF911F910F91EF90E7
:105820000895CF93DF93982F87FDE4C08091D90529
:105830008B7F8093D9058091DE058B7F8093DE0579
:10584000892F829586958695837080FF50C08091C0
:10585000D90582608093D9058091DE058D7F809384
:10586000DE05292F2F7309F450C0273108F0B1C08D
:105870009091DE058091D905877E977E8061809327
:10588000D9059093DE05222309F04CC0C0E3D3E094
:1058900041E050E088818832C0F4E82FE695E69533
:1058A000E695F0E087709A0102C0220F331F8A95B7
:1058B000E2F72095DF01A752BA4F8C9182238C9397
:1058C000E252FA4F808128232083219683E0CD3352
:1058D000D80701F78091DA0581608093DA0580911D
:1058E000DF058E7F8093DF05DF91CF910895809152
:1058F000D9058D7F8093D9058091DE058D7F8093BA
:10590000DE05292F2F7309F0B0CF9091DE0580912D
:10591000D905877E8093D905977E9093DE05222353
:1059200009F4B4CF8091DA058E7F8093DA058091F7
:10593000DF058E7F8093DF05C22FD0E04BE050E083
:1059400061E070E04C175D07F1F0FA01EB5DFC4F90
:1059500080818832C0F4E82FE695E695E695F0E080
:1059600087709B0102C0220F331F8A95E2F72095B2
:10597000DF01A752BA4F8C9182238C93E252FA4FE7
:105980008081282320834F5F5F4F48315105D1F636
:10599000CB5DDC4F2881283208F0A6CFE22FE695B8
:1059A000E695E695F0E0277081E090E001C0880F71
:1059B0002A95EAF7DF01A752BA4F2C91282B2C9396
:1059C000E252FA4F8095208182238083DF91CF912C
:1059D00008952432D0F02033D0F428519091DE0580
:1059E0008091D905877E977E88608093D9059093B2
:1059F000DE0595CF8091D90584608093D90580918B
:105A0000DE058B7F8093DE051BCF2C507ECF2C33A1
:105A100068F424529091D9058091DE058F7E8860CC
:105A20008093DE05977E9093D90579CF20536DCF73
:105A3000AC0161157105A1F020E0E0E0A0E0B0E06C
:105A4000A40FB51F8C91E827F0E0E75DFB4FE081E4
:105A50002F5FA22FB0E0A617B70790F38E2F0895FF
:105A6000E0E0FCCFEF92FF920F931F93CF93DF9371
:105A70007C018B016115710561F0C0E0D0E0F70198
:105A8000EC0FFD1F80810E94CE022196C017D10726
:105A9000B0F3DF91CF911F910F91FF90EF90089598
:105AA0008F929F92AF92BF92CF92DF92EF92FF922E
:105AB0000F931F93CF93DF936C0184E88093A90623
:105AC0001092AA061092AC06F601EE2406C0E394EA
:105AD00031964FEFE41609F481C080818823B9F72D
:105AE0008E2D60E30E943B87A82E282F30E080EDAA
:105AF0009FEFAC01249FC001259F900D349F900D16
:105B000011248E0D911D892B09F06AC0AA2009F479
:105B100050C0FF24BB248824839481E3982EFE1474
:105B200008F060C0F601EF0DF11D80818093AD0695
:105B3000F394AEEAB6E091E00AC0F601EF0DF11D74
:105B400080818D939F5FF394903309F43FC0FE14DE
:105B5000A0F39F5F9093AB06492F4D5F642F70E0D9
:105B6000D9F190E020E030E0F901E755F94F80816C
:105B70009827E92FF0E0E75DFB4F90812F5F3F4FC3
:105B8000241790F3FB01E755F94F90838B010F5FCA
:105B90001F4FC0E0D0E0FE01E755F94F80810E9421
:105BA000CE022196C017D107B0F3B394BA1408F40B
:105BB000B6CFDF91CF911F910F91FF90EF90DF90C3
:105BC000CF90BF90AF909F908F9008959092AB062A
:105BD00044E364E370E0C5CF90E0D4CF95E0A92E14
:105BE000A39494CF8092AB0644E064E070E0B9CF18
:105BF0008F929F92AF92BF92CF92DF92EF92FF92DD
:105C00000F931F93CF93DF936C01E62E84E880936C
:105C1000A9061092AA0687E08093AC06862F60E35F
:105C20000E943B87A82E282F30E080ED9FEFAC012B
:105C3000249FC001259F900D349F900D11248E0D3F
:105C4000911D892B09F0A394AA2009F450C0FF24C8
:105C5000BB248824839421E3922EFE1408F05CC0B8
:105C6000F601EF0DF11D80818093AD06F394AEEA4D
:105C7000B6E091E00AC0F601EF0DF11D80818D9331
:105C80009F5FF394903309F43FC0FE14A0F39F5F2D
:105C90009093AB06492F4D5F642F70E0D9F190E0EF
:105CA00020E030E0F901E755F94F80819827E92F8E
:105CB000F0E0E75DFB4F90812F5F3F4F241790F39B
:105CC000FB01E755F94F90838B010F5F1F4FC0E039
:105CD000D0E0FE01E755F94F80810E94CE02219667
:105CE000C017D107B0F3B394BA1408F4B6CFDF915C
:105CF000CF911F910F91FF90EF90DF90CF90BF90C9
:105D0000AF909F908F9008959092AB0644E364E328
:105D100070E0C5CF90E0D4CF8092AB0644E064E061
:105D200070E0BDCFCF93DF9394E89093A9061092D3
:105D3000AA0691E09093AC068093AD0682E0809332
:105D4000AB06C9EAD6E0DE01E0E08D91E827F0E09D
:105D5000E75DFB4FE08186E0AE3AB807B1F7EC9320
:105D600089910E94CE0286E0CF3AD807C9F7DF9129
:105D7000CF910895CF93DF9322E42093A906109248
:105D8000AA0622E02093AB069093AC068093AD0662
:105D9000C9EAD6E0DE01E0E08D91E827F0E0E75DBA
:105DA000FB4FE08186E0AE3AB807B1F7EC938991FA
:105DB0000E94CE0286E0CF3AD807C9F7DF91CF9193
:105DC0000895CF93DF9390E89093A9061092AA06C6
:105DD00091E09093AB068093AC06E091A904F0E0CB
:105DE000E75DFB4FE081E927F0E0E75DFB4FE081F5
:105DF000E827F0E0E75DFB4F80818093AD06C9EABC
:105E0000D6E089910E94CE0286E0CE3AD807C9F743
:105E1000DF91CF9108950F931F93DF93CF9300D01D
:105E20000F92CDB7DEB769837A838B839C8384E836
:105E30008093A9061092AA0695E09093AC06FE0105
:105E400031966093AD0681818093AE068281809306
:105E5000AF0683818093B0069093AB0609EA16E003
:105E6000D801E0E08D91E827F0E0E75DFB4FE081AD
:105E700086E0A13BB807B1F7EC93F80181918F015F
:105E80000E94CE02F6E0023B1F07B9F70F900F9079
:105E90000F900F90CF91DF911F910F9108950F9365
:105EA0001F93DF93CF930F920F92CDB7DEB79A83F4
:105EB000898394E89093A9061092AA0693E09093A0
:105EC000AC068093AD068A818093AE069093AB06B4
:105ED00009EA16E0D801E0E08D91E827F0E0E75DFF
:105EE000FB4FE08186E0AF3AB807B1F7EC93F801D9
:105EF00081918F010E94CE02F6E0003B1F07B9F7A7
:105F00000F900F90CF91DF911F910F9108950F93F4
:105F10001F93DF93CF9300D00F92CDB7DEB7698385
:105F20007A838B839C8384E88093A9061092AA06C7
:105F300086E08093AC06FE0131966093AD068181C8
:105F40008093AE0682818093AF0683818093B006F2
:105F500085E08093AB0609EA16E0D801E0E08D9178
:105F6000E827F0E0E75DFB4FE08186E0A13BB80762
:105F7000B1F7EC93F80181918F010E94CE02F6E017
:105F8000023B1F07B9F70F900F900F900F90CF9122
:105F9000DF911F910F9108950F931F93DF93CF937C
:105FA0000F920F92CDB7DEB79A83898394E89093CE
:105FB000A9061092AA0694E09093AC068093AD06D1
:105FC0008A818093AE0683E08093AB0609EA16E0EF
:105FD000D801E0E08D91E827F0E0E75DFB4FE0813C
:105FE00086E0AF3AB807B1F7EC93F80181918F01E1
:105FF0000E94CE02F6E0003B1F07B9F70F900F900A
:10600000CF91DF911F910F910895CF93DF9394E883
:106010009093A9061092AA0692E09093AC06809302
:10602000AD069093AB06C9EAD6E0DE01E0E08D91C3
:10603000E827F0E0E75DFB4FE08186E0AE3AB80785
:10604000B1F7EC9389910E94CE0286E0CF3AD8074F
:10605000C9F7DF91CF9108951F920F920FB60F925B
:106060000BB60F921124DF92EF92FF920F931F93C2
:106070002F933F934F935F936F937F938F939F9350
:10608000AF93BF93CF93DF93EF93FF931091CE0025
:1060900080912804882309F48FC08091E7059091AE
:1060A000E805895E934008F0A1C09091E505903421
:1060B00008F0AAC0292F2F5FE92FF0E0E751F94F30
:1060C00010832093E5051092E8051092E705233030
:1060D00008F472C07091E9069091EA0680E0609140
:1060E000EB06462F50E0482B592B30E0CA010496AE
:1060F0002817390708F460C09A012D5F3F4FF90156
:10610000E751F94F10812115310509F445C190E09F
:10611000E0E0A0E0B0E0A751B94F8C91E827F0E0B3
:10612000E75DFB4FE0819F5FA92FB0E0A217B307A7
:1061300090F31E1709F494C02115310509F42EC1FE
:1061400090E0E0E0A0E0B0E0A751B94F8C91E827E3
:10615000F0E0E75DFB4FE0819F5FA92FB0E0A21761
:10616000B30790F38E2F90E00E94F60D1092E50594
:1061700080E88093A9061092AA0681E08093AB067E
:106180001092AC06E091A904F0E0E75DFB4FE081DE
:10619000E827F0E0E75DFB4FE081F0E0E75DFB4FD3
:1061A00080818093AD06C9EAD6E089910E94CE0233
:1061B00086E0CE3AD807C9F7FF91EF91DF91CF91F2
:1061C000BF91AF919F918F917F916F915F914F910F
:1061D0003F912F911F910F91FF90EF90DF900F90C3
:1061E0000BBE0F900FBE0F901F9018950E94F227C4
:1061F0000E94A7241093E90681E08093E5051092A0
:10620000E8051092E705D8CF80E88093A9061092A0
:10621000AA0681E08093AB069093AC06E091A904B6
:10622000F0E0E75DFB4FE081E827F0E0E75DFB4F42
:10623000E081E927F0E0E75DFB4F80818093AD06C8
:10624000C9EAD6E089910E94CE0236E0CE3AD30761
:10625000C9F71092E5051092E8051092E705ACCF5A
:10626000713809F48DC17238B0F5713109F426C165
:10627000723108F096C0713051F1703131F080E028
:106280000E94E12E1092E50597CF6231C1F780910F
:10629000EC06082F10E0000F111F000F111F000F58
:1062A000111F8091ED06080F111D02951295107FA8
:1062B0001027007F1027CEEED6E08991B8010E940A
:1062C00016450F5F1F4FF6E0CE3FDF07B1F781E0C5
:1062D0000E94E12ED7CF763809F430C1773808F024
:1062E00073C0723809F47FC1753849F643305105DF
:1062F00009F0A5C03091EC06932F80E02091ED06C7
:10630000E22EFF24E82AF92AD090EE06EAE3ED1502
:1063100008F4B6CF7093A9061092AA06F2E0DF0E39
:10632000D092AB068EEFD80E3093AC062093AD061C
:10633000DD2071F00EEA16E0E701CE010E945A4519
:10634000F80181938F0121969E012E192D15A8F336
:106350008091AB06682F6D5F09F4EEC1A9EAB6E043
:1063600090E08E5F282F30E02655394F8D91982789
:10637000E92FF0E0E75DFB4F9081A217B307B1F77B
:10638000E62FF0E0E755F94F90836F5F89EA96E0DA
:1063900070E00E94322D76CFE0E0CBCE80E090E03E
:1063A000E3CE703409F45EC1713409F068CF623015
:1063B00009F065CF9091EC0680E02091ED06820F08
:1063C000911D0E9470015ECF7738E9F1783809F0AD
:1063D00056CF7093A9061092AA068091EC068130E0
:1063E00009F47FC1813008F06CC180E18093AC0674
:1063F0001092AD068093AE061092AF0684E047E09F
:10640000A7E0B0E068E070E08093AB0690E020E0A9
:1064100030E0F901E755F94F80819827E92FF0E046
:10642000E75DFB4F90812F5F3F4F241790F3A755F7
:10643000B94F9C9389EA96E00E94322D23CF80E0E9
:106440000E94E12E1FCF8091EC06882309F011C134
:106450004230510509F014CFE091ED06E43008F028
:106460000ECF89E18093A9061092AA0680E180935D
:10647000AB064E2F50E042955295507F5427407FF7
:106480005427ACEAB6E008C0ED934F5F5F4F36E0AB
:10649000AC3BB30709F432C1FA01EC5CF74FE08181
:1064A0002E2F30E0C9018F7090700D976CF720731C
:1064B00030702033310541F7EF7DE6CF623009F0CF
:1064C000DECE8091EC06082F10E0000F111F000FA8
:1064D000111F000F111F8091ED06080F111D02956D
:1064E0001295107F1027007F102789E18093A9065D
:1064F0001092AA0680E18093AB06CCEAD6E0C801F0
:106500000E945A4589930F5F1F4FE6E0CC3BDE07A0
:10651000B1F7DE015397E0E08D91E827F0E0E75D09
:10652000FB4FE081CA17DB07B9F7E093BC0689EAA5
:1065300096E064E170E00E94322DA4CE9091EC06CA
:1065400080E02091ED06E22EFF24E82AF92A7EEF72
:10655000D72ED60E63506A3308F071CFDD2009F4D0
:10656000B6CE0EEE16E0E701F80181918F01BE0173
:106570000E94164521969E012E192D15A8F3A7CE2F
:1065800087E190E09093AD068093AC0681ED90E0BA
:106590009093AF068093AE06E9E7F3E0A0EBB6E098
:1065A00081918D9323E0EF37F207D1F781E8809353
:1065B000A9061092AA068AE08093AB06A9EAB6E083
:1065C000E0E08D91E827F0E0E75DFB4FE08136E009
:1065D000A63BB307B1F7EC93CD010D976EE070E0E9
:1065E0000E94322D4FCE4230510509F028CF309114
:1065F000EC06332309F071C09091ED06973808F04E
:1066000092C0943820F121E082E88093A90610928C
:10661000AA0683E08093AB063093AC069093AD0658
:106620002093AE06A9EAB6E0E0E08D91E827F0E01D
:10663000E75DFB4FE08186E0AF3AB807B1F7EC9336
:10664000CD01069767E070E00E94322D1BCE993194
:1066500009F470C0993120F0892F8158823098F266
:1066600020E0D2CF80913E0690913F060E94BA2E44
:1066700009CE813009F003CE4231510509F0FFCD3A
:10668000E091ED06E43008F0FACD2E2F30E0AEEECA
:10669000B6E022953295307F3227207F32278D91C8
:1066A000F901EC5CF74F80832F5F3F4FE6E0AE3F90
:1066B000BE07A9F781E00E94E12E81E08093F705F3
:1066C000E1CD883009F0DBCD81E08093AC0644E079
:1066D000A4E0B0E065E070E097CE9091ED0620E098
:1066E00093CF88E08093AC0680E18093AD0682E092
:1066F00045E0A5E0B0E066E070E086CE5397E0E0CC
:106700008D91E827F0E0E75DFB4FE08186E0AC3B50
:10671000B807B1F7E093BC06CD01439764E170E0A0
:106720000E94322DAFCD973849F0983809F46BCFDD
:1067300020E06ACF20E168CF90E022CE24E064CF51
:106740002F923F924F925F926F927F928F929F9281
:10675000AF92BF92CF92DF92EF92FF920F931F936F
:10676000DF93CF93CDB7DEB729970FB6F894DEBF8E
:106770000FBECDBF3324198645E0488758E05F83BC
:106780008DE08E831D821C829BE19B838FEA682EA5
:1067900086E0782E25C08AE00E945C1F882311F0D5
:1067A0000C94784083E00E94721F882331F0832D7F
:1067B0008F5F63E00E943B87392E332011F00C94E9
:1067C0007E4184E00E945C1F882311F00C943041CC
:1067D0000E945F0E0E945457882311F00C945C4174
:1067E0000E94452289E00E945C1F8823A1F28AE072
:1067F0000E94721F882379F284E88093A906109280
:10680000AA061092AC06E0E2F4E0CC2407C0C394E0
:1068100031964FEFC41611F40C94474380818823BE
:10682000B1F78C2D60E30E943B87A82E282F30E023
:1068300080ED9FEFFC012E9FC0012F9F900D3E9F8A
:10684000900D11248C0D911D892B11F00C9449434E
:10685000AA2009F458C0DD24BB248824839411E3C2
:10686000912EDC1410F00C948243ED2DF0E0E05EEC
:10687000FB4F80818093AD06D394AEEAB6E091E001
:106880000CC0ED2DF0E0E05EFB4F80818D939F5FAB
:10689000D394903311F40C940442DC1490F39F5F72
:1068A0009093AB06492F4D5F642F70E011F40C9468
:1068B0004C4290E020E030E0F901E755F94F80814B
:1068C0009827E92FF0E0E75DFB4F90812F5F3F4F66
:1068D000241790F3FB01E755F94F90837B0108944F
:1068E000E11CF11C00E010E0F801E755F94F808150
:1068F0000E94CE020F5F1F4F0E151F05A8F3B39421
:10690000BA1408F4AECF90919C0584E88093A90650
:106910001092AA0681E08093AC069093AD0682E0C7
:106920008093AB06B9EA4B2EB6E05B2ED201E0E0D5
:106930008D91E827F0E0E75DFB4FE081F6E0AE3AAD
:10694000BF07B1F7EC938D0105501040F80181911C
:106950008F010E94CE02F6E00F3A1F07B9F784E8D4
:106960008093A9061092AA061092AC06EFE0F4E01C
:10697000CC2407C0C39431964FEFC41611F40C9485
:10698000424380818823B1F78C2D60E30E943B87CE
:10699000A82E282F30E080ED9FEFFC012E9FC00134
:1069A0002F9F900D3E9F900D11248C0D911D892BD2
:1069B00011F00C944443AA2009F458C0DD24BB24F0
:1069C00088248394F1E39F2EDC1410F00C94894307
:1069D000ED2DF0E0E15FFB4F80818093AD06D39415
:1069E000AEEAB6E091E00CC0ED2DF0E0E15FFB4FC8
:1069F00080818D939F5FD394903311F40C94EA417E
:106A0000DC1490F39F5F9093AB06492F4D5F642F8A
:106A100070E011F40C944F4290E020E030E0F90176
:106A2000E755F94F80819827E92FF0E0E75DFB4FAC
:106A300090812F5F3F4F241790F3FB01E755F94FEB
:106A400090837B010894E11CF11C00E010E0F80148
:106A5000E755F94F80810E94CE020F5F1F4F0E1540
:106A60001F05A8F3B394BA1408F4AECF909175063D
:106A700084E88093A9061092AA0681E08093AC0670
:106A80009093AD0682E08093AB06A9EAB6E0E0E021
:106A90008D91E827F0E0E75DFB4FE081F6E0AE3A4C
:106AA000BF07B1F7E093AE068D0105501040F80125
:106AB00081918F010E94CE0260167106C1F784E8B1
:106AC0008093A9061092AA061092AC06EDE0F4E0BD
:106AD000CC2407C0C39431964FEFC41611F40C9424
:106AE0003D4380818823B1F78C2D60E30E943B8772
:106AF000A82E282F30E080ED9FEFFC012E9FC001D3
:106B00002F9F900D3E9F900D11248C0D911D892B70
:106B100011F00C943F43AA2009F458C0DD24BB2493
:106B20008824839471E3972EDC1410F00C94D543E1
:106B3000ED2DF0E0E35FFB4F80818093AD06D394B1
:106B4000AEEAB6E091E00CC0ED2DF0E0E35FFB4F64
:106B500080818D939F5FD394903311F40C940B42FA
:106B6000DC1490F39F5F9093AB06492F4D5F642F29
:106B700070E011F40C945B4290E020E030E0F90109
:106B8000E755F94F80819827E92FF0E0E75DFB4F4B
:106B900090812F5F3F4F241790F3FB01E755F94F8A
:106BA00090837B010894E11CF11C00E010E0F801E7
:106BB000E755F94F80810E94CE020F5F1F4F0E15DF
:106BC0001F05A8F3B394BA1408F4AECF90916206EF
:106BD00084E88093A9061092AA0681E08093AC060F
:106BE0009093AD0682E08093AB06A9EAB6E0E0E0C0
:106BF0008D91E827F0E0E75DFB4FE081F6E0AE3AEB
:106C0000BF07B1F7E093AE068D0105501040F801C3
:106C100081918F010E94CE0260167106C1F784E84F
:106C20008093A9061092AA061092AC06E6E0F4E062
:106C3000CC2407C0C39431964FEFC41611F40C94C2
:106C4000384380818823B1F78C2D60E30E943B8715
:106C5000A82E282F30E080ED9FEFFC012E9FC00171
:106C60002F9F900D3E9F900D11248C0D911D892B0F
:106C700011F00C943A43AA2009F458C0DD24BB2437
:106C80008824839451E3952EDC1410F00C94CE43A9
:106C9000ED2DF0E0EA5FFB4F80818093AD06D39449
:106CA000AEEAB6E091E00CC0ED2DF0E0EA5FFB4FFC
:106CB00080818D939F5FD394903311F40C94124292
:106CC000DC1490F39F5F9093AB06492F4D5F642FC8
:106CD00070E011F40C94564290E020E030E0F901AD
:106CE000E755F94F80819827E92FF0E0E75DFB4FEA
:106CF00090812F5F3F4F241790F3FB01E755F94F29
:106D000090837B010894E11CF11C00E010E0F80185
:106D1000E755F94F80810E94CE020F5F1F4F0E157D
:106D20001F05A8F3B394BA1408F4AECF20913E0621
:106D300080913F0629838A8384E88093A906109274
:106D4000AA0693E09093AC062093AD068A818093C7
:106D5000AE069093AB06A9EAB6E0E0E08D91E82795
:106D6000F0E0E75DFB4FE0816A167B06B9F7E09340
:106D7000AF0609EA16E0F80181918F010E94CE0268
:106D8000F6E0003B1F07B9F784E88093A90610924C
:106D9000AA061092AC06EDEFF3E0CC2407C0C39432
:106DA00031964FEFC41611F40C943343808188233D
:106DB000B1F78C2D60E30E943B87A82E282F30E08E
:106DC00080ED9FEFFC012E9FC0012F9F900D3E9FF5
:106DD000900D11248C0D911D892B11F00C943543CD
:106DE000AA2009F458C0DD24BB248824839431E30D
:106DF000932EDC1410F00C949043ED2DF0E0E35052
:106E0000FC4F80818093AD06D394AEEAB6E091E06A
:106E10000CC0ED2DF0E0E350FC4F80818D939F5F1F
:106E2000D394903311F40C94F741DC1490F39F5FEA
:106E30009093AB06492F4D5F642F70E011F40C94D2
:106E4000444290E020E030E0F901E755F94F8081BD
:106E50009827E92FF0E0E75DFB4F90812F5F3F4FD0
:106E6000241790F3FB01E755F94F90837B010894B9
:106E7000E11CF11C00E010E0F801E755F94F8081BA
:106E80000E94CE020F5F1F4F0E151F05A8F3B3948B
:106E9000BA1408F4AECF9091000284E88093A9065A
:106EA0001092AA0681E08093AC069093AD0682E032
:106EB0008093AB06A9EAB6E0E0E08D91E827F0E028
:106EC000E75DFB4FE081F6E0AE3ABF07B1F7E09334
:106ED000AE068D0105501040F80181918F010E948E
:106EE000CE0260167106C1F784E88093A90610925D
:106EF000AA061092AC06E2EFF3E0CC2407C0C394DC
:106F000031964FEFC41611F40C942E4380818823E0
:106F1000B1F78C2D60E30E943B87A82E282F30E02C
:106F200080ED9FEFFC012E9FC0012F9F900D3E9F93
:106F3000900D11248C0D911D892B11F00C94304370
:106F4000AA2009F458C0DD24BB248824839491E34B
:106F5000992EDC1410F00C94B043ED2DF0E0EE50BF
:106F6000FC4F80818093AD06D394AEEAB6E091E009
:106F70000CC0ED2DF0E0EE50FC4F80818D939F5FB3
:106F8000D394903311F40C943342DC1490F39F5F4C
:106F90009093AB06492F4D5F642F70E011F40C9471
:106FA000474290E020E030E0F901E755F94F808159
:106FB0009827E92FF0E0E75DFB4F90812F5F3F4F6F
:106FC000241790F3FB01E755F94F90837B01089458
:106FD000E11CF11C00E010E0F801E755F94F808159
:106FE0000E94CE020F5F1F4F0E151F05A8F3B3942A
:106FF000BA1408F4AECF90915C0684E88093A90699
:107000001092AA0681E08093AC069093AD0682E0D0
:107010008093AB06A9EAB6E0E0E08D91E827F0E0C6
:10702000E75DFB4FE081F6E0AE3ABF07B1F7E093D2
:10703000AE068D0105501040F80181918F010E942C
:10704000CE0260167106C1F784E88093A9061092FB
:10705000AA061092AC0680EE882E83E0982EF401EA
:10706000CC2407C0C39431964FEFC41611F40C948E
:10707000294380818823B1F78C2D60E30E943B87F0
:10708000A82E282F30E080ED9FEFFC012E9FC0013D
:107090002F9F900D3E9F900D11248C0D911D892BDB
:1070A00011F00C942B43AA2009F456C0DD24BB2414
:1070B00011E3212EDC1410F00C94C643ED2DF0E00A
:1070C000E052FC4F80818093AD06D394AEEAB6E0E7
:1070D00091E00CC0ED2DF0E0E052FC4F80818D93EB
:1070E0009F5FD394903311F40C943A42DC1490F3E4
:1070F0009F5F9093AB06492F4D5F642F70E011F4B2
:107100000C94414290E020E030E0F901E755F94F5E
:1071100080819827E92FF0E0E75DFB4F90812F5F9A
:107120003F4F241790F3FB01E755F94F90837B0104
:107130000894E11CF11C00E010E0F801E755F94F5C
:1071400080810E94CE020F5F1F4F0E151F05A8F30E
:10715000B394BA1408F4AECF90915F0684E880939C
:10716000A9061092AA0681E08093AC069093AD0622
:1071700082E08093AB06A9EAB6E0E0E08D91E827D3
:10718000F0E0E75DFB4FE081F6E0AE3ABF07B1F714
:10719000E093AE068D0105501040F80181918F01FA
:1071A0000E94CE0260167106C1F784E88093A9069A
:1071B0001092AA061092AC06E2EEF3E0CC2407C0CF
:1071C000C39431964FEFC41611F40C94244380817C
:1071D0008823B1F78C2D60E30E943B87A82E282FCF
:1071E00030E080ED9FEFFC012E9FC0012F9F900D9E
:1071F0003E9F900D11248C0D911D892B11F00C9444
:107200002643AA2009F456C0DD24BB24A1E32A2E7C
:10721000DC1410F00C94BE43ED2DF0E0EE51FC4F69
:1072200080818093AD06D394AEEAB6E091E00CC0C5
:10723000ED2DF0E0EE51FC4F80818D939F5FD39454
:10724000903311F40C942C42DC1490F39F5F9093D4
:10725000AB06492F4D5F642F70E011F40C9463422C
:1072600090E020E030E0F901E755F94F8081982760
:10727000E92FF0E0E75DFB4F90812F5F3F4F241730
:1072800090F3FB01E755F94F90837B010894E11CD3
:10729000F11C00E010E0F801E755F94F80810E94F1
:1072A000CE020F5F1F4F0E151F05A8F3B394BA143B
:1072B00008F4AECF9091970284E88093A9061092CB
:1072C000AA0681E08093AC069093AD0682E080939D
:1072D000AB06A9EAB6E0E0E08D91E827F0E0E75DD3
:1072E000FB4FE081F6E0AE3ABF07B1F7E093AE06A0
:1072F0008D0105501040F80181918F010E94CE024E
:1073000060167106C1F784E88093A9061092AA0658
:107310001092AC06CC2409C0C3940894811C911C23
:10732000FFEFCF1611F40C941F43F40180818823E2
:1073300099F78C2D60E30E943B87982E282F30E030
:1073400080ED9FEFAC01249FC001259F900D349FDD
:10735000900D11248C0D911D892B11F00C9421435B
:10736000992009F458C0DD24BB2488248394E1E3E8
:10737000AE2EDC1410F00C94B743ED2DF0E0E0528B
:10738000FC4F80818093AD06D394AEEAB6E091E0E5
:107390000CC0ED2DF0E0E052FC4F80818D939F5F9B
:1073A000D394903311F40C942542DC1490F39F5F36
:1073B0009093AB06492F4D5F642F70E011F40C944D
:1073C000604290E020E030E0F901E755F94F80811C
:1073D0009827E92FF0E0E75DFB4F90812F5F3F4F4B
:1073E000241790F3FB01E755F94F90837B01089434
:1073F000E11CF11C00E010E0F801E755F94F808135
:107400000E94CE020F5F1F4F0E151F05A8F3B39405
:10741000B91408F4AECF9091980284E88093A9063D
:107420001092AA0681E08093AC069093AD0682E0AC
:107430008093AB06A9EAB6E0E0E08D91E827F0E0A2
:10744000E75DFB4FE08156E0AE3AB507B1F7E09358
:10745000AE068D0105501040F80181918F010E9408
:10746000CE0260167106C1F784E88093A9061092D7
:10747000AA061092AC06E2EDF3E0CC2407C0C39458
:1074800031964FEFC41611F40C941A43808188236F
:10749000B1F78C2D60E30E943B87982E282F30E0B7
:1074A00080ED9FEFFC012E9FC0012F9F900D3E9F0E
:1074B000900D11248C0D911D892B11F00C941C43FF
:1074C000992009F456C0DD24BB248824839461E309
:1074D000A62EDC1410F00C94DC43ED2DF0E0EE52FF
:1074E000FC4F80818093AD06D394AEEAB6E091E084
:1074F0000BC0ED2DF0E0EE52FC4F80818D939F5F2D
:10750000D394903309F49BC7DC1498F39F5F909356
:10751000AB06492F4D5F642F70E009F4CFC790E0B0
:1075200020E030E0F901E755F94F80819827E92FF5
:10753000F0E0E75DFB4F90812F5F3F4F241790F302
:10754000FB01E755F94F90837B010894E11CF11C86
:1075500000E010E0F801E755F94F80810E94CE026B
:107560000F5F1F4F0E151F05A8F3B394B91408F44D
:10757000B0CF8DE090E00E94490394E89093A90673
:107580001092AA0692E09093AC068093AD06909379
:10759000AB06A9EAB6E0E0E08D91E827F0E0E75D10
:1075A000FB4FE081F6E0AE3ABF07B1F7E093AE06DD
:1075B0008D0105501040F80181918F010E94CE028B
:1075C00060167106C1F784E88093A9061092AA0696
:1075D0001092AC06E9ECF3E0CC2407C0C3943196DA
:1075E0004FEFC41611F40C94154380818823B1F732
:1075F0008C2D60E30E943B87982E282F30E080ED91
:107600009FEFFC012E9FC0012F9F900D3E9F900D7C
:1076100011248C0D911D892B11F00C941743992086
:1076200009F456C0DD24BB248824839441E3A42EAE
:10763000DC1410F00C94A943ED2DF0E0E753FC4F5F
:1076400080818093AD06D394AEEAB6E091E00BC0A2
:10765000ED2DF0E0E753FC4F80818D939F5FD39435
:10766000903309F4E6C6DC1498F39F5F9093AB0661
:10767000492F4D5F642F70E009F41BC790E020E0B4
:1076800030E0F901E755F94F80819827E92FF0E0C4
:10769000E75DFB4F90812F5F3F4F241790F3FB0175
:1076A000E755F94F90837B010894E11CF11C00E041
:1076B00010E0F801E755F94F80810E94CE020F5F7C
:1076C0001F4F0E151F05A8F3B394B91408F4B0CFDB
:1076D0009091520684E88093A9061092AA0681E050
:1076E0008093AC069093AD0682E08093AB06A9EA46
:1076F000B6E0E0E08D91E827F0E0E75DFB4FE08148
:10770000F6E0AE3ABF07B1F7E093AE068D01055043
:107710001040F80181918F010E94CE02601671061F
:10772000C1F784E88093A9061092AA061092AC06CD
:10773000E1ECF3E0CC2406C0C39431964FEFC416BD
:1077400009F46FC780818823B9F78C2D60E30E940C
:107750003B87982E282F30E080ED9FEFFC012E9F75
:10776000C0012F9F900D3E9F900D11248C0D911DF7
:10777000892B09F058C7992009F455C0DD24BB2492
:107780008824839421E3A22EDC1408F0DCC7ED2DBD
:10779000F0E0EF53FC4F80818093AD06D394AEEAC6
:1077A000B6E091E00BC0ED2DF0E0EF53FC4F80818F
:1077B0008D939F5FD394903309F420C6DC1498F323
:1077C0009F5F9093AB06492F4D5F642F70E009F4E3
:1077D0006BC690E020E030E0F901E755F94F808179
:1077E0009827E92FF0E0E75DFB4F90812F5F3F4F37
:1077F000241790F3FB01E755F94F90837B01089420
:10780000E11CF11C00E010E0F801E755F94F808120
:107810000E94CE020F5F1F4F0E151F05A8F3B394F1
:10782000B91408F4B1CF9091B40584E88093A90607
:107830001092AA0681E08093AC069093AD0682E098
:107840008093AB06A9EAB6E0E0E08D91E827F0E08E
:10785000E75DFB4FE081F6E0AE3ABF07B1F7E0939A
:10786000AE068D0105501040F80181918F010E94F4
:10787000CE0260167106C1F784E88093A9061092C3
:10788000AA061092AC06E9EBF3E0CC2406C0C39440
:1078900031964FEFC41609F4C0C680818823B9F72A
:1078A0008C2D60E30E943B87982E282F30E080EDDE
:1078B0009FEFFC012E9FC0012F9F900D3E9F900DCA
:1078C00011248C0D911D892B09F0A9C6992009F46A
:1078D00055C0DD24BB248824839481E3A82EDC14C6
:1078E00008F071C7ED2DF0E0E754FC4F80818093E4
:1078F000AD06D394AEEAB6E091E00BC0ED2DF0E01A
:10790000E754FC4F80818D939F5FD394903309F4AB
:1079100068C5DC1498F39F5F9093AB06492F4D5FC9
:10792000642F70E009F4BEC590E020E030E0F9017A
:10793000E755F94F80819827E92FF0E0E75DFB4F8D
:1079400090812F5F3F4F241790F3FB01E755F94FCC
:1079500090837B010894E11CF11C00E010E0F80129
:10796000E755F94F80810E94CE020F5F1F4F0E1521
:107970001F05A8F3B394B91408F4B1CF809169023C
:107980008A5094E89093A9061092AA0692E09093E8
:10799000AC068093AD069093AB06A9EAB6E0E0E0B2
:1079A0008D91E827F0E0E75DFB4FE081F6E0AE3A2D
:1079B000BF07B1F7E093AE068D0105501040F80106
:1079C00081918F010E94CE0260167106C1F784E892
:1079D0008093A9061092AA061092AC06E6EBF3E09B
:1079E000CC2406C0C39431964FEFC41609F411C6D7
:1079F00080818823B9F78C2D60E30E943B87982E05
:107A0000282F30E080ED9FEFFC012E9FC0012F9FBB
:107A1000900D3E9F900D11248C0D911D892B09F026
:107A2000FAC5992009F455C0DD24BB248824839429
:107A300011E3A12EDC1408F053C6ED2DF0E0EA545A
:107A4000FC4F80818093AD06D394AEEAB6E091E01E
:107A50000BC0ED2DF0E0EA54FC4F80818D939F5FC9
:107A6000D394903309F4B0C4DC1498F39F5F9093DF
:107A7000AB06492F4D5F642F70E009F42DC590E0EF
:107A800020E030E0F901E755F94F80819827E92F90
:107A9000F0E0E75DFB4F90812F5F3F4F241790F39D
:107AA000FB01E755F94F90837B010894E11CF11C21
:107AB00000E010E0F801E755F94F80810E94CE0206
:107AC0000F5F1F4F0E151F05A8F3B394B91408F4E8
:107AD000B1CF80916B028A5094E89093A9061092DE
:107AE000AA0692E09093AC068093AD069093AB0605
:107AF000A9EAB6E0E0E08D91E827F0E0E75DFB4F12
:107B0000E081F6E0AE3ABF07B1F7E093AE068D0133
:107B100005501040F80181918F010E94CE0260163D
:107B20007106C1F784E88093A9061092AA06109204
:107B3000AC06E2EBF3E0CC2406C0C39431964FEFE1
:107B4000C41609F462C580818823B9F78C2D60E3DF
:107B50000E943B87982E282F30E080ED9FEFFC019C
:107B60002E9FC0012F9F900D3E9F900D11248C0DD4
:107B7000911D892B09F04BC5992009F455C0DD24CE
:107B8000BB2488248394A1E3AA2EDC1408F0B4C596
:107B9000ED2DF0E0EE54FC4F80818093AD06D39440
:107BA000AEEAB6E091E00BC0ED2DF0E0EE54FC4FF4
:107BB00080818D939F5FD394903309F4FFC3DC14CD
:107BC00098F39F5F9093AB06492F4D5F642F70E051
:107BD00009F480C490E020E030E0F901E755F94F66
:107BE00080819827E92FF0E0E75DFB4F90812F5FC0
:107BF0003F4F241790F3FB01E755F94F90837B012A
:107C00000894E11CF11C00E010E0F801E755F94F81
:107C100080810E94CE020F5F1F4F0E151F05A8F333
:107C2000B394B91408F4B1CF90916C029A5084E8DF
:107C30008093A9061092AA0681E08093AC069093E7
:107C4000AD0682E08093AB06A9EAB6E0E0E08D9154
:107C5000E827F0E0E75DFB4FE081F6E0AE3ABF07D2
:107C6000B1F7E093AE068D0105501040F801819107
:107C70008F010E94CE0260167106C1F784E88093DE
:107C8000A9061092AA061092AC06E0EBF3E0CC2411
:107C900006C0C39431964FEFC41609F4B2C4808174
:107CA0008823B9F78C2D60E30E943B87982E282FFC
:107CB00030E080ED9FEFFC012E9FC0012F9F900DC3
:107CC0003E9F900D11248C0D911D892B09F09BC4B2
:107CD000992009F455C0DD24BB2488248394E1E372
:107CE000AE2EDC1408F002C5ED2DF0E0E055FC4F9F
:107CF00080818093AD06D394AEEAB6E091E00BC0EC
:107D0000ED2DF0E0E055FC4F80818D939F5FD39483
:107D1000903309F44DC3DC1498F39F5F9093AB0646
:107D2000492F4D5F642F70E009F4D2C390E020E04A
:107D300030E0F901E755F94F80819827E92FF0E00D
:107D4000E75DFB4F90812F5F3F4F241790F3FB01BE
:107D5000E755F94F90837B010894E11CF11C00E08A
:107D600010E0F801E755F94F80810E94CE020F5FC5
:107D70001F4F0E151F05A8F3B394B91408F4B1CF23
:107D800084E88093A9061092AA061092AC06E9EA4C
:107D9000F3E0CC2406C0C39431964FEFC41609F427
:107DA0002CC480818823B9F78C2D60E30E943B8727
:107DB000982E282F30E080ED9FEFFC012E9FC00110
:107DC0002F9F900D3E9F900D11248C0D911D892B9E
:107DD00009F015C4992009F455C0DD24BB2488247A
:107DE000839461E3A62EDC1408F074C4ED2DF0E05A
:107DF000E755FC4F80818093AD06D394AEEAB6E0A0
:107E000091E00BC0ED2DF0E0E755FC4F80818D93A4
:107E10009F5FD394903309F4C5C2DC1498F39F5F3D
:107E20009093AB06492F4D5F642F70E009F432C385
:107E300090E020E030E0F901E755F94F8081982784
:107E4000E92FF0E0E75DFB4F90812F5F3F4F241754
:107E500090F3FB01E755F94F90837B010894E11CF7
:107E6000F11C00E010E0F801E755F94F80810E9415
:107E7000CE020F5F1F4F0E151F05A8F3B394B91460
:107E800008F4B1CF8091C105882309F427C384E8A1
:107E90008093A9061092AA061092AC06EFE9F3E0CF
:107EA000CC2406C0C39431964FEFC41609F499C48C
:107EB00080818823B9F78C2D60E30E943B87A82E30
:107EC000282F30E080ED9FEFFC012E9FC0012F9FF7
:107ED000900D3E9F900D11248C0D911D892B09F062
:107EE00082C4AA2009F455C0DD24BB2499249394AC
:107EF00041E3842EDC1408F078C4ED2DF0E0E15667
:107F0000FC4F80818093AD06D394AEEAB6E091E059
:107F10000BC0ED2DF0E0E156FC4F80818D939F5F0B
:107F2000D394903309F4BEC3DC1498F39F5F90930D
:107F3000AB06492F4D5F642F70E009F44CC490E00C
:107F400020E030E0F901E755F94F80819827E92FCB
:107F5000F0E0E75DFB4F90812F5F3F4F241790F3D8
:107F6000FB01E755F94F90837B010894E11CF11C5C
:107F700000E010E0F801E755F94F80810E94CE0241
:107F80000F5F1F4F0E151F05A8F3B394BA1408F422
:107F9000B1CF84E88093A9061092AA061092AC068D
:107FA000EFE8F3E0CC2406C0C39431964FEFC4163B
:107FB00009F48CC380818823B9F78C2D60E30E947B
:107FC0003B87982E282F30E080ED9FEFFC012E9FFD
:107FD000C0012F9F900D3E9F900D11248C0D911D7F
:107FE000892B09F075C3992009F455C0DD24BB2401
:107FF0008824839481E3A82EDC1408F098C3ED2D27
:10800000F0E0E157FC4F80818093AD06D394AEEA57
:10801000B6E091E00BC0ED2DF0E0E157FC4F808120
:108020008D939F5FD394903309F436C3DC1498F397
:108030009F5F9093AB06492F4D5F642F70E009F46A
:108040003DC390E020E030E0F901E755F94F808131
:108050009827E92FF0E0E75DFB4F90812F5F3F4FBE
:10806000241790F3FB01E755F94F90837B010894A7
:10807000E11CF11C00E010E0F801E755F94F8081A8
:108080000E94CE020F5F1F4F0E151F05A8F3B39479
:10809000B91408F4B1CF9091720284E88093A906D4
:1080A0001092AA0681E08093AC069093AD0682E020
:1080B0008093AB06A9EAB6E0E0E08D91E827F0E016
:1080C000E75DFB4FE081F6E0AE3ABF07B1F7E09322
:1080D000AE06F20181912F010E94CE026414750454
:1080E000C1F78AE00E945C1F882311F40C94D233FC
:1080F00089E00E94721F882311F40C94D23384E823
:108100008093A9061092AA061092AC06E0E8F3E06C
:10811000CC2406C0C39431964FEFC41609F469C24B
:1081200080818823B9F78C2D60E30E943B87982ECD
:10813000282F30E080ED9FEFFC012E9FC0012F9F84
:10814000900D3E9F900D11248C0D911D892B09F0EF
:1081500052C2992009F455C0DD24BB24882483949D
:1081600011E3A12EDC1408F0E8C2ED2DF0E0E05898
:10817000FC4F80818093AD06D394AEEAB6E091E0E7
:108180000BC0ED2DF0E0E058FC4F80818D939F5F98
:10819000D394903309F400C1DC1498F39F5F90935B
:1081A000AB06492F4D5F642F70E009F48FC190E05A
:1081B00020E030E0F901E755F94F80819827E92F59
:1081C000F0E0E75DFB4F90812F5F3F4F241790F366
:1081D000FB01E755F94F90837B010894E11CF11CEA
:1081E00000E010E0F801E755F94F80810E94CE02CF
:1081F0000F5F1F4F0E151F05A8F3B394B91408F4B1
:10820000B1CF2091C9053091CA053A83298384E80A
:108210008093A9061092AA0693E09093AC0620934F
:10822000AD068A818093AE069093AB0609EA16E00C
:10823000D801E0E08D91E827F0E0E75DFB4FE081B9
:10824000F6E0AF3ABF07B1F7EC93F80181918F01E7
:108250000E94CE02F6E0003B1F07B9F70C94D23320
:1082600089E00E94721F882359F080917202823047
:1082700038F080917202815080937202F1E0FC83A9
:108280008AE00E94721F882311F40C94E8338091D5
:1082900072028F3010F00C94E833809172028F5F7D
:1082A0008093720241E04C830E945F0E0E945457FB
:1082B000882311F40C94F0335C81552331F06091E4
:1082C000720283E190E00E94500329960FB6F89461
:1082D000DEBF0FBECDBFCF91DF911F910F91FF90F9
:1082E000EF90DF90CF90BF90AF909F908F907F9056
:1082F0006F905F904F903F902F90089589850E94D6
:1083000000250E941B2488850E9400250E94BD2311
:108310008F810E9400250E94852341E0341609F4D4
:10832000CFC10E94A72481E00E9478165D815F5F23
:108330005D838B815817B0F089858F5F60E50E945F
:108340003B87998788858F5F0E943B8798878F81BD
:108350008F5F0E943B879F838E818F5F0E943B8748
:108360009E831D8289E00E94721F882329F09B81D1
:10837000953010F091509B838AE00E94721F8823F1
:1083800011F40C94E133EB81E03610F00C94E133FE
:10839000EF5FEB830C94E133A092AB0644E364E31C
:1083A00070E005CFA092AB0644E364E370E040CDFB
:1083B000A092AB0644E364E370E0B8CCA092AB06B5
:1083C00044E364E370E006CCA092AB0644E364E3CC
:1083D00070E055CB9092AB0644E364E370E00C94FC
:1083E0000C35A092AB0644E364E370E09DCA909222
:1083F000AB0644E364E370E00C942137A092AB0633
:1084000044E364E370E0E5C99092AB0644E364E3BF
:1084100070E00C9459349092AB0644E364E370E04E
:108420000C94BC359092AB0644E364E370E00C948A
:108430006C36A092AB0644E364E370E01FC9A092DF
:10844000AB0644E364E370E06AC8A092AB0644E381
:1084500064E370E00C94E1392092AB0644E364E3FA
:1084600070E00C9430399092AB0644E364E370E022
:108470000C94D1372092AB0644E364E370E00C9493
:10848000823890E00C94933890E00C94323790E06E
:108490000C94E23790E0DDCC90E00C946A3490E0EC
:1084A0000C941D3590E051CA90E0A4C990E00C9462
:1084B0007D3690E0F4C890E00C94CD3590E040C853
:1084C00090E00C94F23990E00C94413990E080CE29
:1084D00090E03DCC90E08FCB90E0E2CA84E88093BE
:1084E000A9061092AA061092AC06E4EAF3E0CC24A6
:1084F00006C0C39431964FEFC41609F46EC1808153
:108500008823B9F78C2D60E30E943B87A82E282F83
:1085100030E080ED9FEFFC012E9FC0012F9F900D5A
:108520003E9F900D11248C0D911D892B09F057C190
:10853000AA2009F42ECDDD24BB249924939421E3B1
:10854000822EDC1408F04FC0ED2DF0E0EC55FC4F0E
:1085500080818093AD06D394AEEAB6E091E00BC083
:10856000ED2DF0E0EC55FC4F80818D939F5FD3940F
:10857000903309F49DC0DC1498F39F5F9093AB0691
:10858000492F4D5F642F70E009F423C190E020E093
:1085900030E0F901E755F94F80819827E92FF0E0A5
:1085A000E75DFB4F90812F5F3F4F241790F3FB0156
:1085B000E755F94F90837B010894E11CF11C00E022
:1085C00010E0F801E755F94F80810E94CE020F5F5D
:1085D0001F4F0E151F05A8F3B394BA1408F0D9CC99
:1085E000DC1408F4B1CF9092AB0644E064E070E094
:1085F000CDCF05E0902E9394ACCD75E0972E93945B
:10860000E9CBF5E09F2E939463CBB5E09B2E93943A
:10861000B3CA05E0902E939404CA95E0992E9394E2
:1086200055C935E0932E9394A6C855E0952E9394A2
:108630000C940F3B75E0972E93940C94603AF5E000
:108640009F2E93940C94B039B5E0AB2EA3940C9468
:10865000013905E0A02EA3940C94533825E0A22EF6
:10866000A3940C94A03745E0A42EA3940C94F03668
:1086700065E0A62EA3940C943B36E5E0AE2EA394C1
:108680000C948B35A5E0AA2EA3940C94DB3405E062
:10869000A02EA3940C942834A092AB0644E364E388
:1086A00070E0CFCC8092AB0644E364E370E047CC4B
:1086B0008092AB0644E364E370E068CF90E0D2CCF4
:1086C0008E810E9400250E94BD232BCE95E0992E1D
:1086D000939489CC8092AB0644E064E070E0A8CB30
:1086E0008092AB0644E064E070E0C9C98092AB06BA
:1086F00044E064E070E01ACB8092AB0644E064E0B2
:1087000070E068CA8092AB0644E064E070E00C94CC
:1087100059348092AB0644E064E070E00C940C3570
:108720008092AB0644E064E070E00C9421378092C4
:10873000AB0644E064E070E084CC8092AB0644E099
:1087400064E070E034CD8092AB0644E064E070E019
:1087500040C88092AB0644E064E070E00C943E3B7D
:108760008092AB0644E064E070E00C94D1378092D4
:10877000AB0644E064E070E00C94E13991E0909342
:10878000AB0644E064E070E00C94303981E0809303
:10879000AB0644E064E070E00C9482388092AB0653
:1087A00044E064E070E00C946C368092AB0644E0E8
:1087B00064E070E00C94BC358092AB0644E064E069
:1087C00070E00C948F3A8092AB0644E064E070E075
:1087D000ABC890E0ECCE90E0C3CB35E0A32EA394E1
:1087E000A7CE55E0A52EA3947CCB9092AB0644E097
:1087F00064E070E0A4CB2C98803408F08FE3611122
:1088000060E4442349F090E0882349F0682B962BDC
:1088100098B92C9A2D9A089590E88823B9F7962B49
:1088200098B90895882319F42D982C980895469A9C
:108830002C980895CF92DF92EF92FF920F931F939F
:10884000CF93DF930E9492240E94F22780916206C8
:108850000E9442270E9445220E94F21F8091EC054F
:108860006091ED05662309F0D3C020E030E0882355
:1088700009F4D3C0C901880F991F820F931FD82E06
:10888000DD0CDD0C83E00E94D72384E06091EC05D1
:108890000E94D72388E06091EB050E94D723EE2445
:1088A000CC24C3940E9445220E945F0E0E9454571C
:1088B000882309F07BC01D2D185EC0E0D0E014C0F5
:1088C000802F0E94881F882351F08091EB05811131
:1088D00080E8812B0E9400188F2D0E94ED2A21969E
:1088E0001F5FCD30D105F1F0FC2EFE01E75DFA4FA0
:1088F0000081802F0E94721F882311F3812F8D50D9
:108900006E2D4091EB050E94FB438091EB05811198
:1089100080E8812B0E94DA178F2D0E946527EE24B4
:10892000E394CECF8FE00E94721F882309F449C0E0
:108930006091ED056C256093ED0583E00E94D723DF
:108940009091EC058091ED05882309F04EC020E060
:1089500030E0992311F421E030E0C901880F991F1C
:10896000820F931FD82EDD0CDD0C84E10E94721F54
:10897000882309F044C086B190E08F739070892BF2
:1089800009F490CF0E949E1F882309F48BCF80E0CA
:108990000E9412440E943029EE240E9445220E9427
:1089A0005F0E0E945457882309F485CF0E94551802
:1089B000DF91CF911F910F91FF90EF90DF90CF90BB
:1089C00008958EE00E94721F882379F26091EC0571
:1089D0006C256093EC0584E00E94D7239091EC0510
:1089E0008091ED05882309F4B2CF8923E1F084E278
:1089F000D82E84E10E94721F882309F4BCCF6091B5
:108A0000EB056C256093EB0588E00E94D723B3CF7C
:108A1000862331F054E2D52E35CF21E030E02ACF45
:108A200078E1D72E2FCF98E1D92E9FCF282FF89419
:108A300095E0289800000000000000009EBD0DB4E5
:108A400007FEFDCF00000000000000001EBC0DB4BA
:108A500007FEFDCF8EB5289A000000000000000040
:108A600080FDE7CF28980000000086E08EBD0DB4A1
:108A700007FEFDCF00000000289A00000000000063
:108A8000000028980000000082E08EBD0DB407FEB3
:108A9000FDCF7EBD0DB407FEFDCF6EBD0DB407FE4C
:108AA000FDCF2EBD0DB407FEFDCF00000000289ABB
:108AB00078940895382FF89425E028980000000055
:108AC000000000002EBD0DB407FEFDCF0000000029
:108AD000000000001EBC0DB407FEFDCF8EB5289A25
:108AE000000000000000000080FDE7CF2898000093
:108AF000000083E08EBD0DB407FEFDCF9EBD0DB41A
:108B000007FEFDCF3EBD0DB407FEFDCF0000000007
:108B10001EBC0DB407FEFDCF8EB5289A789408953B
:108B2000382FF89425E0289800000000000000008D
:108B30002EBD0DB407FEFDCF0000000000000000B8
:108B40001EBC0DB407FEFDCF8EB5289A00000000B4
:108B50000000000080FDE7CF28980000000083E0BF
:108B60008EBD0DB407FEFDCF9EBD0DB407FEFDCF3B
:108B70003EBD0DB407FEFDCF00000000662389F066
:108B80006150FA01CA01860F911DBC011EBC0DB4D3
:108B900007FEFDCF8EB58083E617F70711F03196FB
:108BA000F5CF289A78940895892F8F7184FD806E6F
:108BB0000895EF92FF920F931F93FA01D9018695C2
:108BC0008083862F90E08F7090709595879595950E
:108BD0008795959587958C93862F8770F80180836C
:108BE00062956F70F70160831F910F91FF90EF9076
:108BF0000895FC0130E022953295307F3227207FA6
:108C0000322720838081660F660F660F640F6F70B6
:108C1000862B808308958091E905882349F087FD9C
:108C20000EC083E00E94852384E00E941B240895E7
:108C300083E00E941B2484E00E941B24089583E0AB
:108C40000E941B2484E00E9485230895962F803182
:108C500010F08FEF0895682F70E0660F771F6F5F39
:108C6000734F892F0E94164580E008959B01803143
:108C700020F5682F70E0FB01EE0FFF1FEA5CFA4F52
:108C80008081918128173907A0F0009749F0815021
:108C9000660F771F6050744F0E94164580E008955C
:108CA00080E0660F771F6050744F0E94164580E089
:108CB0000895C901009759F7F3CF8FEF08958031D8
:108CC00098F470E06050784F90E000249695879576
:108CD0000794969587950794982F802D680F791F94
:108CE0008CE06030780710F08FEF0895842F0E9499
:108CF000164580E00895EF92FF920F931F93CF9354
:108D0000DF93C82FD0E0CC0FDD1FCC0FDD1FCC0FC1
:108D1000DD1FC60FD11DC05CDF4FCC0FDD1FC2951C
:108D2000D295D07FDC27C07FDC27EE24FF2487018B
:108D3000000F111F075D184FF80180819181892F65
:108D4000BE010E941645F801808191812196BE01E5
:108D50000E9416450894E11CF11C2196F0E1EF16E3
:108D6000F10429F7DF91CF911F910F91FF90EF90C0
:108D7000089590E0880F991F8F5F934F0E945A4586
:108D800090E008950F931F93082F10E0000F111F1C
:108D9000C8018050944F0E945A4590E001960A5CA9
:108DA0001A4FF801208131818217930708F49C0142
:108DB000C9011F910F910895803198F470E06050BF
:108DC000784F90E00024969587950794969587951F
:108DD0000794982F802D680F791F8CE060307807FA
:108DE00010F08FEF0895CB010E945A450895EF923D
:108DF000FF920F931F938091490790914A0780E05B
:108E00000E94B11F882309F07DC080915E078230E7
:108E100009F491C080915E07843009F4B0C080915C
:108E20005E0780FD47C080E00E94881F882329F4E8
:108E30001F910F91FF90EF90089582E20E94852389
:108E400080915E07823009F4C5C0209158073091A7
:108E5000590780915E07843009F4B5C010925E070F
:108E600021153105B9F0E0915B07F0E0EE0FFF1F2F
:108E7000EA5CFA4F808191818217930758F0215064
:108E8000304030934A07209349078091DB088823BC
:108E900009F4F2C08091A605823028F00E941B28B8
:108EA00081E08093F6051092A6051F910F91FF9027
:108EB000EF9008950E942A20482F882309F0BEC011
:108EC00084E10E94721F882309F0A9C085E10E94F5
:108ED000721F882309F094C087E10E94721F8823C3
:108EE00009F083C083E00E94721F882309F49BCF9E
:108EF00080915407909155070E94EB0283E0809384
:108F0000A60591CF81E080935E07109259071092D9
:108F1000580782E20E941B248091490790914A07DA
:108F200001960E94EB0282E08093A60580915E0785
:108F3000823009F06FCF0E942A20482F882309F43D
:108F400069CF41502091580730915907C901880FC6
:108F5000991F880F991F880F991F220F331F820FA7
:108F6000931F840F911D90935907809358078C5934
:108F70009F4F0E94EB0283E08093A6054BCF0E9497
:108F80002A20482F882309F44ACF415020915807BE
:108F900030915907C901880F991F880F991F880FB1
:108FA000991F220F331F820F931F840F911D9093DF
:108FB00059078093580788539F4F0E94EB0283E024
:108FC0008093A6052CCF28533F4F30935907209309
:108FD000580744CF20915807309159072C593F4FDB
:108FE000309359072093580734CF80915C079091B4
:108FF0005D0701960E94EB0283E08093A60572CF85
:1090000084E080935E07109259071092580788EC0D
:1090100090E00E94EB0283E08093A6055DCF82E0A2
:1090200080935E07109259071092580784E690E0EB
:109030000E94EB0283E08093A60548CF13E01093D3
:109040005E0741502091580730915907C901880F98
:10905000991F880F991F880F991F220F331F820FA6
:10906000931F840F911D90935907809358070E9476
:10907000EB021093A60524CF80915B07609149070E
:1090800070914A070E94DC468093510780915B07EC
:109090006091510749EA57E021E637E003E617E01F
:1090A00097E7E92E98E0F92E0E94D94581E0809358
:1090B000F1070E94765EEECEAF92BF92CF92DF9222
:1090C000EF92FF920F931F93CF93DF93C82EDD246F
:1090D000CC0CDD1CCC0CDD1CCC0CDD1CC60ED11C5C
:1090E00080E490E0C80ED91ECC0CDD1CC294D29452
:1090F00010EFD122DC24C122DC24AA24BB24C60127
:109100000E945A45D82FC0E07501EE0CFF1CE9E221
:10911000F7E0EE0EFF1EF701D183C08300811181BD
:10912000C60101960E945A4590E0082B192BF701C1
:10913000118300830894A11CB11C82E090E0C80E4A
:10914000D91E90E1A916B104D1F6DF91CF911F91FC
:109150000F91FF90EF90DF90CF90BF90AF90089568
:109160001092530784E20E941B240E9492240E94C2
:10917000E7241092EF0780E00E94124408951092B5
:1091800052071092EF0710924B0780E00E941244A2
:109190000E9492240E94E7240E94F21F0895809169
:1091A0004F0790915007682F677096958795969511
:1091B0008795969587958F700E941A5C60914F07EE
:1091C000709150079B0140E050E0DA01C9018070C6
:1091D0009078A070B070892F9A2FAB2FBB27809307
:1091E0002F06DA01C90180709074A070B070892FC9
:1091F0009A2FAB2FBB2780932D06207030724070C2
:109200005070232F342F452F552720932E06109270
:109210006407872F8F7184FD806E089581E08093AD
:10922000530784E20E9485230E94F2270895CF937A
:10923000DF938091980680935B0780915B07C82F2E
:10924000D0E0CC0FDD1FCE018050944F0E945A45D4
:10925000282F30E0CA5CDA4F888199812F5F3F4F19
:109260008217930708F49C01309355072093540705
:1092700080915B0790E0880F991F8F5F934F0E944A
:109280005A4590E090935D0780935C0720915C07BE
:1092900030915D0780915407909155072817390741
:1092A00020F010925D0710925C0780914907909121
:1092B0004A07E0915B07F0E0EE0FFF1FEA5CFA4F10
:1092C000608171810E94478790934A078093490784
:1092D000DF91CF910895DF92EF92FF920F931F934A
:1092E000CF93DF93C0914907D0914A07219680E040
:1092F0000E94B11F882309F0DFC0DD2480915E0742
:10930000823009F4ECC080915E07843009F4ACC16E
:1093100080915E0780FD1AC080E00E94881F88232C
:1093200029F080915E07882309F020C181E0D816DA
:1093300009F47FC193E0D91609F489C1DF91CF9177
:109340001F910F91FF90EF90DF9008950E942A20C7
:10935000282F882309F0EEC084E10E94721F882321
:1093600009F0C2C185E10E94721F882309F0ADC1D6
:1093700087E10E94721F882339F0C0915C07D09169
:109380005D072196B3E0DB2E83E00E94721F8823E5
:1093900009F0C9C089E00E94721F882309F021C228
:1093A00089E00E94881F882309F0ADC18AE00E94ED
:1093B000721F882309F07CC18AE00E94881F8823DD
:1093C00009F4AACF8CE10E941B24E0915B07209155
:1093D000540730915507F0E0EE0FFF1FEA5CFA4F9B
:1093E000808191812817390708F096CF8091540722
:1093F000909155070196909355078093540780915B
:109400005B0760915407709155070E943646809122
:109410005B070E94C24690935507809354070091C2
:1094200054071091550701501040809149079091C1
:109430004A0780179107E0F580915B078031B0F40F
:10944000282F30E0002436952795079436952795E8
:109450000794322F202D2050384F802F8150280F15
:10946000311D9CE02030390708F4C8C18FEF6091AE
:109470005B076031A0F470E000247695679507944F
:10948000769567950794762F602D6050784F600F22
:10949000711D2CE06030720710F40E9416450150D7
:1094A00010408091490790914A078017910720F258
:1094B00088E08093F60530CF81E080935E071092BC
:1094C0005907109258078093F30582E20E941B24EB
:1094D000DD24D39480915E07823009F014CF0E947E
:1094E0002A20482F882309F40ECF41502091580795
:1094F00030915907C901880F991F880F991F880F4C
:10950000991F220F331F820F931F840F911D909379
:109510005907809358078C599F4F0E94EB0283E0B4
:109520008093A605F0CEC0915407D0915507A3E0D3
:10953000DA2E30CF83E080935E0721508091580768
:1095400090915907EC01CC0FDD1FCC0FDD1FCC0F24
:10955000DD1F880F991FC80FD91FC20FD11DD093CF
:109560005907C093580713E0D12EF6CE82E20E942D
:1095700085231092F30580915E07823009F449C17A
:10958000209158073091590780915E07843009F483
:1095900039C110925E0721153105C1F1E0915B07D9
:1095A000F0E0EE0FFF1FEA5CFA4F80819181821795
:1095B000930760F12150304030934A0720934907C8
:1095C00088E08093F6058091DB088823F9F4809188
:1095D0005B076091490770914A070E94DC468093BF
:1095E000510780915B076091510749EA57E021E6F6
:1095F00037E003E617E097E7E92E98E0F92E0E949E
:10960000D94581E08093F1070E94765E8091A6059E
:10961000823048F00E941B288091F605882319F4B7
:1096200081E08093F6051092A60581E0D81609F036
:1096300081CECE010E94EB0282E08093A605DF91ED
:10964000CF911F910F91FF90EF90DF900895CE0181
:109650000E94EB02D092A605DF91CF911F910F914E
:10966000FF90EF90DF9008950E942A20482F8823D2
:1096700009F44ECE41502091580730915907C90145
:10968000880F991F880F991F880F991F220F331F6A
:10969000820F931F840F911D909359078093580751
:1096A00088539F4F0E94EB0283E08093A60530CE43
:1096B0008CE10E9485231092590710925807C0919F
:1096C0004907D0914A07219677CE84E080935E07C0
:1096D000109259071092580788EC90E00E94EB0214
:1096E00083E08093A60544CE82E080935E071092CB
:1096F00059071092580784E690E00E94EB0283E03D
:109700008093A6052FCE8BE10E941B240091490770
:1097100010914A070F5F1F4F809154079091550792
:109720000817190708F042CE80915B07803198F442
:1097300090E00024969587950794969587950794D1
:10974000982F802D8050984F800F911D2CE08030F5
:10975000920708F442C09FEF60915B076031B8F454
:1097600070E0002476956795079476956795079441
:10977000762F602D6050784F802F8150680F711DBB
:109780008CE06030780718F4892F0E9416450F5F2F
:109790001F4F80915407909155070817190720F221
:1097A00080915407909155070197909355078093A6
:1097B000540780915B0760915407709155070E9490
:1097C000364680915B070E94C2469093550780936E
:1097D000540788E08093F605E9CD0E945A45982FFA
:1097E000BBCF8BE10E948523109259071092580736
:1097F000C0914907D0914A072196D2CDC9010E9454
:109800005A4535CE28533F4F309359072093580778
:10981000C0CE20915807309159072C593F4F3093B3
:10982000590720935807B0CEEF92FF920F931F93E2
:10983000CF93DF931092EE058091DB08882309F423
:1098400030C284E00E94345910924E0780914E0736
:1098500080934D0710925E0710925A071092590795
:10986000109258078091980680935B0780915B0760
:10987000C82FD0E0CC0FDD1FCE018050944F0E9446
:109880005A45282F30E0CA5CDA4F888199812F5FD2
:109890003F4F8217930708F49C013093550720939C
:1098A000540780915B0790E0880F991F8F5F934F5B
:1098B0000E945A4590E090935D0780935C07209149
:1098C0005C0730915D0780915407909155072817E8
:1098D000390720F010925D0710925C0780914907CC
:1098E00090914A07E0915B07F0E0EE0FFF1FEA5C02
:1098F000FA4F608171810E94478790934A07809355
:10990000490710E0FF24F3940E9445220E945F0E55
:1099100000917408013089F0043009F48DC00E9470
:109920007D5A882389F70E94405A0E9445220E944E
:109930005F0E00917408013079F70E943A5988232C
:1099400009F0BBC0113009F4E0C0112309F449C18A
:10995000123009F451C18091F605882309F0A5C0A1
:1099600090915B0780919806981709F44FC08091F9
:10997000980680935B0780915B07C82FD0E0CC0FDF
:10998000DD1FCE018050944F0E945A45282F30E0B1
:10999000CA5CDA4F888199812F5F3F4F8217930706
:1099A00008F49C01309355072093540780915B077E
:1099B00090E0880F991F8F5F934F0E945A4590E067
:1099C00090935D0780935C0720915C0730915D0761
:1099D00080915407909155072817390720F010926D
:1099E0005D0710925C078091490790914A07E091CA
:1099F0005B07F0E0EE0FFF1FEA5CFA4F60817181B8
:109A00000E94478790934A07809349078091740882
:109A1000813011F0109233068091DB088823E1F544
:109A20000E945457882309F47ACFDF91CF911F9178
:109A30000F91FF90EF9008950E943A59882309F002
:109A40008CC080915B0786958093A206113009F443
:109A5000B3C0112309F4DAC0123009F4E1C08091D7
:109A60007408843011F0109233068091DB0888234B
:109A700009F46DC080913206813009F050CF109208
:109A800032068091EE05882309F049CF0E94545791
:109A9000882309F444CFC9CF84E00E9434590E943E
:109AA0005457882309F43BCFC0CF1092F60581E0CC
:109AB00061E042E00E94B65753CF0E94922482E2B6
:109AC0000E9485230093330681E061E042E00E941A
:109AD000B65781E20E941B248091EA076091F0074B
:109AE000409163072091F1070091EA07E090610738
:109AF0000E945B2B8091EE05882309F4A4C083E2C9
:109B00000E948523113009F020CF0E940766882328
:109B100009F06BC083E00E94B11F8823B1F08091EF
:109B2000EE058F5F8093EE058091EE058170809346
:109B3000EE058091EE05882309F48DC083E20E9432
:109B4000852310924A071092490710E004CF81E064
:109B50000E9434591092EE058DCF0E94922482E229
:109B60000E948523F092330681E061E042E00E948A
:109B7000B65781E20E9485238091EA076091F00741
:109B8000409163072091F1070091EA07E090610797
:109B90000E945B2B8091EE05882309F458C083E274
:109BA0000E94A1230E94A72480915B078695809341
:109BB000A206113009F04DCF0E940766882351F5A7
:109BC00083E00E94721F882329F08091EE05813086
:109BD00009F461C087E10E94721F882369F510E0D3
:109BE0003ECF0E940766882311F011E0B4CE0E9498
:109BF0005C1F882309F48ECF0E94F74680E00E9404
:109C00005C1F882309F486CF12E0A5CE0E94076668
:109C1000882311F011E023CF0E945C1F882381F27A
:109C200080E00E94721F882369F580E00E94881FEF
:109C30008823A9F412E013CFF0924E0780E00E942F
:109C4000A12310E00CCF83E20E941B247BCE83E291
:109C50000E941B24A7CF83E20E941B2472CF82E2C2
:109C60000E94852310925E078091A605823010F035
:109C70000E941B281092A60581E061E042E00E944C
:109C8000B6579ECFF0925E0782E20E941B2482E0CC
:109C90008093A605CACF80934D0783E20E94852357
:109CA00099CF81E00E943459CFCD81E08093520753
:109CB00081E20E94852310922D0680912D068093CB
:109CC0002E0680912E0680932F0610924B0710923D
:109CD000EF078091290790912A079093500780936E
:109CE0004F072FEF8F3F920709F448C01092570794
:109CF0001092640710923C06682F677096958795BE
:109D000096958795969587958F700E941A5C6091BD
:109D10004F07709150079B0140E050E0DA01C90104
:109D200080709078A070B070892F9A2FAB2FBB27CE
:109D300080932F06DA01C90180709074A070B07012
:109D4000892F9A2FAB2FBB2780932D06207030725E
:109D500040705070232F342F452F552720932E0607
:109D6000109264077F7174FD706E7093E9058091A5
:109D70009D0580FDFCCF81E080934B070E94F22778
:109D80000895CF93DF938091980680935B0780912D
:109D90005B07C82FD0E0CC0FDD1FCE018050944F61
:109DA0000E945A45282F30E0CA5CDA4F8881998199
:109DB0002F5F3F4F8217930708F49C01309355079C
:109DC0002093540780915B0790E0880F991F8F5F65
:109DD000934F0E945A4590E090935D0780935C07F3
:109DE00020915C0730915D07809154079091550751
:109DF0002817390720F010925D0710925C078091B8
:109E0000490790914A07E0915B07F0E0EE0FFF1FD2
:109E1000EA5CFA4F608171810E94478790934A07FC
:109E20008093490740915B078091490790914A07C9
:109E30004031A8F4282F30E02050384F842F90E094
:109E40000024969587950794969587950794982F63
:109E5000802D280F391F8CE02030380750F18FEF0C
:109E60008093510780915B072091510786958093DD
:109E7000A907822F90E08F709070959587959595A2
:109E800087959595879580936107822F877080933A
:109E9000630722952F702093770881E08093F10764
:109EA0008091DB08882311F40E94765EDF91CF91C8
:109EB0000895C9010E945A45D3CFEF92FF920F93A4
:109EC0001F93CF93DF938091DB08882309F482C22C
:109ED00084E00E94345910924E0780914E0780937F
:109EE0004D0710925E0710925A0710925907109270
:109EF00058078091980680935B0780915B07C82F75
:109F0000D0E0CC0FDD1FCE018050944F0E945A4507
:109F1000282F30E0CA5CDA4F888199812F5F3F4F4C
:109F20008217930708F49C01309355072093540738
:109F300080915B0790E0880F991F8F5F934F0E947D
:109F40005A4590E090935D0780935C0720915C07F1
:109F500030915D0780915407909155072817390774
:109F600020F010925D0710925C0780914907909154
:109F70004A07E0915B07F0E0EE0FFF1FEA5CFA4F43
:109F8000608171810E94478790934A0780934907B7
:109F900040915B078091490790914A074031B0F4A6
:109FA000282F30E02050384F842F90E000249695E1
:109FB00087950794969587950794982F802D280F5D
:109FC000391F8CE02030380708F40CC28FEF8093E3
:109FD000510780915B072091510786958093A907CF
:109FE000822F90E08F7090709595879595958795C5
:109FF0009595879580936107822F8770809363077B
:10A0000022952F702093770881E08093F10780914B
:10A01000DB08882311F40E94765E10E0FF24F3949D
:10A020000E9445220E945F0E00917408013009F4DD
:10A0300055C0043089F001E00E947D5A882309F45C
:10A040004AC0002369F71092A605DF91CF911F91B6
:10A050000F91FF90EF9008950E943A59882309F0DC
:10A060004EC180915B0786958093A206143009F457
:10A0700073C1133009F4A8C1123009F48CC1112343
:10A0800009F46FC1113009F415C28091F6058823D7
:10A0900009F071C180917408843011F01092330678
:10A0A0008091DB08882309F46EC10E9462578823DF
:10A0B00061F480913206813009F0BDCF10923206F2
:10A0C0000E945457882309F4B6CF00E00E947D5ABD
:10A0D000882309F0B6CF0E94405AB3CF0E943A5964
:10A0E000882309F0D3C0133009F4F3C0123009F407
:10A0F000BFC0112309F4C4C0113009F477C18091A5
:10A10000F605882309F0ACC090915B078091980612
:10A11000981709F493C08091980680935B0780910B
:10A120005B07C82FD0E0CC0FDD1FCE018050944FCD
:10A130000E945A45282F30E0CA5CDA4F8881998105
:10A140002F5F3F4F8217930708F49C013093550708
:10A150002093540780915B0790E0880F991F8F5FD1
:10A16000934F0E945A4590E090935D0780935C075F
:10A1700020915C0730915D078091540790915507BD
:10A180002817390720F010925D0710925C07809124
:10A19000490790914A07E0915B07F0E0EE0FFF1F3F
:10A1A000EA5CFA4F608171810E94478790934A0769
:10A1B0008093490740915B078091490790914A0736
:10A1C0004031B0F4282F30E02050384F842F90E0F9
:10A1D0000024969587950794969587950794982FD0
:10A1E000802D280F391F8CE02030380708F4F6C086
:10A1F0008FEF8093510780915B07209151078695DF
:10A200008093A907822F90E08F7090709595879525
:10A21000959587959595879580936107822F87708F
:10A220008093630722952F7020937708F092F107AF
:10A230008091DB08882311F40E94765E8091740877
:10A24000813011F0109233068091DB08882309F0E9
:10A250009EC00E945457882309F4EDCE00E036CF0B
:10A260001092F60581E060E041E00E94B6574CCFC5
:10A270000E94F74680E00E945C1F882309F03FCFD0
:10A280000E940766882371F111E039CF0E94922461
:10A2900082E20E9485230093330681E060E041E082
:10A2A0000E94B65781E20E941B248091EA076091C8
:10A2B000F007409163072091F1070091EA07E090D1
:10A2C00061070E945B2B81E00E942703133009F095
:10A2D0000DCF0E94625A882309F011CF0E940766B1
:10A2E000882391F680E00E945C1F882309F016C144
:10A2F0000E94625A882309F47EC013E000CF0E94B6
:10A30000922482E20E948523F09233060091BB05DD
:10A3100081E060E041E00E94B657033009F4FBC0E1
:10A3200081E20E9485238091EA076091F0074091C5
:10A3300063072091F1070091EA07E09061070E940E
:10A340005B2B81E00E94270380915B0786958093B9
:10A35000A206143009F08DCE0E94C457882309F05C
:10A3600094CE0E940766882311F111E08091F605D2
:10A37000882309F48FCE1092F60581E060E041E079
:10A380000E94B65787CE81E00E9434598ECE84E079
:10A390000E9434595ECF0E94F74680E00E945C1F05
:10A3A000882309F072CE0E9407668823F1F680E0C8
:10A3B0000E945C1F882309F0B5C00E94625A88235E
:10A3C00009F4B8C013E061CE0E94625A882309F0F4
:10A3D0005CCEC7CF81E00E9434597DCDC9010E9477
:10A3E0005A4507CFC9010E945A45F1CD0E94076620
:10A3F000882309F084CE83E00E94B11F882361F492
:10A4000083E00E94881F882311F410E078CE83E255
:10A410000E941B2410E073CE10924A071092490745
:10A4200040915B078091490790914A074031B0F411
:10A43000282F30E02050384F842F90E0002496954C
:10A4400087950794969587950794982F802D280FC8
:10A45000391F8CE02030380708F468C08FEF8093F4
:10A46000510780915B072091510786958093A9073A
:10A47000822F90E08F709070959587959595879530
:10A480009595879580936107822F877080936307E6
:10A4900022952F7020937708F092F1070E94765E44
:10A4A00083E20E94852383E00E94881F882309F4A9
:10A4B000ACCFADCF0E940766882309F0E6CD86E1D8
:10A4C0000E94721F882369F483E00E94721F882310
:10A4D000B9F40E947020882311F0F092BA0510E0C0
:10A4E000D4CDF0924E0780E00E94852310924D0754
:10A4F00083E20E941B2483E00E94721F882349F399
:10A50000F0924D0783E20E94852310924E0780E06F
:10A510000E941B24DECF0093BB0502CF0E94F746AA
:10A5200012E0EDCD0E94F74612E0AFCDC9010E94C6
:10A530005A4595CF0E94C457882309F214E0A5CD4F
:10A54000EF92FF920F931F93CF93DF938091DB08DD
:10A55000882309F49DC484E00E94345910924E0768
:10A5600080914E0780934D0710925E0710925A0714
:10A5700010925907109258078091980680935B07B4
:10A5800080915B07C82FD0E0CC0FDD1FCE0180503B
:10A59000944F0E945A45282F30E0CA5CDA4F8881D8
:10A5A00099812F5F3F4F8217930708F49C013093E6
:10A5B00055072093540780915B0790E0880F991FFF
:10A5C0008F5F934F0E945A4590E090935D07809370
:10A5D0005C0720915C0730915D0780915407909152
:10A5E00055072817390720F010925D0710925C0775
:10A5F0008091490790914A07E0915B07F0E0EE0FE8
:10A60000FF1FEA5CFA4F608171810E944787909337
:10A610004A078093490740915B07809149079091D1
:10A620004A074031B0F4282F30E02050384F842FB3
:10A6300090E00024969587950794969587950794C2
:10A64000982F802D280F391F8CE02030380708F410
:10A6500027C48FEF8093510780915B0720915107AA
:10A6600086958093A907822F90E08F7090709595C2
:10A670008795959587959595879580936107822F06
:10A6800087708093630722952F702093770881E06D
:10A690008093F1078091DB08882311F40E94765E95
:10A6A00010E0F8E0FF2E0E9445220E945F0E00910C
:10A6B0007408013089F0043009F452C10E947D5AB7
:10A6C000882389F70E94405A0E9445220E945F0E0B
:10A6D00000917408013079F70E943A59882309F0F3
:10A6E00007C280915B0786958093A20690915B07D5
:10A6F00080919806981709F494C0809198068093E9
:10A700005B0780915B07C82FD0E0CC0FDD1FCE0127
:10A710008050944F0E945A45282F30E0CA5CDA4F8F
:10A72000888199812F5F3F4F8217930708F49C011E
:10A73000309355072093540780915B0790E0880F72
:10A74000991F8F5F934F0E945A4590E090935D0749
:10A7500080935C0720915C0730915D0780915407DE
:10A76000909155072817390720F010925D07109235
:10A770005C078091490790914A07E0915B07F0E000
:10A78000EE0FFF1FEA5CFA4F608171810E944787DC
:10A7900090934A078093490740915B07809149074E
:10A7A00090914A074031B0F4282F30E02050384FC4
:10A7B000842F90E000249695879507949695879529
:10A7C0000794982F802D280F391F8CE020303807F0
:10A7D00008F48AC18FEF8093510780915B07209125
:10A7E000510786958093A907822F90E08F70907013
:10A7F000959587959595879595958795809361070C
:10A80000822F87708093630722952F70209377089B
:10A8100081E08093F1078091DB08882311F40E9486
:10A82000765E123009F48EC1112309F493C1113000
:10A8300009F49DC286E10E94721F882309F474C046
:10A8400080914E07882309F020C28091F007882369
:10A8500011F140E04F5F8091490790914A070196BE
:10A8600090934A07809349078091490790914A073E
:10A87000E0915B07F0E0EE0FFF1FEA5CFA4F6081AA
:10A8800071810E94478790934A078093490780917E
:10A89000F0074817F8F280914D07882309F0EFC1BF
:10A8A000123009F4DFC140915B0780914907909114
:10A8B0004A074031B0F4282F30E02050384F842F21
:10A8C00090E0002496958795079496958795079430
:10A8D000982F802D280F391F8CE02030380708F47E
:10A8E000FFC08FEF8093510780915B072091510744
:10A8F00086958093A907822F90E08F709070959530
:10A900008795959587959595879580936107822F73
:10A9100087708093630722952F702093770881E0DA
:10A920008093F1078093F6058091F605882309F05E
:10A9300001C180917408813011F01092330680912A
:10A94000DB08882309F0F2C00E945457882309F4D9
:10A95000B5CEDF91CF911F910F91FF90EF900895A9
:10A960000E943A59882309F00FC180915B078695B0
:10A970008093A206123009F4F8C0112309F4FDC037
:10A98000113009F40AC286E10E94721F882309F47B
:10A990007FC08091F107882309F09DC180917708DD
:10A9A00080937C08C0914907D0914A0780914E0757
:10A9B000882309F070C18091F007882309F45EC0F4
:10A9C00000E02091CE083091EA0780917C0890E069
:10A9D00082959295907F9827807F98278093510742
:10A9E00080915107220F220F220F230F200F2F706B
:10A9F000282B2093510780915B0760914907709144
:10AA00004A07209151078031B0F470E06050784FD0
:10AA100090E00024969587950794969587950794DE
:10AA2000982F802D680F791F8CE06030780718F41C
:10AA3000822F0E9416450F5F8091490790914A0727
:10AA4000019690934A078093490721968091490780
:10AA500090914A07E0915B07F0E0EE0FFF1FEA5C80
:10AA6000FA4F608171810E94478790934A078093D3
:10AA700049078091F007081708F4A3CF80914D078C
:10AA8000882309F038C1F092F605123009F426C186
:10AA90008091F605883009F49CC08091F6058130DC
:10AAA00009F490C080917408843011F0109233063C
:10AAB0008091DB08882309F454C0809132068130EC
:10AAC00009F0FCCD109232060E945457882309F4F5
:10AAD000F5CDDF91CF911F910F91FF90EF900895E9
:10AAE000C9010E945A45FECEC9010E945A4573CE43
:10AAF0000E94922482E20E9485230093330681E023
:10AB000060E041E00E94B65781E20E941B248091E0
:10AB1000EA076091F007409163072091F1070091E7
:10AB2000EA07E09061070E945B2BDBCD84E00E9486
:10AB300034590ACF1092F6050E94765E81E0809328
:10AB4000FA05F7CE0E946B4980E00E945C1F8823C3
:10AB500009F070CE0E940766882309F48DC111E0C8
:10AB600069CE81E00E943459A8CF0E946B4980E0F1
:10AB70000E945C1F882309F006CF0E940766882385
:10AB800009F42AC111E0FFCE0E94922482E20E94C1
:10AB9000852381E08093330661E042E00E94B6574E
:10ABA00081E20E9485238091EA076091F00740913D
:10ABB00063072091F1070091EA07E09061070E9486
:10ABC0005B2BD3CE1092F60561E042E00E94B657AF
:10ABD00069CF40915B078091490790914A074031C6
:10ABE000A8F4282F30E02050384F842F90E0002424
:10ABF000969587950794969587950794982F802D1D
:10AC0000280F391F8CE02030380740F18FEF8093F8
:10AC1000510780915B072091510786958093A90782
:10AC2000822F90E08F709070959587959595879578
:10AC30009595879580936107822F8770809363072E
:10AC400022952F702093770881E08093F10761E0CF
:10AC500042E00E94B6571092F6051FCFC9010E942C
:10AC60005A45D5CF8091A605833009F41CCE80913A
:10AC7000490790914A0701960E94EB0214CE109268
:10AC80004D0783E20E941B240BCE10924E0780E0FA
:10AC90000E941B24DACD10924E0760915B07603151
:10ACA00040F470E0660F771F6F5F734F8C2F0E9428
:10ACB000164580915B0790E0880F991F8F5F934F37
:10ACC0000E945A4590E090935D0780935C0780E076
:10ACD0000E941B2470CE0E94A35760CE8091A605CF
:10ACE000833009F4D5CE8091490790914A070196A7
:10ACF0000E94EB02CDCE10924D0760915B07603150
:10AD0000B8F470E0FB01EE0FFF1FEA5CFA4F208100
:10AD100031812C173D0708F09E012115310509F0FE
:10AD2000B4C080E0660F771F6050744F0E941645D4
:10AD300080915B07C82FD0E0CC0FDD1FCE01805083
:10AD4000944F0E945A45282F30E0CA5CDA4F888120
:10AD500099812F5F3F4F8217930708F49C0130932E
:10AD600055072093540783E20E941B248CCE0E9437
:10AD70000766882309F05ECD83E00E94721F882356
:10AD800099F583E00E94881F882311F410E052CDCA
:10AD900083E20E941B2410E04DCD0E9407668823A9
:10ADA00009F0F1CD83E00E94721F882331F081E029
:10ADB00080934D0783E20E94A12387E10E94721FC6
:10ADC000882311F410E0DFCD81E080934E0780E00E
:10ADD0000E94A12310E0D7CD0E945C1F882311F3AD
:10ADE0000E946B4912E0CFCD10924A07109249079A
:10ADF00040915B078091490790914A074031A8F440
:10AE0000282F30E02050384F842F90E00024969572
:10AE100087950794969587950794982F802D280FEE
:10AE2000391F8CE020303807B8F18FEF809351073D
:10AE300080915B072091510786958093A907822F07
:10AE400090E08F70907095958795959587959595DD
:10AE5000879580936107822F87708093630722957F
:10AE60002F702093770881E08093F1078093F60597
:10AE700083E20E94852385CF0E945C1F882309F40A
:10AE80007BCF0E946B4912E0D5CC822F81504ACFF4
:10AE900081E00E94345962CBC9010E945A45C6CF55
:10AEA000C9010E945A45D6CB9091970680919D0684
:10AEB000891731F08091970680939D0681E008956F
:10AEC00080E008959091970680919D06891781F002
:10AED000809197068D3071F080919706853051F002
:10AEE00080919706833031F080919706813011F080
:10AEF00080E008958091970680939D0681E00895F3
:10AF00008091F107882391F08091A90780938D08A3
:10AF1000809161078093CE08809163078093EA0750
:10AF20008091F1078093F0071092F1078091F0076C
:10AF3000882329F08091F0078093F007089581E03D
:10AF40008093F00708958091A90780938D088091E0
:10AF500061078093CE08809163078093EA07809110
:10AF6000F1078093F0071092F107089580936F0224
:10AF700080936E0260937102409370021092BB0541
:10AF800081E08093FA05089580E008958091FE05A0
:10AF9000882309F05EC08091B805882309F069C054
:10AFA00020912706A22FB0E08091B605FD01ED5F4C
:10AFB000F94F80838093120650912806E52FF0E028
:10AFC000E55FF94F808340912906E42FF0E0ED5EC4
:10AFD000F94F8083FD01E170F070ED5EF94F8683DB
:10AFE00030912A06E32FF0E0E55EF94F80839091DF
:10AFF0002B06E92FF0E0E55EF94F8583A370B07072
:10B00000AD5DB94F8C932F5F277020932706852F56
:10B010008F5F80932806873010F010922806842FC7
:10B020008F5F80932906863010F010922906832FB7
:10B030008F5F80932A06853010F010922A06892FA0
:10B040008F5F80932B06833018F010922B060895A3
:10B0500008958091B805882309F4A2CF209127068E
:10B06000509128064091290630912A0690912B068E
:10B07000CACF6091B7056830D1F120912706A22F81
:10B08000B0E08091B605FD01ED5FF94F808361303E
:10B0900009F454C080931206673009F070C04091E3
:10B0A0002906E42FF0E0ED5EF94F8083A170B070C7
:10B0B000AD5EB94F16968C9330912A06E32FF0E0DF
:10B0C000E55EF94F80835091280690912B06E92F79
:10B0D000F0E0E55EF94F8583643009F494CFE22F08
:10B0E000F0E0E370F070ED5DF94F80838CCF8091DC
:10B0F000B6058093120650912806E52FF0E0E55F33
:10B10000F94F808340912906E42FF0E0ED5EF94F7E
:10B11000808320912706E22FF0E0E170F070ED5E71
:10B12000F94F86836530F1F490912B06E92FF0E01A
:10B13000E55EF94F858330912A06D1CF50912806DC
:10B14000E52FF0E0E55FF94F808340912906E42F79
:10B15000F0E0ED5EF94F8083A170B070AD5EB94F45
:10B1600016968C9330912A06E32FF0E0E55EF94FB6
:10B170008083633009F0A9CF90912B06B0CF509116
:10B180002806E52FF0E0E55FF94F80836630B9F4DB
:10B19000A170B070AD5EB94F16968C9330912A06AF
:10B1A000E32FF0E0E55EF94F808390912B06E92FC5
:10B1B000F0E0E55EF94F85834091290690CF4091FC
:10B1C0002906E42FF0E0ED5EF94F8083623009F04C
:10B1D000A2CF30912A06E32FF0E0E55EF94F80839D
:10B1E00090912B06E92FF0E0E55EF94F858377CF4C
:10B1F000FC0187858F708D30C1F030E020E190E058
:10B2000080818F708E3061F09F5F31969217C0F30E
:10B21000892F913118F48150832B089580E1FBCF61
:10B220009923B1F780E0832B089530E12FE0E7CF39
:10B23000E82FF0E0EF73F070E75AFA4F808108953D
:10B24000409365076093A8078093740881E080931A
:10B25000ED070895882339F08091A807809374083A
:10B2600081E08093ED0708958093740881E08093D6
:10B27000ED0708958091ED07882319F01092ED07EE
:10B2800081E008952F923F924F925F926F927F924A
:10B290008F929F92AF92BF92CF92DF92EF92FF92E6
:10B2A0000F931F93CF93DF935C01562E3A016901F0
:10B2B000662309F45DC0482EEC0130E060E0EE2426
:10B2C000FF24FA9480E000E010E05FE04EE0342ECE
:10B2D0002DE0222E98E7892E98E0992E800E911E5F
:10B2E000F40170817F707F5FDE0190E0442D419515
:10B2F0000BC05C93223089F0E42EEA0E3F5F9F5F23
:10B300001196822F9717D0F4F601E30FF11D2081DB
:10B31000213079F7882349F45C93F301E60FF11D9E
:10B32000F0806F5FFC9222E0E7CF5C93F501EE0DB9
:10B33000F11D808180648083FC92DECF903158F4CF
:10B34000FE01E90FF11D30829F5F05C0FE01E90F8C
:10B35000F11D50839F5F9031C8F3F401808184FD1B
:10B360002F860F5F1F4F6096822F051508F4B2CF0E
:10B37000DF91CF911F910F91FF90EF90DF90CF90D1
:10B38000BF90AF909F908F907F906F905F904F9005
:10B390003F902F900895809165070E94881F882311
:10B3A00039F08091A8078093740881E08093ED07BD
:10B3B00008951092530784E20E941B241092F00516
:10B3C00080E00E941B240E94E7240E948F280E9494
:10B3D000F2278091A1060E94422780E00E94124439
:10B3E000089581E08093530784E20E9485230E94A0
:10B3F000F22780E00E94422780E00E9412440895D4
:10B400001092EF070E948F280E94F2270E94E724E3
:10B410008091A1060E9442271092EB0781E20E94D0
:10B420001B2480E00E9412441092DB088CEF0E94E3
:10B43000261808951092640781E08093EB0781E25B
:10B440000E94852380E00E94124480919C058823FD
:10B4500021F480919D0580FDFCCF10929D051092F6
:10B46000D005109248068091480680934A0681E0F4
:10B470008093EF078093DB088AEF0E9426180895D7
:10B4800080913306882329F081E00E94721F88236F
:10B4900061F41092BE0580E00E945C1F882321F0B9
:10B4A00081E08093BE0580E0089581E080933406BA
:10B4B00080E00E945C1F882319F082E080933406AC
:10B4C00081E0089582E00E94721F882329F08FE0B6
:10B4D0000E945C1F882361F482E00E945C1F882325
:10B4E00029F481E08093B30580E0089580E0089519
:10B4F00082E08093B30581E0089580919C058230BD
:10B5000011F080E008950E94C0188093D00880E078
:10B51000089590916D029093B7058091B90580933D
:10B52000B805882321F08091FF058823A9F0809138
:10B53000BB058330B1F1882341F48091B80588239D
:10B5400029F460E084E00E94D723089580912706C3
:10B5500080FFF7CF63E0F6CF983009F440C0913018
:10B5600009F444C0973009F046C0E0912806F0E0A5
:10B57000E55FF94FE08180910206882331F08091E8
:10B58000B5058E27807FEF70E82B80910106882318
:10B5900011F080EFE827E093B5058091BB0583307B
:10B5A00051F60E9407299091B7059150983060F4A8
:10B5B0008091B805882341F08091FF058823C9F464
:10B5C00061E0892F0E94E32560E08091FF058111F1
:10B5D00061E082E00E94D7238091BB05ACCFE0916F
:10B5E0002706F0E0ED5FF94FE081C5CFE09112064C
:10B5F000C2CF63E0E6CF963039F4E0912906F0E05F
:10B60000ED5EF94FE081B7CFE0E0923049F4E09190
:10B610002706F0E0E170F070ED5EF94FE681ABCF08
:10B62000953039F4E0912A06F0E0E55EF94FE081CB
:10B63000A2CF933039F4E0912B06F0E0E55EF94FAC
:10B64000E58199CF943009F096CFE0912706F0E09C
:10B65000E370F070ED5DF94FE0818DCFCF93DF9314
:10B66000EB0190E082959295907F9827807F9827B4
:10B6700060E1AE010E949045FE0120E091E004C02F
:10B680009F5F3196913159F02223D1F780818F70DD
:10B690008E30B1F7292F9F5F31969131A9F7222380
:10B6A00059F490E18F858F708D3071F0892F815022
:10B6B0008F70DF91CF910895922F915099F791E07B
:10B6C0008F858F708D3091F7903120F08EE1DF9172
:10B6D000CF910895892F81508F708061DF91CF9134
:10B6E00008950F931F9390E0880F991F860F911D67
:10B6F000880F991F880F991F880F991F840F911D1C
:10B7000030E022953295307F3227207F3227829594
:10B710009295907F9827807F9827622FA8010E949A
:10B7200090451092F7051F910F910895EF92FF92A7
:10B730000F931F93CF93DF93182F062F0E94A724F8
:10B74000E12EFF24EE0CFF1CEE0CFF1CEE0CFF1C88
:10B75000E00EF11CE294F294A0EFFA22FE24EA2219
:10B76000FE24C0E0D0E0FE01E358F74F8081BE0127
:10B770006E0D7F1D0E9416452196C031D10599F7A7
:10B780000E94A724DF91CF911F910F91FF90EF901E
:10B790000895CF92DF92EF92FF920F931F93CF9372
:10B7A000DF93E22E6801082F10E0000F111F060F33
:10B7B000111D000F111F000F111F000F111F040F8B
:10B7C000111D02951295107F1027007F1027FF246E
:10B7D000E294F29480EFF822FE24E822FE24FE2C6C
:10B7E00082E00E9485230E94A724EE2099F0C0E009
:10B7F000D0E0F601EC0FFD1F8081B8016C0F7D1FBA
:10B800000E94164582E00E9478160E945F0E2196E3
:10B81000CF1578F382E00E941B240E94A724109287
:10B82000F705DF91CF911F910F91FF90EF90DF907F
:10B83000CF900895EF92FF920F931F93CF93DF93D2
:10B84000182F062F0E94A724E12EFF24EE0CFF1CC8
:10B85000EE0CFF1CEE0CFF1CE00EF11CE294F294C7
:10B8600040EFF422FE24E422FE24C0E0D0E0CE012A
:10B870008E0D9F1D0E945A45FE01E358F74F8083AD
:10B880002196C031D10599F71092F00580E00E9411
:10B8900038240E94A724DF91CF911F910F91FF9030
:10B8A000EF90089580919C05882369F40E946E01B1
:10B8B00080919C05813069F00E94071F80919C0552
:10B8C000823069F008950E946F0180919C0581305B
:10B8D00099F70E940E1F80919C05823099F781E0B4
:10B8E0008093960208958091F305823008F00895C0
:10B8F0009091CE0880916107981709F448C0809113
:10B9000061078093CE0891E08091F107882359F573
:10B91000992369F380918D082091CE083091EA0730
:10B920006091F00790E0880F991F820F911D880F9A
:10B93000991F880F991F880F991F830F911D70E021
:10B9400062957295707F7627607F762782959295B3
:10B95000907F9827807F982744E358E00E94904585
:10B960001092F70508958091A90780938D08809122
:10B9700061078093CE08809163078093EA078091E6
:10B98000F1078093F0071092F1079160C1CF90E02A
:10B99000BBCF4F925F926F927F928F929F92AF92A6
:10B9A000BF92CF92DF92EF92FF920F931F93CF93AC
:10B9B000DF93562E4A015901662309F4E0C09C0129
:10B9C000E90100E010E0AFEFEE246624772422E0E6
:10B9D000C22E442443948F858F708D3009F4CCC0DF
:10B9E00030E020E1FE0190E080818F708E3009F41C
:10B9F000BEC09F5F31969217B8F3892F913108F03E
:10BA000080E18150832BF301E858F74F8083D08089
:10BA10008FE0D822D39440E050E012C0A627AF7B3D
:10BA2000F1F4F501E00FF11D4082112309F06FC020
:10BA3000EE24E3940F5F4F5F5F4FA62F4D1588F5FF
:10BA4000742FFE01E40FF51F6081262F30E0C9013D
:10BA50008F7090700F9709F454C0EE20F9F6F5013D
:10BA6000E00FF11DC082E12FF0E0D401AE0FBF1F47
:10BA70006C937295707FEE50F84F70831F5F0024B7
:10BA8000220F331F001C220F331F001C232F302DC9
:10BA9000EE24E394E2220F5F4F5F5F4FA62F4D1518
:10BAA00078F20894611C711C6096651408F493CFB9
:10BAB000003408F068C0912FF501E00FF11D1082ED
:10BAC0000F5F0034C8F3812F192F103448F49FEF13
:10BAD000E12FF0E0EE50F84F90831F5F1034C0F379
:10BAE000DF91CF911F910F91FF90EF90DF90CF905A
:10BAF000BF90AF909F908F907F906F905F904F908E
:10BB00000895F501E00FF11D1082EE2493CFE12F8F
:10BB1000F0E03197E80DF91D60831150A12FB0E0DE
:10BB20001F5FAE50B84F7C917F70F72EF3948C91CD
:10BB300082958F70E82FF0E0CF018F0D911D409717
:10BB40000CF0F72E0024220F331F001C220F331F8E
:10BB5000001C232F302DEE24E394E222E295F2958F
:10BB6000F07FFE27E07FFE27FE2AFC9263CF992319
:10BB700009F043CF80E046CF30E12FE033CF00E043
:10BB800010E090E099CF812FA0CFDF93CF930F9259
:10BB9000CDB7DEB7FC0187858F708D3079F130E04D
:10BBA00020E190E080818F708E30E9F09F5F3196C8
:10BBB0009217C0F3892F9131A0F48150832B898390
:10BBC00089818F708F5F80935805609367078981A3
:10BBD00084FD0DC08CE0809357050F90CF91DF91CD
:10BBE000089580E1EACF992329F780E0E7CF80E14B
:10BBF000809357050F90CF91DF91089530E12FE0AA
:10BC0000D0CF1F93DF93CF930F92CDB7DEB715B18F
:10BC100080E00E94124480919D068C3041F0109289
:10BC2000320884E398E09093760880937508109228
:10BC30009D05109235061092B2051092480680912B
:10BC4000480680934A0610926207E0917508F091C9
:10BC500076084091EA0787858F708D3009F443C0DC
:10BC600030E020E190E080818F708E30B1F19F5FF5
:10BC700031969217C0F3892F913168F58150832B4B
:10BC8000898389818F708F5F809358054093670700
:10BC9000898184FD26C08CE08093570583E08093E2
:10BCA000DB0880919C05813011F00E94151F8AEFFE
:10BCB0000E94261883E08093A4051092A905109293
:10BCC000AA0515FF03C081E00E9478160F90CF915E
:10BCD000DF911F91089580E1D1CF992361F680E033
:10BCE000CECF80E1D9CF30E12FE0BCCFDF93CF932F
:10BCF0000F92CDB7DEB78091F305823070F080915E
:10BD000077088D3010F01092770880917708809333
:10BD10007C080F90CF91DF9108959091CE0880918B
:10BD20006107981709F47EC0809161078093CE085F
:10BD300091E08091F107882309F057C09923F9F227
:10BD400080918D082091CE083091EA076091F0072C
:10BD500090E0880F991F820F911D880F991F880FFF
:10BD6000991F880F991F830F911D70E0629572953E
:10BD7000707F7627607F762782959295907F9827AF
:10BD8000807F982744E358E00E9490451092F70581
:10BD9000E0917508F09176084091EA0787858F70E9
:10BDA0008D30E9F130E020E190E080818F708E30BD
:10BDB00081F19F5F31969217C0F3892F913108F07E
:10BDC00080E18150832B898389818F708F5F80937D
:10BDD000580540936707898184FD1FC08CE08093DC
:10BDE000570581E08093FA058ACF8091A907809357
:10BDF0008D08809161078093CE08809163078093BE
:10BE0000EA078091F1078093F0071092F1079160A3
:10BE100095CF992391F680E0D5CF80E1E0CF30E156
:10BE20002FE0C2CF90E085CF4F925F926F927F92CA
:10BE30008F929F92AF92BF92CF92DF92EF92FF923A
:10BE40000F931F93CF93DF931092560581E0809359
:10BE500074088093ED07FF24C0E0D0E0CC24EE24EA
:10BE6000E394BB24BA9472E0D72E64E0A62E53E08C
:10BE7000952E44E1842E30E2732E22E1622E90E171
:10BE8000592E81E1482E0E9445220E945F0E80912A
:10BE90007408873009F4EAC0883008F088C084301C
:10BEA00009F434C3863009F464C2813061F78091AB
:10BEB000ED07882331F01092ED070E9492240E9432
:10BEC000A72487E10E94B11F882361F08091740844
:10BED00097E1909365078093A80787E080937408A3
:10BEE000E092ED0788E00E94B11F882361F0809105
:10BEF000740898E0909365078093A80786E0809384
:10BF00007408E092ED0781E00E94B11F882351F090
:10BF100080917408E09265078093A807A092740846
:10BF2000E092ED078EE00E94B11F882361F08091BE
:10BF300074089EE0909365078093A8078FE0809334
:10BF40007408E092ED0782E00E94B11F882351F04F
:10BF500080917408D09265078093A8075092740866
:10BF6000E092ED078FE00E945C1F882309F0E1C397
:10BF70009091970680919D06891709F484CF80914E
:10BF8000970680939D0681E080935605DF91CF91BF
:10BF90001F910F91FF90EF90DF90CF90BF90AF90E7
:10BFA0009F908F907F906F905F904F900895803119
:10BFB00009F41DC2813108F0EDC08F3009F063CF64
:10BFC0008091ED07882349F01092ED07E092F60585
:10BFD000809198068093F505FF24809165070E9463
:10BFE000881F882349F08091A80780937408E09205
:10BFF000ED07FF2009F02DC40E947020882371F006
:10C00000982F9150943050F480915C06981731F03D
:10C0100090935C06E092F605FF24F39480915C0611
:10C02000813009F4FEC28091F605882309F42BCFF4
:10C030001092F6050E9407290E94F22780915C0663
:10C040008F5F0E94AB2780915C06813009F01BCF87
:10C0500080915F0681500E9442270E9445220E94E3
:10C060005F0E80917408873009F016CF8091ED073C
:10C07000882361F01092ED07E092F60580E00E94BF
:10C080008523809198068093F505FF2480916507AC
:10C090000E94881F882349F08091A8078093740824
:10C0A000E092ED07FF2009F0E6C30E94702088238C
:10C0B00001F1982F91509330E0F480919C059817EE
:10C0C000C1F090939C05992309F426C40E946F0146
:10C0D00080919C05813009F426C40E94071F80913D
:10C0E0009C05823011F4E0929602E092F605FF245E
:10C0F000F39483E00E94721F882371F08091F90508
:10C100008F5F8093F9058091F90581708093F9051F
:10C11000E092F605FF24F394909198068091F5053E
:10C12000981781F0809198068093F5058091F50528
:10C13000853040F48091F5058093B405E092F605D2
:10C14000FF24F39486E10E94721F882309F041C204
:10C150008091F605882309F496CE1092F6050E9488
:10C16000072980919C058F5F0E94AB2783E20E9484
:10C170001B248091F905882309F4B2C30E94F22799
:10C1800080919C05823009F0F1C08091B4050E9435
:10C190004227ECC0813109F47FC0823109F073CEAF
:10C1A0008091ED07882349F01092ED07E092F605A3
:10C1B0001092F4051092C405FF24809165070E9437
:10C1C000881F882379F08091A80780937408E092F3
:10C1D000ED07FF2009F010C38BE10E941B248CE1C6
:10C1E0000E941B2489E00E94721F882321F0109274
:10C1F000F405E092F6058AE00E94721F882321F080
:10C20000E092F405E092F6058091F4058823B9F4F4
:10C210008091C405882399F09091C40580916B02A8
:10C22000980F97FDC4C39B300CF45EC38AE08093E3
:10C230006B02E092F6051092C405FF24F3948091FE
:10C24000F405813009F4D4C18091F605882309F4FE
:10C250001ACE8091F405882309F07DC28BE10E94FB
:10C2600085238CE10E941B2410916B021B5F09F453
:10C27000D2C300E0802F0E94112B0F5F0117D0F373
:10C28000103138F4012F802F0E9442270F5F0031B8
:10C29000D0F31092F605F7CD8091ED078823C1F019
:10C2A0001092ED07E092F605B092F40580915206E7
:10C2B000813009F406C3823009F400C3843009F4E4
:10C2C000FAC2883009F4F4C282E00E948523FF2478
:10C2D000809165070E94881F882349F08091A807F4
:10C2E00080937408E092ED07FF2009F098C20E9445
:10C2F0007020882341F1982F9150943020F580913F
:10C30000F405981701F19093F405E092F6058091F9
:10C31000F405882309F4EBC242E08091F4058230F1
:10C3200009F4EBC28091F405833009F4ECC2242FA8
:10C3300030E0C901880F991F820F931F880F8093E7
:10C340005906409352068091F605882309F49BCD47
:10C350001092F6050E9407298091F405843008F0B8
:10C3600031C28091F4058F5F0E94AB270E94A72401
:10C370008ACD8091ED07882339F01092ED07109255
:10C38000F6051092F405FF24809165070E94881F2E
:10C39000882349F08091A80780937408E092ED0704
:10C3A000FF2009F01CC28091F405882309F456C1CE
:10C3B0002091F405213009F46DC12091F40522305B
:10C3C00009F48AC18091F605813009F4A7C18091F2
:10C3D000F605823009F057CD1092F6050E94F2273B
:10C3E000809162060E9442270E94A7244CCD809132
:10C3F000ED07882349F01092ED07E092F605E092F0
:10C40000F405FF24C0E0D0E0809165070E94881FFA
:10C410008823A1F08091A80780937408E092ED072B
:10C42000FF2051F08091F405813009F49EC2809183
:10C43000F405823009F47AC21092A60580E00E94C9
:10C44000721F882361F08091F405823041F0D09210
:10C45000F40582E20E94A123E092F605FF240E94E7
:10C460002A20282F882391F0CE01880F991F880F4A
:10C47000991F880F991FCC0FDD1FC80FD91F21509E
:10C48000C20FD11DD092F605FF24F3940091F4055C
:10C49000023009F47CC18091F605882309F4F3CCBD
:10C4A0008091F405813009F4C4C18091F405823093
:10C4B00009F0E9CC8091F605823009F42BC28DE0B9
:10C4C00090E00E944903282F992787FD909597FDBA
:10C4D000A4C2082F27FD9CC2CC24C3948BE10E94E8
:10C4E0001B248CE10E941B24002339F0C7FC99C255
:10C4F0001C141CF48CE10E948523802F90E00E9484
:10C50000EB02E092A6051092F605BDCC8091ED07F6
:10C51000882339F01092ED07E092F6051092F405A9
:10C52000FF24809165070E94881F882331F1809144
:10C53000A80780937408E092ED07FF20E1F0809156
:10C54000F405882311F4E092F4058091F40581321A
:10C5500010F07092F405909100028091F405981704
:10C5600051F08091F405809300026091000287E011
:10C5700090E00E9450031092A6050E942A20382FB6
:10C58000882391F08091F4052AE0829FC001112454
:10C590008093F4058091F4058150830F8093F40516
:10C5A000D092F605FF24F3948091F605882309F4D0
:10C5B0006ACC909100028091F605823009F4FFC0A8
:10C5C000892F90E00E94EB02E092A6051092F605FA
:10C5D0005ACC9091A80787E1809365079093A807AC
:10C5E00040927408E092ED0780E00E941B24B0CDD9
:10C5F0008091C405882309F427CE9091C4058091C9
:10C600006C02980F9A300CF481C195310CF0D8C1AE
:10C6100090936C02E092F6051092C405FF24F39407
:10C6200013CE9091F50580919806981709F4FBCCEC
:10C63000809198068093F5059091F5059F5F923063
:10C6400008F4B8C180915F06981709F4ECCC909378
:10C650005F06E092F605FF24F394E5CC8AE00E94A1
:10C66000721F882309F030C189E00E94721F88235D
:10C6700009F49ECE8BE10E948523D092F405D092DE
:10C68000F605809198068093F5052091F4052130F8
:10C6900009F093CE909198068091F505981761F076
:10C6A000809198068093F5052093F6058091F50515
:10C6B00080937506FF24F3948AE00E94881F8823E4
:10C6C00009F47BCE1092F4058CE10E941B2420918A
:10C6D000F405223009F076CE909198068091F50508
:10C6E000981761F0809198068093F5052093F605E0
:10C6F0008091F50580936206FF24F39489E00E94FF
:10C70000881F882309F45ECE1092F4058BE10E9405
:10C710001B248091F605813009F059CE1092F60560
:10C720000E94F227809175060E9442270E94A7244A
:10C73000AACB82E00E94721F882309F419CC909141
:10C7400074088FE0809365079093A807609274083F
:10C75000E092ED070DCC8BE10E941B248CE10E943E
:10C76000852310916C021A5000E0802F0E9442270E
:10C770000F5F1017D0F7003108F08BCD802F0E948B
:10C78000112B0F5F0031D0F31092F6057CCB89E0BE
:10C790000E94721F882331F01C1424F40093F605C4
:10C7A000CC24CA948AE00E94721F882309F473CEB5
:10C7B000C7FE71CED092F605CC24C3946CCE909176
:10C7C000F405FECE85E00E94AB2786E00E94AB27F1
:10C7D00087E00E94AB2788E00E94AB27C7CD83E0AB
:10C7E00090E0609175060E94500384E090E06091B3
:10C7F00062060E945003D7CD80916C0290E00A97A8
:10C8000082959295907F9827807F982760916B0200
:10C810006F70682B81E190E00E945003DDCC8EE0C8
:10C8200090E0609152060E94500382E00E941B2417
:10C830005ECD8091F605823009F4BEC080913E063F
:10C8400090913F060E94EB02E092A6051092F60539
:10C850002CCE80915F0660915C0690E001978295F6
:10C860009295907F9827807F9827682B8AE090E0A8
:10C870000E945003C1CB8091F90590E081709070C7
:10C8800082959295907F9827807F982760919C054C
:10C890006F70682B82E090E00E9450036091B405B5
:10C8A0008FE090E00E94500380E00E941B24FDCBAB
:10C8B0009092F40509CDD092F40506CDE092F405EE
:10C8C00003CD1092F40500CD8CE10E948523E09207
:10C8D000F405E092F605809198068093F505C4CEA4
:10C8E00083E20E9485234ACC90936B02A2CC41E064
:10C8F0008091F405823009F015CD44E08091F40573
:10C90000833009F014CD48E080E319CD8AE08093AC
:10C910006C0280CE0C2FE2CD0E946E0180919C05AE
:10C92000813009F0DACB0E940E1FD9CBC7FC6EC054
:10C9300081E0C536D10508F44DC0C0E0D0E0CC247C
:10C9400060E87DE88BE590E000E0F89460930902F0
:10C9500070930A0280930B0290930C028DE090E09A
:10C96000602F0E945003789467CDC431D10558F5EB
:10C97000C4E1D0E0F89480913E0690913F068C1778
:10C980009D0799F0CE010E94700180913E06909122
:10C990003F06909358068093570660913E0670912B
:10C9A0003F0685E090E00E94E20D789440CD109221
:10C9B0006B023FCC92E046CECE010E94EB0244CF08
:10C9C00080926C0227CE81E0CD32D80798F2CCE27B
:10C9D000D1E0D0CF992787FD90958C9F80018D9FC6
:10C9E000100D9C9F100D1124C02E602F772767FD1E
:10C9F0007095872F972F20E737E140E050E00E94A5
:10CA00001C8760587247844A9F4F9FCF8FEF91CF0A
:10CA1000CC24CA9463CD00E036CC909581959F4F8D
:10CA200058CD8BE10E94852363CDDF93CF930F9286
:10CA3000CDB7DEB71092DB0880E00E9412448CEF85
:10CA40000E94261880919C05813011F00E94DD1E05
:10CA500080919D068C3091F11092320884E398E029
:10CA60009093760880937508109248068091480646
:10CA700080934A06109262078091F3058230D8F1C4
:10CA8000809177088D3010F01092770880917708A8
:10CA900080937C088091AA058823E1F48091A90500
:10CAA000882311F58091B805882321F01092B905EB
:10CAB0001092B8050F90CF91DF910895109248061B
:10CAC0008091480680934A06109262078091AA05D9
:10CAD000882321F38091AA050E9400181092AA05CC
:10CAE0008091A9058823F1F28091A9050E94001880
:10CAF0001092A905D7CF9091CE0880916107981721
:10CB000009F483C0809161078093CE0891E0809101
:10CB1000F107882399F08091A90780938D0880916F
:10CB200061078093CE08809163078093EA07809124
:10CB3000F1078093F0071092F1079160992309F4AF
:10CB40009FCF80918D082091CE083091EA076091A7
:10CB5000F00790E0880F991F820F911D880F991F91
:10CB6000880F991F880F991F830F911D70E06295A0
:10CB70007295707F7627607F762782959295907F59
:10CB80009827807F982744E358E00E9490451092B0
:10CB9000F705E0917508F09176084091EA078785DE
:10CBA0008F708D3079F130E020E190E080818F70DE
:10CBB0008E3001F19F5F31969217C0F3892F91312A
:10CBC000F8F48150832B898389818F708F5F8093E4
:10CBD000580540936707898184FD10C08CE08093DD
:10CBE000570581E08093FA05809177088D3008F031
:10CBF0004BCF4CCF992311F780E0E4CF80E1EFCF0A
:10CC000080E1DFCF30E12FE0D0CF90E080CFEF9216
:10CC10000F931F93DF93CF930F920F92CDB7DEB791
:10CC20008091BB05882309F45DC01A8210E0813031
:10CC300009F4B7C0823069F18091DB08882319F4C8
:10CC4000112309F070C08A81813021F08091FA05AA
:10CC5000882321F080916E02882351F48091BB05D6
:10CC60000F900F90CF91DF911F910F91EF9008954A
:10CC70008091EA076091F007409163072091F107E6
:10CC80000091EA07E09061070E945B2B1092FA0581
:10CC9000E5CF80917002823009F4F2C08A8182303F
:10CCA00009F404C188E00E94881F882351F488E0B9
:10CCB0000E945C1F882329F080917002882309F06C
:10CCC000BBCF1092BB0582E20E94852384E20E94C2
:10CCD0001B240E949B2980916F0280936E0281E049
:10CCE0008A83AACF88E00E945C1F882339F4809150
:10CCF0007102882341F58091BB0597CF8091700226
:10CD00008823A9F382E08093BB0582E20E941B2462
:10CD100084E20E94852310926E0282E08A8310E0F2
:10CD20008091BB0584CF8091F305823008F4CCC09C
:10CD3000809177088D3010F01092770880917708F5
:10CD400080937C0880CF84E10E945C1F882309F0D7
:10CD5000B5C01A8210E085E10E945C1F882329F08B
:10CD600081E0809361078A8311E00E94702088230C
:10CD700019F48091BB055BCF21E02093BB05982F70
:10CD800091509093BC059093BD058091A20680932D
:10CD9000A907909363072093F107109277082A83DD
:10CDA00011E084E10E94721F882329F0109261072C
:10CDB00081E08A8311E085E10E94721F882329F0B7
:10CDC00081E0809361078A8311E000E08091BC05D7
:10CDD000081709F18091BD050817E9F0802F0E941E
:10CDE0002B228823C1F08091BD05982F901B191626
:10CDF0009CF5943084F48093BC050093BD0580912C
:10CE0000A2068093A9079F5F9093F10700936307A1
:10CE100081E08A8311E00F5F0830C1F68091BC0584
:10CE20006091BD050E942C23882399F480917102A2
:10CE3000882379F088E00E945C1F882339F0809174
:10CE40007002882319F01092BB05F6CE8091BB05C5
:10CE5000F1CE1092BB05EECF9923E9F29195943073
:10CE6000D4F68093BC050093BD058091A206809303
:10CE7000A9079F5F9093F10781E08A8311E0CBCFF0
:10CE80000E946321882309F409CF982F9150809143
:10CE90007708981709F402CF909377088091DB0800
:10CEA000882321F48091770880937C080E949B2935
:10CEB000809177080E9465271A82F4CE109261074C
:10CEC00081E08A8311E047CF9091CE08809161077D
:10CED000981709F47DC0809161078093CE0891E096
:10CEE0008091F107882399F08091A90780938D089C
:10CEF000809161078093CE08809163078093EA0751
:10CF00008091F1078093F0071092F10791609923C7
:10CF100009F40ECF80918D082091CE083091EA0758
:10CF20006091F00790E0880F991F820F911D880F84
:10CF3000991F880F991F880F991F830F911D70E00B
:10CF400062957295707F7627607F7627829592959D
:10CF5000907F9827807F982744E358E00E9490456F
:10CF60001092F705E0917508F09176084091EA0774
:10CF700087858F708D3049F130E020E190E080812D
:10CF80008F708E30E1F09F5F31969217C0F3892F3A
:10CF9000913108F080E18150832B898389818F70E2
:10CFA0008F5F8093580540936707898184FD0BC08C
:10CFB0008CE08093570581E08093FA05B9CE9923E0
:10CFC00031F780E0E9CF80E1F4CF30E12FE0D6CF38
:10CFD00090E086CF2F923F924F925F926F927F9216
:10CFE0008F929F92AF92BF92CF92DF92EF92FF9279
:10CFF0000F931F93DF93CF9300D00F920F92CDB773
:10D00000DEB70E9445228091DB08882311F40C943E
:10D01000017084E08093740881E08093ED071C82A6
:10D02000662455241B821A823324339484E398E0C7
:10D030008D83F2E02F2EEFE07E2E0E9445220E948B
:10D040005F0E10917408173009F476C3183008F099
:10D05000ACC0143009F47DC7153008F0FFC01130A2
:10D06000A1F111E080919C05823009F499C0809172
:10D070003306882339F081E00E94721F882311F063
:10D080000C9425731092BE0580E00E945C1F8823DB
:10D0900011F03092BE05112381F60F900F900F9082
:10D0A0000F900F90CF91DF911F910F91FF90EF9014
:10D0B000DF90CF90BF90AF909F908F907F906F90B8
:10D0C0005F904F903F902F9008958091ED078823B7
:10D0D00011F00C94F5700E94076680E00E94721FA8
:10D0E000882329F085E0809374083092ED0783E06F
:10D0F0000E94721F882361F08091740893E09093DE
:10D1000065078093A80788E0809374083092ED0744
:10D1100088E00E94B11F882329F086E0809374087C
:10D120003092ED0787E10E94B11F882329F0F7E0D4
:10D13000F09374083092ED078BE00E94B11F8823B2
:10D1400059F0909174088BE0809365079093A8073D
:10D15000809374083092ED078DE00E94B11F882300
:10D1600011F00C943D7280917408813011F010928E
:10D1700033068091DB08882311F00C944B72909158
:10D18000970680919D06891709F46BCF80919706C9
:10D1900080939D0610E080919C05823009F067CF56
:10D1A0000E94C0188093D00862CF1A3009F460C67C
:10D1B0001B3008F0B4C1183009F410C6193009F05A
:10D1C00050CF8091ED07882311F00C942971809144
:10D1D000DB08882311F40C943F719091F405809141
:10D1E00066079817D9F06090F405809166078093E0
:10D1F000F4058091F605833011F40C940379809145
:10D20000F605823058F080916007882339F4E09168
:10D21000F405F0E0E859F84F81E0808386E10E9450
:10D22000721F882309F0F3C68091F605833009F454
:10D230002AC786E10E94881F882309F412CF8091B3
:10D24000F605823009F00DCF3092F60580E00E949D
:10D25000124482E00E941B2411E004CF153009F42F
:10D2600084C4163009F0FDCE8091ED07882309F4BF
:10D27000A9C01092ED070E9492246090F0076620EA
:10D2800011F40C94117900E0FF247FEFA0E08824D2
:10D290009924AA24BB2424E3C22E28E0D22ECA0C4F
:10D2A000DB1CF501ED5BF74F80818F708D3011F441
:10D2B0000C94F37330E020E1F60190E080818F70F0
:10D2C0008E3011F40C941E739F5F31969217B0F359
:10D2D000892F913108F080E18150832BF401E858C7
:10D2E000F74F8083E080EFE0EE22E39440E050E0EF
:10D2F00014C071277F7B09F5EF2DF0E0E859F84F56
:10D3000081E08083002311F00C94B472A1E0F394C7
:10D310004F5F5F4F4E1590F5712F642FF601E40FAC
:10D32000F51F1081212F30E0C9018F7090700F9789
:10D3300011F40C946772AA23E1F6EF2DF0E0E8599E
:10D34000F84F2082E02FF0E0DF01A257B74F1C9387
:10D350006295607FEE50F84F60830F5F0024220FCC
:10D36000331F001C220F331F001C232F302DA22F30
:10D37000A170F3944F5F5F4F4E1570F20894811CBB
:10D38000911CE0E1F0E0AE0EBF1E861410F00C948C
:10D390000977712F80CFE02FF0E0EE50F84F9FEF2C
:10D3A00090830F5F0034B8F384E20E9485231092CB
:10D3B000F6051092F50583E68093F4051C82662439
:10D3C00055241A8280E00E94B11F882311F0E1E009
:10D3D000EC8388E00E94B11F882309F0CFC68091BA
:10D3E000F405833609F4D1C68091F405813011F437
:10D3F0000C94BD778091F405833011F40C9446773A
:10D400008091F405882311F40C9451748091F605F1
:10D4100090E083709070892B11F00C9420748C81B3
:10D42000882309F41ECE4090F007442009F466C01A
:10D43000AD8040E0FF24BB24EE24EA9460E0CC24DD
:10D44000DD2400E010E098012C5C374F58E7852E72
:10D4500058E0952E8C0C9D1CF40150815F705F5F2D
:10D46000D90190E0702F7A190BC07C92E230A1F0C4
:10D470006E2FB72EBA0E4F5F9F5F11969517D8F497
:10D48000E42FF0E0E859F84FE081E13071F76623CE
:10D4900011F00C946F727C92EF2DF0E0E257F74F91
:10D4A000E080F394EC9262E0B72EBA0E4F5F9F5F7C
:10D4B0001196951728F3903160F4F901E90FF11DE9
:10D4C0008EE080839F5F05C0F901E90FF11D708236
:10D4D0009F5F9031C8F3F401808184FF05C0F8019B
:10D4E000ED5BF74F8DE080830894C11CD11C005F79
:10D4F0001F4F90E1A90EC41408F4A5CFEA81EE23D2
:10D5000011F00C943276FC81F13011F40C941C76FD
:10D510008C81823011F40C9413761A82A2CD1B30C8
:10D52000B1F11C3009F09DCD8091ED07882391F079
:10D530001092ED079091F1058091F007981711F482
:10D540000C946E783092F6058091A8078093740849
:10D550003092ED07809165070E94881F882309F4A7
:10D5600080CD8091A807809374083092ED07809158
:10D57000F605882311F40C9482788DE00E941B2418
:10D5800082E00E941B240E94A72411E06BCD8091B1
:10D59000ED07882309F015C6809165070E94881F52
:10D5A000882309F442C08091A807809374083092C0
:10D5B000ED078091F605882391F580918D083091D3
:10D5C000CE082091EA0790E0880F991F830F911DE4
:10D5D000880F991F880F991F880F991F280F209374
:10D5E000F2058091F0078093F1058823C1F090E067
:10D5F000A0E0B0E0282F30E022953295307F32272E
:10D60000207F3227FD01EC5CF74F8081A655B84F93
:10D610008C939F5FA92FB0E0A217B3079CF38FE014
:10D620000E941B248DE00E941B248DE00E94721F2B
:10D63000882309F416CD8091F605882309F011CDD1
:10D640008091F105882309F40CCD3092F605809184
:10D650008D082091CE081091EA0790E0880F991F5D
:10D66000820F911D880F991F880F991F880F991F8E
:10D67000180F8091F205181709F4F3CC8DE00E9481
:10D68000852382E00E9485230E94A7246091F205F1
:10D690008091F007882309F442C0C62EDD24C2948D
:10D6A000D294B0EFDB22DC24CB22DC24A12EBB24DD
:10D6B000A294B294A0EFBA22BA24AA22BA24750185
:10D6C00000E010E0C6010E945A45582E0C5C174F2E
:10D6D000F8018083C7010E945A45B6010E94164591
:10D6E000852DB7010E94164582E00E9478160E949F
:10D6F0005F0E0894C11CD11C0894E11CF11C8E2DF6
:10D700008A19082F10E08091F00790E08295929599
:10D71000907F9827807F9827081719079CF26091BF
:10D72000EA0784E398E00E94C55D82E00E941B2422
:10D730000E94A72411E096CC8091ED07882309F47C
:10D74000BCC01092ED070E9492246090F007662002
:10D7500011F40C940E7900E0FF247FEFA0E0882400
:10D760009924AA24BB2424E3C22E28E0D22ECA0C7A
:10D77000DB1CF501ED5BF74F80818F708D3011F46C
:10D780000C94F77330E020E1F60190E080818F7017
:10D790008E3009F44EC79F5F31969217B8F3892FE8
:10D7A000913108F080E18150832BF401E858F74F64
:10D7B0008083E0809FE0E922E39440E050E013C0E2
:10D7C00071277F7BF9F4EF2DF0E0E859F84F81E005
:10D7D0008083002309F0F7C6A1E0F3944F5F5F4F09
:10D7E0004E1588F5712F642FF601E40FF51F108197
:10D7F000212F30E0C9018F7090700F9709F460C637
:10D80000AA23F1F6EF2DF0E0E859F84F2082E02F3F
:10D81000F0E0DF01A257B74F1C936295607FEE5096
:10D82000F84F60830F5F0024220F331F001C220F6C
:10D83000331F001C232F302DA22FA170F3944F5FB4
:10D840005F4F4E1578F20894811C911CE0E1F0E0E6
:10D85000AE0EBF1E861410F00C94F976712F83CF94
:10D86000E02FF0E0EE50F84F9FEF90830F5F003411
:10D87000B8F380E00E9485231092F60589E080933A
:10D88000F4051092F5058091F007882391F020E0CF
:10D89000E22FF0E0E858F74F90818091F5058F5F17
:10D8A0009F70890F8093F5052F5F8091F0072817EF
:10D8B00078F31C8266241B821A8280E00E94B11FCA
:10D8C000882311F0E1E0EC8388E00E94B11F8823F7
:10D8D00011F0F2E0FC8387E10E94B11F882309F078
:10D8E0003BC48091F405893009F43DC48091F4056E
:10D8F000813011F40C9419778091F405882311F488
:10D900000C94F3748091F405882309F4A9C08091E4
:10D91000F405807F09F0A4C08091F405883009F4F3
:10D9200012C184E00E94721F882319F0E2E0E093A4
:10D93000F60584E00E94881F882309F0B7C3809110
:10D94000F60590E083709070892B09F0BAC3FC81D2
:10D95000FF2309F486CB4090F007442009F465C00A
:10D96000AD8040E0FF24BB24EE24EA9460E0CC24A8
:10D97000DD2400E010E098012C5C374F58E7852E3D
:10D9800058E0952E8C0C9D1CF40150815F705F5FF8
:10D99000D90190E0702F7A190BC07C92E23099F097
:10D9A0006E2FB72EBA0E4F5F9F5F11969517D0F46A
:10D9B000E42FF0E0E859F84FE081E13071F7662399
:10D9C00009F099C57C92EF2DF0E0E257F74FE08027
:10D9D000F394EC9262E0B72EBA0E4F5F9F5F119600
:10D9E000951730F3903160F4F901E90FF11D8EE0E5
:10D9F00080839F5F05C0F901E90FF11D70829F5F71
:10DA00009031C8F3F401808184FF05C0F801ED5B1B
:10DA1000F74F8DE080830894C11CD11C005F1F4F1D
:10DA200090E1A90EC41408F4A6CFEA81EE2311F008
:10DA30000C942476FC81F13011F40C941C768C81CA
:10DA4000823011F40C9413769C81933009F065CDEB
:10DA5000E7E0E09374083092ED071A8211E002CB00
:10DA60001091F4058EE00E94721F882351F080917E
:10DA7000F40580618093F40585E08093F605E2E08B
:10DA8000EB838FE00E94721F882351F08091F40590
:10DA900080628093F40585E08093F605F1E0FB83D6
:10DAA00084E10E94721F882349F08091F40580640C
:10DAB0008093F40585E08093F6051B828EE00E943A
:10DAC000881F882341F08091F405807E8093F405BF
:10DAD00084E08093F6058FE00E94881F882341F040
:10DAE0008091F405807D8093F40584E08093F605B1
:10DAF00084E10E94881F882341F08091F405807B97
:10DB00008093F40584E08093F6058091F6058530D6
:10DB100009F4C9C78091F605843009F0FDCE1123C0
:10DB200059F08091F405882339F463948091F505C8
:10DB3000681610F0F1E0FC833092F6058091F40550
:10DB4000883009F0EECEE62DF0E0E859F84F8B81F1
:10DB5000808363948091F505681610F091E09C83B2
:10DB60003092F6051092F405DCCE8091ED07882303
:10DB7000D9F11092ED070E9492243092F60580911F
:10DB800043088F708D3011F40C947E7850E040E1A2
:10DB900020E030E0922FF901EC5CF74F80818F702C
:10DBA0008E3029F09F5F2F5F3F4F241798F3992302
:10DBB00031F0892F913108F080E1815001C080E07F
:10DBC000852B282F2F702F5F2093F40590E09295DE
:10DBD00082958F7089279F70892781708093F505C2
:10DBE000109256051092C4058EE00E94F91F8230F3
:10DBF00009F418C68091C4051816ECF48091F50557
:10DC0000882309F454C49FE023E08091F405891728
:10DC100080F48091F4058F5F8093F4058091C405B2
:10DC200081508093C4052093F6058091C405882314
:10DC300061F71092C4058091C40588230CF4E7C6EF
:10DC40008AE00E94F91F823009F4E2C589E00E944F
:10DC5000F91F823009F4CFC58FE00E94721F88231C
:10DC6000A1F083E08093F6058091F505882319F4EF
:10DC70008CE08093F4058091F5058F5F8093F50526
:10DC80008091F50581708093F5058091F60580FF00
:10DC900022C08091F60581508093F6058091F505AC
:10DCA000882309F4CCC68091F405803108F4B8C704
:10DCB00081E08093F40583E00E9485238091F40540
:10DCC000882309F4CCC68091F4058093F4058091F3
:10DCD000F4050E9444288091F605823008F4CBC6F2
:10DCE00080E00E94881F882309F4BBC98091F60553
:10DCF000823008F437C582E08093F30580914308B1
:10DD00008F708D3011F40C94B07650E040E120E03B
:10DD100030E0922FF901EC5CF74F80818F708E30EC
:10DD200029F09F5F2F5F3F4F241798F3992311F439
:10DD30000C94F676892F913108F080E18150852B83
:10DD400080937808E09078089FE0E922E394A0E0CF
:10DD50006FEF10E020E030E015C060276F7B09F521
:10DD6000F901E859F84F81E08083112311F00C94F8
:10DD7000C776A1E08F2D8F5F2F5F3F4F2E1508F0E4
:10DD8000B5C6602FF22EF901EC5CF74F0081402FF1
:10DD900050E0CA018F7090700F9709F4E5C7AA236D
:10DDA000E1F6F901E859F84F2082E12FF0E0DF01B8
:10DDB000A257B74F0C938F2D8295807FEE50F84F6E
:10DDC00080831F5F0024440F551F001C440F551F04
:10DDD000001C452F502DA42FA170CCCF8091ED07B2
:10DDE000882309F0DDC1809165070E94881F882380
:10DDF00081F18091A807809374083092ED0710920A
:10DE0000F30580918D082091CE083091EA0760914A
:10DE1000F00790E0880F991F820F911D880F991FBE
:10DE2000880F991F880F991F830F911D70E06295CD
:10DE30007295707F7627607F762782959295907F86
:10DE40009827807F982744E358E00E9490451092DD
:10DE5000F7050E947020882309F094C50E94EA20EB
:10DE6000882309F4FEC881500E947A2911E0FAC87B
:10DE70008091ED07882309F45AC01092ED0780E0E5
:10DE80000E9485230E94A72480918D089091CE083E
:10DE90002091EA070091F007E82EFF24EE0CFF1C0A
:10DEA000E90EF11CEE0CFF1CEE0CFF1CEE0CFF1C2F
:10DEB000E20EF11CE294F29410EFF122FE24E12232
:10DEC000FE2410E002951295107F1027007F102786
:10DED000D02E82E00E9485230E94A7240023A1F077
:10DEE00000E010E0F801EC5CF74F8081B701600FB3
:10DEF000711F0E94164582E00E9478160E945F0EF4
:10DF00000F5F1F4F0D1570F382E00E941B240E94CB
:10DF1000A7241092F70580E00E941B240E94A724EA
:10DF200084E0809374083092ED071092F30580919D
:10DF3000F605882339F084E0809374083092ED0769
:10DF40001092F6058091F6058F5F8093F60511E03B
:10DF500089C88091ED07882309F05FC282E00E94A2
:10DF6000721F882309F440C08FE00E945C1F882341
:10DF7000D9F182E08093B30583E00E94B11F88232A
:10DF800009F0B7C180917408843011F01092330603
:10DF90008091DB08882309F485C2809197069091CF
:10DFA0009D069817A1F0809197068D3009F4EEC870
:10DFB00080919706853009F4E9C8809197068330EF
:10DFC00009F4E4C880919706813009F4DFC8809194
:10DFD0003206813009F045C81092320680919706CA
:10DFE000981709F0D3C83DC882E00E945C1F8823BF
:10DFF00019F63092B30583E00E94B11F882311F215
:10E0000078C181E0809374088093ED0708C88091FF
:10E010006007882309F008C992E09093F6050E94F2
:10E02000A921882319F083E08093F605E091F40597
:10E03000F0E0E859F84F2082E091F505F0E0E25772
:10E04000F74F50805092EE07E52DF0E0EF73F0703F
:10E05000E75AFA4F452D4078808160E00E94FB43EB
:10E060008091F405681639F06090F4058091F5050B
:10E070008F5F8093F50582E00E9485238091F605ED
:10E08000833009F0D6C80E94C821882309F4D1C87A
:10E09000E2E0E093F60586E10E945C1F882309F028
:10E0A000C8C83092F6050E941244C3C8F2E0F0934B
:10E0B000F6058091F60590E083709070892B09F445
:10E0C00046CC0E94F22784E00E945C1F882309F45A
:10E0D00088C58091F0078823B9F090E000E001C086
:10E0E000012FE92FF0E0E858F74F10811F701F5FF4
:10E0F000100F601620F0611610F40C9423799F5FC6
:10E100008091F007981760F384E00E941B2483E05D
:10E110000E941B2488E00E941B248091F60580FD4C
:10E1200016C08B81823011F40C9461799B819130FF
:10E1300011F40C947C79EB81EE2331F084E00E94A1
:10E14000852383E00E94852388E00E9485230E9426
:10E15000A7241092F605FBCB83E08C838091F40515
:10E16000893009F0C3CB87E10E94881F882309F416
:10E17000BDCB1092F4053092F605B8CBF2E0FC83EB
:10E180008091F405833609F02FC988E00E94881F2A
:10E19000882309F429C91092F4053092F60524C9A0
:10E1A0001092ED070E94922483E20E948523309210
:10E1B000F305809165070E94881F882309F019CE16
:10E1C00048CE1092ED0782E20E941B248FE00E944D
:10E1D00085230E94A7241092F605809165070E946E
:10E1E000881F882309F0DFC920CA1092ED0780E05C
:10E1F0000E9427030E94922482E20E9485231093AA
:10E20000330610936F0210936E02109371021092F6
:10E2100070021092BB051093FA0581E20E941B2444
:10E220008091EA076091F007409163072091F10720
:10E230000091EA07E09061070E945B2B0E9407664D
:10E2400080E00E94721F882311F40C9477680C946C
:10E2500072681092ED0782E20E941B2481E00E9406
:10E26000124480E00E94124481E00E942703309211
:10E2700033068091DB08882311F00C94ED6881E06F
:10E280000E94124480E00E9412441092F8051092FD
:10E290004A06309274083092ED071092F30580918F
:10E2A0008D082091CE083091EA076091F00790E048
:10E2B000880F991F820F911D880F991F880F991F32
:10E2C000880F991F830F911D70E062957295707F82
:10E2D0007627607F762782959295907F9827807F1A
:10E2E000982744E358E00E9490451092F7050C945B
:10E2F000ED688091F107882309F0DDC69091CE0882
:10E3000080916107981709F03AC46090F007662081
:10E3100009F48AC700E0FF247FEFA0E08824992455
:10E32000AA24BB2424E3C22E28E0D22ECA0CDB1C74
:10E33000F501ED5BF74F80818F708D3009F476C168
:10E3400030E020E1F60190E080818F708E3009F49A
:10E3500068C19F5F31969217B8F3892F913108F009
:10E3600080E18150832BF401E858F74F8083E080EF
:10E370009FE0E922E39440E050E013C071277F7BE7
:10E38000F9F4EF2DF0E0E859F84F81E080830023A5
:10E3900009F0BCC0A1E0F3944F5F5F4F4E1588F5C4
:10E3A000712F642FF601E40FF51F1081212F30E04B
:10E3B000C9018F7090700F9709F47BC0AA23F1F602
:10E3C000EF2DF0E0E859F84F2082E02FF0E0DF0178
:10E3D000A257B74F1C936295607FEE50F84F608351
:10E3E0000F5F0024220F331F001C220F331F001C5D
:10E3F000232F302DA22FA170F3944F5F5F4F4E1546
:10E4000078F20894811C911CE0E1F0E0AE0EBF1E92
:10E41000861408F0B0C1712F85CF1092ED070E94CD
:10E42000922482E20E9485233092330630926F025A
:10E4300030926E0210927102109270021092BB051F
:10E440003092FA0581E20E9485238091EA0760916B
:10E45000F007409163072091F1070091EA07E090EF
:10E4600061070E945B2B81E00E94270382E00E94EB
:10E47000721F882309F4B8CD77CD809174089DE090
:10E48000909365078093A8078CE08093740830927E
:10E49000ED070C94B36884E0809374083092ED0724
:10E4A0000C94BF68309274083092ED0776CD90E1FD
:10E4B000ABCBEF2DF0E0E859F84F1082A0E06BCF26
:10E4C000EF2DF0E0E859F84F1082A0E086C9EF2D5B
:10E4D000F0E0E859F84F1082A0E00C9487697C9234
:10E4E000EB2DF0E0EC5CF74F808180648083EC9250
:10E4F00061E00C94396A7C92EB2DF0E0EC5CF74F14
:10E50000808180648083EC9261E04BCAE02FF0E070
:10E51000E357F74F10830150E02FF0E00F5FEE500C
:10E52000F84FA081AF70BA2FBF5F808182958F7046
:10E53000682F70E0CB018B0F911D40970CF0BA2F24
:10E540000024220F331F001C220F331F001C232F17
:10E55000302DA22FA17062957295707F7627607F13
:10E560007627B62BB08317CFE02FF0E0E357F74FB5
:10E5700010830150E02FF0E00F5FEE50F84FA081C4
:10E58000AF70BA2FBF5F808182958F70682F70E067
:10E59000CB018B0F911D40970CF0BA2F0024220F56
:10E5A000331F001C220F331F001C232F302DA22FDE
:10E5B000A17062957295707F7627607F7627B62B63
:10E5C000B0830C948769E02FF0E0E357F74F108396
:10E5D0000150E02FF0E00F5FEE50F84FA081AF70D8
:10E5E000BA2FBF5F808182958F70682F70E0CB015A
:10E5F0008B0F911D40970CF0BA2F0024220F331F70
:10E60000001C220F331F001C232F302DA22FA170BE
:10E6100062957295707F7627607F7627B62BB083E0
:10E62000DCC8992309F099CE80E09CCE30E12FE040
:10E6300089CE992309F0B3C880E0B6C8992311F0B8
:10E640000C94686980E00C946D693092340680E027
:10E650000E945C1F882311F40C944B68F2E0F09345
:10E6600034060C944B68803170F4E82FF0E0EC5CD9
:10E67000F74F9EE090838F5F06C0E82FF0E0EC5CE0
:10E68000F74F70828F5F8031C0F38091780884FFEC
:10E6900003C0EDE0E093430880918D089091CE088F
:10E6A0002091EA07E82EFF24EE0CFF1CE90EF11C76
:10E6B000EE0CFF1CEE0CFF1CEE0CFF1CE20EF11C1E
:10E6C000E294F29450EFF522FE24E522FE2482E04B
:10E6D0000E9485230E94A72400E010E0F801EC5C72
:10E6E000F74F8081B701600F711F0E94164582E0CD
:10E6F0000E9478160E945F0E0F5F1F4F00311105B8
:10E7000069F782E00E941B240E94A7241092F7055B
:10E7100080918D082091CE083091EA076091F00732
:10E7200090E0880F991F820F911D880F991F880F05
:10E73000991F880F991F830F911D70E06295729544
:10E74000707F7627607F762782959295907F9827B5
:10E75000807F982744E358E00E9490451092F70587
:10E760001092F305309274083092ED0730925605FE
:10E7700011E00C943268FFE3FF1590F0EF2DF0E00C
:10E78000E859F84F1082F3948FE38F15B8F70034EF
:10E7900048F4E02FF0E0EE50F84F9FEF90830F5FCA
:10E7A0000034B8F380E090E0FC01E859F84F1082A3
:10E7B000019680349105C1F7E2E0E093F3051092F1
:10E7C000D1081092F5051092F4051092F6051092FA
:10E7D00060073092F80589E0809374083092ED0765
:10E7E00066246A94CFCB30E12FE00C945C6930E171
:10E7F0002FE00C94C46B8091F40590E00E968F701E
:10E8000090708F5F8093F40583E08093F60524CAAF
:10E810008091F4058F708F5F8093F40583E080937F
:10E82000F60514CA8091F605823008F400C580917F
:10E83000F4058F5F8093F40583E08093F605DAC9D1
:10E840000E94F227E62DF0E0EE50F84F80818F3FD6
:10E85000D1F0108112951F7000810F70010F0F5FB2
:10E86000101738F010C0812F0E942B261F5F101741
:10E8700050F48091F60580FDF6CF812F0E9442274B
:10E880001F5F1017B0F38091F60580FDA5C1852D9F
:10E8900061E00E94D8291092F6050E94A7240C94EA
:10E8A0000F6A86E10E94721F882309F01EC20E942F
:10E8B0004D20882309F0E4C187E10E94881F882346
:10E8C00029F0FFE36F0E6F223092F6058EE00E9472
:10E8D000721F882331F080E1582A3092F60591E0CA
:10E8E0009A838FE00E94721F882331F0E0E25E2A53
:10E8F0003092F605F1E0FA8384E10E94721F8823CA
:10E9000031F080E8582A3092F60591E09A8385E14B
:10E910000E94721F882331F0E0E45E2A3092F605EF
:10E92000F1E0FA838EE00E94881F882331F08FEE99
:10E9300058223092F60591E09A838FE00E94881F5A
:10E94000882331F0EFED5E223092F605F1E0FA8394
:10E9500084E10E94881F882331F08FE7582230928B
:10E96000F60591E09A8385E10E94881F882311F4BF
:10E970000C94066AEFEB5E223092F605F1E0FA8322
:10E980000C94066A182F1150812F0E942227809123
:10E990008D089091CE08E82EFF24EE0CFF1CE90EA6
:10E9A000F11CEE0CFF1CEE0CFF1CEE0CFF1CE10E2C
:10E9B000F11CE294F29440EFF422FE24E422FE24BF
:10E9C0008701005F1F4F8FE0B7010E94164582E06C
:10E9D0000E9478160E945F0E0894E11CF11CE0165C
:10E9E000F10689F73BCA86E10E94B11F882311F422
:10E9F0000C94826CE62DF0E0E859F84F80818B830F
:10EA00003092F40592E09093F6050C94826C93E0BA
:10EA10008091F405882381F08091F40581508093E2
:10EA2000F4058091C4058F5F8093C4059093F6052B
:10EA30008091C405882361F71092C40501C98091B3
:10EA4000F405813108F4E9C081E08093F40583E0A6
:10EA50000E941B248091F405882309F034C981E0C9
:10EA60008093F4058091F4050E9444288091F60576
:10EA7000823008F035C930923306809133068823FE
:10EA800031F081E00E94721F882309F01FC41092A8
:10EA9000BE0580E00E945C1F882311F03092BE0505
:10EAA000109233061DC9112309F0A4C38091F40507
:10EAB000882309F49FC39C81992341F4E62DF0E05B
:10EAC000E859F84F8B81808391E09A83E2E0E093EC
:10EAD000F6058091F605843011F00C948C6C1FC8FB
:10EAE000E82FF0E0E859F84F10828F5F8034C0F3D0
:10EAF000103448F4E12FF0E0EE50F84F9FEF908390
:10EB00001F5F1034B8F39091F4058091F5058111E1
:10EB100080E191509F70892B8093780850917808FC
:10EB20005F705F5F80E070E0A0E06FEF20E030E0BA
:10EB30000FC0D901AC5CB74F7C929230B9F0842FF2
:10EB40008F5F2F5F3F4F251708F08DCD892FA42FA2
:10EB5000422FF901E859F84F9081913051F78823FD
:10EB600009F009C1D901AC5CB74F7C92E72FF0E006
:10EB7000E257F74F60817F5F6C9392E0E0CF809126
:10EB800061078093CE0880918D082091CE08309146
:10EB9000EA076091F00790E0880F991F820F911D9E
:10EBA000880F991F880F991F880F991F830F911D38
:10EBB00070E062957295707F7627607F76278295E8
:10EBC0009295907F9827807F982744E358E00E9491
:10EBD00090451092F70599CB852D60E00E94D829C9
:10EBE0005ACE8091F007882309F48ECA90E080E025
:10EBF00001C08E2FE92FF0E0E858F74FE081EF7069
:10EC0000EF5FE80F681618F06E1608F441C39F5FB7
:10EC10008091F007981768F377CA8091F40515CFB3
:10EC20008091F40546C886E0809374083092ED0721
:10EC30001A8211E00C943268F0937408F093ED0797
:10EC40001A8211E00C94326880918D086091CE0890
:10EC50004091EA072091F00704E318E00E94C95BA5
:10EC60000C941A6D80918D086091CE084091EA074E
:10EC70002091F00704E318E00E94C95B0C94836ABA
:10EC8000582E5A948FE058228EE00E945C1F8823F1
:10EC900011F090E1592A8FE00E945C1F882311F047
:10ECA000E0E25E2A84E10E945C1F882311F0F0E814
:10ECB0005F2A85E10E945C1F882311F080E4582AB6
:10ECC000E52DF0E0EF73F070E75AFA4F452D4078EC
:10ECD000808160E00E94FB4392E09093F60583E020
:10ECE0008093F405E1E0EA83E7CDE62DF0E0E2571A
:10ECF000F74F50808EE00E945C1F882321F0F0E1E6
:10ED00005F2A81E08A838FE00E945C1F882321F0C4
:10ED100090E2592AE1E0EA8384E10E945C1F8823A3
:10ED200021F0F0E85F2A81E08A8385E10E945C1F80
:10ED3000882321F090E4592AE1E0EA83E52DF0E010
:10ED4000EF73F070E75AFA4F452D4078808160E00C
:10ED50000E94FB43F2E0F093F6053092F405A7CD54
:10ED600050E14FE00C94876EF901E859F84F10829A
:10ED7000A0E00C94BA6EF901EC5CF74F7082B0E041
:10ED8000AC5CB74F8C9180648C936083D8CEE12FBC
:10ED9000F0E0E357F74F00831150E12FF0E01F5FE1
:10EDA000EE50F84FA081AF70BA2FBF5F808182957F
:10EDB0008F70682F70E0CB018B0F911D40970CF086
:10EDC000BA2F0024440F551F001C440F551F001C70
:10EDD000452F502DA42FA17062957295707F7627D4
:10EDE000607F7627B62BB0830C94BA6E80E00C94CB
:10EDF0009F6EFFE3FF1510F40C94376CEF2DF0E0DD
:10EE0000E859F84F1082F3948FE38F15B8F70C94FC
:10EE1000376CFFE3FF1510F40C94D269EF2DF0E08E
:10EE2000E859F84F1082F3948FE38F15B8F70C94DC
:10EE3000D26986E10E94881F882319F088E08093B8
:10EE4000F4058EE00E94721F882331F092E09093C7
:10EE5000F6059B83E1E0EA838FE00E94721F88231E
:10EE600031F0F2E0F093F60581E08B838A8384E150
:10EE70000E94721F882311F40C947C6C92E0909392
:10EE8000F6051B82E1E0EA830C947C6C0E944D2025
:10EE9000182F0E94C720882321F4112311F40C9409
:10EEA000006AE62DF0E0E257F74F508280E00E94C2
:10EEB000124482E00E9478166394FFE3F61518F47A
:10EEC0001092F50566243092F6051092F4058FE055
:10EED00058228EE00E945C1F882311F090E1592A8D
:10EEE0008FE00E945C1F882311F0E0E25E2A84E13B
:10EEF0000E945C1F882311F0F0E85F2A85E10E94E0
:10EF00005C1F882311F080E4582A112311F40C941B
:10EF1000006A512E5A949FE059228EE00E945C1F95
:10EF2000882311F0E0E15E2A8FE00E945C1F8823B5
:10EF300011F0F0E25F2A84E10E945C1F882311F047
:10EF400080E8582A85E10E945C1F882311F090E434
:10EF5000592AE52DF0E0EF73F070E75AFA4F452D8E
:10EF60004078808160E00E94FB43E2E0E093F60598
:10EF700083E08093F4050C94006A86E10E94881F68
:10EF80008823A1F1E62DF0E0E257F74F8081851547
:10EF900011F081E08A8350828EE00E945C1F8823FA
:10EFA00009F04CC155248FE00E945C1F882311F0AA
:10EFB00090E2592A84E10E945C1F882311F0E0E866
:10EFC0005E2A85E10E945C1F882311F0F0E45F2A2D
:10EFD00080E00E94124463948FE3861518F4109227
:10EFE000F50566243092F6051092F4058EE00E9435
:10EFF000721F882359F0852D809580719FEE5922CC
:10F00000582AE2E0E093F605F1E0FA838FE00E94EF
:10F01000721F882359F0852D809580729FED5922AB
:10F02000582AE2E0E093F605F1E0FA8384E10E94D9
:10F03000721F882359F0852D809580789FE759228B
:10F04000582AE2E0E093F605F1E0FA8385E10E94B8
:10F05000721F882359F0852D809580749FEB59226B
:10F06000582AE2E0E093F605F1E0FA830E944D2091
:10F07000182F882311F40C94FA6980E00E9412443E
:10F0800082E00E94781611501F7080EF5822512A9A
:10F09000E52DF0E0EF73F070E75AFA4F452D407818
:10F0A000808160E00E94FB4392E09093F605E1E0EE
:10F0B000EA830C94FA698091A90780938D08809166
:10F0C00061078093CE08809163078093EA0780915F
:10F0D000F1078093F0071092F10755CD992311F4B1
:10F0E0000C94A26A82E20E941B248DE00E94852378
:10F0F0000E94A7241092F6050C94AA6A50E14FE0F2
:10F100000C94C86D82E00E9485230E94A7249091F0
:10F110008D082091CE083091EA078091F10588236F
:10F12000C9F1E92EFF24EE0CFF1CE20EF11CEE0CDF
:10F13000FF1CEE0CFF1CEE0CFF1CE30EF11CE29416
:10F14000F29460EFF622FE24E622FE248701A0E07E
:10F15000B0E0FD01E655F84F8081AC5CB74F8C9371
:10F16000B8010E94164582E00E9478160E945F0E48
:10F170000F5F1F4F802F8E19A82FB0E08091F105EF
:10F1800090E082959295907F9827807F9827A81786
:10F19000B907FCF26091EA07809143088F708D30C7
:10F1A00009F473C050E040E120E030E0922FF90113
:10F1B000EC5CF74F80818F708E3029F09F5F2F5F5E
:10F1C0003F4F241798F39923B9F1892F9131C8F54E
:10F1D0008150852B898389818F708F5F809358053B
:10F1E00060936707898184FD25C08CE08093570573
:10F1F0000C94BD6A63948091F505681608F45BCCA5
:10F2000081E08C8363CC0E94A921882311F00C94A7
:10F21000FF68F2E0F093F6050C94FF68FF2400E02D
:10F22000EDCDFF2400E0FACDFF2400E0A7CA109244
:10F23000F405FDCA80E1DACF80E0CBCF60E1562E45
:10F24000B2CE80E1C5CF011708F05BC0F02EEE24EE
:10F2500008C08E2D60E00E94B826F394E394F11666
:10F2600010F5EF2DF0E0E859F84F8081823041F041
:10F270008081813071F78E2D62E00E94B826EDCF3B
:10F280008E2D61E00E94B826E8CF50E14FE08CCF90
:10F29000962D981B8091F60580FF29C0892F0E942A
:10F2A0002B260C948470101B103110F00C94847079
:10F2B000812F63E00E94B8261F5F1031C8F30C94C1
:10F2C000847084E00E9485230C94A77030923406E9
:10F2D00080E00E945C1F882319F0F2E0F09334066E
:10F2E000309274083092ED0730925605D9CB892FB1
:10F2F0000E9442270C94847083E00E9485230C9422
:10F30000A77010E0D5CF0F931F93CF93DF93EC013D
:10F31000442319F18B0150E070E020E030E0F90166
:10F32000E858F74F60816F706F5FD80190E0FE0181
:10F33000E50FF11D80818D939F5F5F5F9617B8F396
:10F34000760F2F5F3F4F005F1F4F241740F3872F2B
:10F35000DF91CF911F910F91089570E0872FDF917A
:10F36000CF911F910F910895BF92CF92DF92EF92AC
:10F37000FF920F931F93CF93DF936B01B42E44231F
:10F3800069F17C0110E000E0C0E0D0E0C7010E941C
:10F39000F858FE01E858F74F808320812F702F5FC7
:10F3A000D70190E08D91F601E10FF11D80839F5F01
:10F3B0001F5F9217B8F3020F219680E190E0E80EEC
:10F3C000F91ECB1518F3802FDF91CF911F910F916C
:10F3D000FF90EF90DF90CF90BF90089500E0F3CFC3
:10F3E000EF920F930E9445228091DB08882309F455
:10F3F000CDC084E00E9434590E9445220E945F0ED5
:10F40000009174080130B9F1043051F001E00E941C
:10F410007D5A882369F1002379F70F91EF900895C1
:10F420000E943A59882309F07DC00E94C45788235E
:10F4300009F473C080917408843011F0109233067F
:10F440008091DB08882309F492C00E9462578823C8
:10F4500051F4809132068130C9F6109232060E9432
:10F460005457882399F200E00E947D5A882399F628
:10F470000E94405AD0CF0E943A59882369F50E94D1
:10F48000076686E10E94721F882391F080913606FC
:10F49000882309F074C080E20E94185990917C087A
:10F4A000980F90933606892F60E040E00E94FB435E
:10F4B0000E94625A80917408813011F010923306D4
:10F4C0008091DB08882309F056C00E945457882396
:10F4D00009F49CCF00E0C8CF0E94922482E20E94EF
:10F4E00085230093330681E061E042E00E94B65735
:10F4F00081E20E941B248091EA076091F00740910D
:10F5000063072091F1070091EA07E09061070E94EC
:10F510005B2B81E00E942703B2CF0E9407660E9406
:10F52000625A88CF0E94922482E20E94852381E061
:10F53000809333060091BB0561E042E00E94B6571C
:10F54000033041F181E20E9485238091EA076091B6
:10F55000F007409163072091F1070091EA07E090DE
:10F5600061070E945B2B81E00E9427035ECF81E050
:10F570000E9434596ACF84E00E943459A6CF80E0BB
:10F580000E94124481E00E94781685CF81E00E949B
:10F59000345932CF0093BB05D5CF6F927F928F92B3
:10F5A0009F92AF92BF92CF92DF92EF92FF920F9312
:10F5B0001F93DF93CF93CDB7DEB7C054D0400FB6C3
:10F5C000F894DEBF0FBECDBF1092F6051092F40581
:10F5D00082E08093F305E090F007EE2009F4B9C2D1
:10F5E0006624FF24CC24DD24AA24BB244E010894E5
:10F5F000811C911C85010C5C174FC8010E94F858B2
:10F60000F601E858F74F808320812F702F5FD801D3
:10F6100090E08D91F401EF0DF11D80839F5FF394D5
:10F620009217B8F3620E0894C11CD11C80E190E0DF
:10F63000A80EB91ECE14F0F28091F505861508F0DB
:10F640008BC28091F0078823F1F020E050E0852FF5
:10F6500090E0FC01E858F74F30813F703F5F452F45
:10F660004295407F90E0E22FF0E0842F892BEE500E
:10F67000F84F80839F5F2F5F9317A8F35F5F8091A0
:10F68000F007581720F30E9445228091DB08882359
:10F6900009F45BC284E00E943459EE244E010894C0
:10F6A000811C911C0E9445220E945F0E10917408DB
:10F6B000113089F0143009F450C00E947D5A88231B
:10F6C00089F70E94405A0E9445220E945F0E1091C5
:10F6D0007408113079F70E943A59882309F0BDC1A6
:10F6E0000E94076686E10E94B11F882329F080915D
:10F6F000F705882309F0CFC187E10E94B11F882355
:10F7000029F08091F705882309F0D9C18091740808
:10F71000813011F0109233068091DB08882309F0C4
:10F72000B3C10E945457882341F21092F305C05C84
:10F73000DF4F0FB6F894DEBF0FBECDBFCF91DF9184
:10F740001F910F91FF90EF90DF90CF90BF90AF90FF
:10F750009F908F907F906F9008950E943A598823D0
:10F7600009F0F6C010E086E10E94B11F882309F07D
:10F7700014C187E10E94B11F882309F02AC186E1E4
:10F780000E94881F882309F040C187E10E94881FDA
:10F79000882309F045C186E10E94721F882309F081
:10F7A0004AC18EE00E94721F882339F08E2D809509
:10F7B00080719FEEE922E82A12E08FE00E94721F1A
:10F7C000882339F08E2D809580729FEDE922E82AFA
:10F7D00012E084E10E94721F882339F08E2D8095FB
:10F7E00080789FE7E922E82A12E085E10E94721FF3
:10F7F000882339F08E2D809580749FEBE922E82ACA
:10F8000012E00E944D20282F882361F08E2D90E079
:10F810008F7090700D9734F421502F7080EFE82294
:10F82000E22A12E088E00E94721F882309F478C05F
:10F830008E2D90E08F7090700D970CF429C190EF91
:10F84000E9228091F505F401E80FF11DE0821091A5
:10F85000F007112309F475C1662420E040E050E070
:10F8600060E070E0FA01E858F74F30813F703F5F89
:10F87000DB01AC5CB74F90E0F401E20FF11D808139
:10F880008D939F5F2F5F9317B8F3630E4F5F5F4FAA
:10F89000605F7F4F411730F381E08093F7058E2D35
:10F8A00090E08F7090700D970CF046C08E2D61E047
:10F8B0000E94D82984E20E9485230E94F227E091C9
:10F8C000F505F0E0EE50F84F10811F70812F0E9477
:10F8D0004227E091F505F0E0EE50F84F80818295E7
:10F8E0008F70181709F42BC163E00E94B8260E949C
:10F8F000A72480917408843011F01092330680910F
:10F90000DB08882309F180913206813009F0D5CED9
:10F91000109232060E945457882309F4CECE05CFA8
:10F92000123009F48ECF113021F78E2D90E08F70B8
:10F9300090700D970CF4BACF8E2D60E00E94D829FC
:10F9400084E20E941B24B9CF81E00E943459DBCFAE
:10F950000E94922482E20E94852381E080933306F4
:10F9600080E060E040E00E94B65781E20E9485237B
:10F970008091F705882309F4DEC082E00E94A1236C
:10F980008091F505F401E80FF11DE08011E086E1BA
:10F990000E94B11F882309F4ECCE8091F5058F5F9A
:10F9A0008093F5058091F505662D0E943B87909325
:10F9B000F5058091F505F401E80FF11DE08082E086
:10F9C0000E94852311E087E10E94B11F882309F47A
:10F9D000D6CE8091F505662D70E090E00197860FF8
:10F9E000971F0E945B878093F5058091F505F401D0
:10F9F000E80FF11DE08080E00E94852311E086E1A0
:10FA00000E94881F882309F4C0CE82E00E941B2434
:10FA10000E94A72487E10E94881F882309F4BBCE97
:10FA200080E00E941B240E94A72486E10E94721F8E
:10FA3000882309F4B6CE80E00E945C1F882309F475
:10FA4000B0CE809166078093F5058091F505F401AD
:10FA5000E80FF11DE08011E0A4CE0E94922482E222
:10FA60000E9485231093330681E060E042E00E940B
:10FA7000B65781E20E941B248091F7058823D9F0B4
:10FA800082E00E94A1232CCE84E00E94345949CE0A
:10FA90008FE0E82ED6CE82E00E941B2480918D0854
:10FAA0006091CE084091EA072091F00704E318E046
:10FAB0000E94C95B21CE82E00E941B2411CE82E00D
:10FAC0000E941B2480918D086091CE084091EA0726
:10FAD0002091F00704E318E00E94715B7090F0073A
:10FAE000772089F16624FF24CC24DD24AA24BB24BA
:10FAF00085010C5C174FC8010E94F858F601E858C0
:10FB0000F74F808320812F702F5FD80190E08D9177
:10FB1000F401EF0DF11D80839F5FF3949217B8F30A
:10FB2000620E0894C11CD11C80E190E0A80EB91EA1
:10FB3000C714F0F2EBCD82E00E941B2421CF62E0DB
:10FB4000D4CE6624A9CE6624E1CD81E00E9434594A
:10FB5000A4CD8091F50566241092F50572CD2F9203
:10FB60003F924F925F926F927F928F929F92AF924D
:10FB7000BF92CF92DF92EF92FF920F931F93DF938A
:10FB8000CF93CDB7DEB7C558D0400FB6F894DEBFDF
:10FB90000FBECDBF1092F6051092F40580E060E034
:10FBA00042E00E94B657F090F007FF2011F40C9449
:10FBB0005C867724EE24CC24DD24AA24BB2411E423
:10FBC000812E912C8C0E9D1E85010C5C174FC80157
:10FBD0000E94F858F601E858F74F808320812F7073
:10FBE0002F5FD80190E08D91F401EE0DF11D80831F
:10FBF0009F5FE3949217B8F3720E0894C11CD11C56
:10FC000080E190E0A80EB91ECF14F0F20E944522C8
:10FC10008091DB08882309F462C484E00E9434598F
:10FC20002224CD57DF4F1882C358D040CE57DF4F24
:10FC30001882C258D040CF57DF4F1882C158D040E9
:10FC400033243A946624B1E4AB2EB12CAC0EBD1E25
:10FC50002E010894411C511C0E9445220E945F0EF7
:10FC6000109174081F3009F415C3103108F090C0CA
:10FC7000113009F4F4C2143021F111E00E947D5AD0
:10FC8000882309F482C0112339F71092F305CB576A
:10FC9000DF4F0FB6F894DEBF0FBECDBFCF91DF911F
:10FCA0001F910F91FF90EF90DF90CF90BF90AF909A
:10FCB0009F908F907F906F905F904F903F902F908C
:10FCC00008950E943A59882309F090C484E00E9464
:10FCD000B11F882309F045C485E00E94B11F882325
:10FCE00009F04BC482E10E94B11F882309F051C47E
:10FCF00081E10E94B11F882309F057C40E94076662
:10FD0000882309F45DC40E94625A86E10E94B11FF3
:10FD1000882329F08091F705882309F0BDC787E182
:10FD20000E94B11F882329F08091F705882309F0EC
:10FD30006CC780917408843061F01092330682E0C1
:10FD40000E941B2482E20E941B240E94F2270E9430
:10FD500007298091DB08882309F43FC58091F705C6
:10FD6000882309F433C580913206813009F085CFAC
:10FD7000109232060E945457882309F47ECF10E077
:10FD80000E947D5A882309F07ECF0E94405A7BCF83
:10FD9000113109F472C1113108F481C0123109F036
:10FDA0006CCF0E943A59882309F07AC40E94CB593B
:10FDB0008CE00E94721F882309F07EC48CE00E94B0
:10FDC000881F882309F086C48EE00E94721F882352
:10FDD00009F089C48FE00E94721F882309F092C441
:10FDE00084E10E94721F882309F09BC485E10E9470
:10FDF000721F882309F0A4C488E00E94721F882320
:10FE000009F0ADC48EE00E94881F882309F0B6C4B3
:10FE10008FE00E94881F882309F0B9C484E10E9402
:10FE2000881F882309F0BCC485E10E94881F8823AD
:10FE300009F0BFC488E00E94881F882309F0C2C46B
:10FE4000222009F41ACFA1E0A093F705772009F446
:10FE5000F4C2850110C00E97F9F08F2D8321D801CF
:10FE60009C919621892BF80181938F018E2F8A19FD
:10FE7000871508F0E2C20E940402F82E90E08F700D
:10FE800090708D30910539F7B7EFFB228F2D90E000
:10FE90008F7090700E9709F7E7EFFE22DECF0E9479
:10FEA0003A59882309F038C50E94CB598CE00E944A
:10FEB000721F882309F02AC587E10E94721F8823D8
:10FEC00009F01EC580E00E94721F882309F012C548
:10FED0008CE00E94881F882309F008C587E10E94F2
:10FEE000881F882309F07DC480E00E94881F882332
:10FEF00009F080C48EE00E94721F882309F083C439
:10FF00008FE00E94721F882309F08CC484E10E9454
:10FF1000721F882309F095C485E10E94721F88230F
:10FF200009F09EC488E00E94721F882309F0A7C4CC
:10FF30008EE00E94881F882309F0B0C48FE00E94E1
:10FF4000881F882309F0B3C484E10E94881F882396
:10FF500009F0B6C485E10E94881F882309F0B9C45E
:10FF600088E00E94881F882309F0BCC4222009F47D
:10FF700084CEF1E0F093F70522E0221609F4F1C5F2
:10FF8000F4E02F1609F4FEC6B1E02B1609F097C66F
:10FF9000772009F1850106C00F5F1F4F802F8A1956
:10FFA0008715C8F40E940402F82EEFE1E817A0F3C9
:10FFB0000E940402D8012C91672D0E943B87F50115
:10FFC000E90FF11D80818C9320830F5F1F4F802FDD
:10FFD0008A19871538F31091F0071123F1F020E00A
:10FFE00040E050E060E070E0FA01E858F74F3081FF
:10FFF0003F703F5FDB01AC5CB74F90E0F501E20F73
:020000021000EC
:10000000F11D80818D939F5F2F5F9317B8F34F5F32
:100010005F4F605F7F4F411738F32090F007222039
:1000200009F49CC27724EE24CC24DD24882499246E
:1000300084010C5C174FC8010E94F858F601E8587B
:10004000F74F808320812F702F5FD80190E08D9132
:10005000F501EE0DF11D80839F5FE3949217B8F3D5
:10006000720E0894C11CD11C80E190E0880E991E8C
:10007000C214F0F2222411E001CE0E943A598823E2
:1000800009F056C50E94CB598CE00E94721F88234C
:1000900009F045C58CE00E94881F882309F03BC504
:1000A0008EE00E94721F882309F02BC58FE00E940A
:1000B000721F882309F01BC584E10E94721F8823E8
:1000C00009F0E4C485E10E94721F882309F0EDC4A1
:1000D00088E00E94721F882309F0F6C48EE00E9417
:1000E000881F882309F0FFC48FE00E94881F88239F
:1000F00009F0C8C484E10E94881F882309F01AC44B
:1001000085E10E94881F882309F010C488E00E94BE
:10011000881F882309F0C0C28DE00E94721F8823C7
:1001200029F08091F105882309F004C2122D10FFF7
:10013000A4CDA1E0A093F70511FFD5C1772099F1D7
:10014000850106C00F5F1F4F802F8A19871558F54C
:100150000E940402F82EBFE3B817A0F30E94040225
:10016000CE57DF4F6881C258D0400E943B87F201D2
:10017000E90FF11DF0808F2D90E08F7090708D3021
:10018000910509F4DDC40E9709F4D7C49F2D93217E
:10019000D8018C918621982B9C930F5F1F4F802F45
:1001A0008A198715A8F2BEEF2B221091F0071123B0
:1001B000F1F020E040E050E060E070E0FA01E85843
:1001C000F74F30813F703F5FDB01AC5CB74F90E091
:1001D000F501E20FF11D80818D939F5F2F5F9317D3
:1001E000B8F34F5F5F4F605F7F4F411738F3E09187
:1001F000F007CC57DF4FE883C458D040EE2309F412
:10020000AEC17724EE24CC24DD24882499248401F3
:100210000C5C174FC8010E94F858F601E858F74FD8
:10022000808320812F702F5FD80190E08D91F501A0
:10023000EE0DF11D80839F5FE3949217B8F3720E69
:100240000894C11CD11C80E190E0880E991ECC5707
:10025000DF4F9881C458D040C916C8F20ECD0E9415
:100260003A59882309F0E5C30E9407660E94625A42
:1002700080917408813011F0109233068091DB0870
:10028000882309F0D2C30E945457882309F4F5CC7F
:1002900010E076CD0E943A59882309F0EDC10E9402
:1002A000CB5986E10E94721F882309F0D7C189E0EB
:1002B0000E94721F882309F0C5C18AE00E94721F44
:1002C000882309F0B3C186E10E94881F882309F0C2
:1002D000A9C189E00E94881F882309F09FC18AE094
:1002E0000E94881F882309F095C18DE00E94721F2B
:1002F000882329F08091F105882309F06FC4B1E0CB
:100300002B1609F424C392E0291609F417C3B3E0AD
:100310002B1609F0B2CCE1E0E093F705CE57DF4FA2
:10032000F881C258D0406F2F70E0CD57DF4F288141
:10033000C358D040822F992787FD9095860F971F2D
:10034000CF57DF4FA881C158D0408A0F911D0E941E
:100350005B87CF57DF4F8883C158D0407720D9F0D3
:1003600020E030E0F501E20FF31FCF57DF4F888127
:10037000C158D040820FCE57DF4F6881C258D0405D
:100380000E943B87D201A90FB11D8C9180832F5F02
:100390003F4F271538F31091F0071123F1F020E0BB
:1003A00040E050E060E070E0FA01E858F74F30813B
:1003B0003F703F5FDB01AC5CB74F90E0F501E20FAF
:1003C000F11D80818D939F5F2F5F9317B8F34F5F6F
:1003D0005F4F605F7F4F411738F32090F007222076
:1003E00009F4BCC07724EE24CC24DD24882499248D
:1003F00084010C5C174FC8010E94F858F601E858B8
:10040000F74F808320812F702F5FD80190E08D916E
:10041000F501EE0DF11D80839F5FE3949217B8F311
:10042000720E0894C11CD11CE0E1F0E08E0E9F1EFC
:10043000C214F0F2222411E021CC1091F007112314
:10044000F1F020E040E050E060E070E0FA01E858B0
:10045000F74F30813F703F5FDB01AC5CB74F90E0FE
:10046000F501E20FF11D80818D939F5F2F5F931740
:10047000B8F34F5F5F4F605F7F4F411738F32090B5
:10048000F007222009F46AC07724EE24CC24DD246E
:100490008824992484010C5C174FC8010E94F858E5
:1004A000F601E858F74F808320812F702F5FD80125
:1004B00090E08D91F501EE0DF11D80839F5FE39437
:1004C0009217B8F3720E0894C11CD11C80E190E021
:1004D000880E991EC214F0F2222411E0CFCB81E0E5
:1004E0000E9434599DCB772009F45DCE850107C069
:1004F0000F5F1F4F802F8A19871508F054CE0E9476
:100500000402F82EBFE3B81798F30E940402F82EF5
:1005100090E08F7090708D30910509F41BC30E9799
:1005200009F415C39F2D9321D8018C918621982B16
:100530009C93DECF822D8095827091E02922282A1B
:100540008DE00E941B24122D21FC44C4CE57DF4FA6
:100550001882C258D0400E94A724E9CD22247724D3
:100560008CCB609174088FE044E00E94205985E0B4
:100570000E94B11F882309F4B5CB6091740880E113
:1005800045E00E94205982E10E94B11F882309F4AE
:10059000AFCB6091740882E142E10E94205981E171
:1005A0000E94B11F882309F4A9CB6091740881E1EE
:1005B00041E10E9420590E940766882309F0A3CBDD
:1005C00080E20E94BD2389E10E94BD238CE00E944D
:1005D000BD238BE00E94BD238091F705882309F499
:1005E00012C362E082E00E94D7238DCB0E94922446
:1005F00082E20E94852391E09093330680E060E0E0
:1006000042E00E94B65781E20E94852381E00E9469
:1006100027035CCB8CE10E941B2467CE8BE10E94F8
:100620001B245DCE82E00E941B2453CE8CE10E94ED
:1006300085232F2C239491E0CD57DF4F9883C35807
:10064000D04041CE8BE10E9485232F2C23948FEF45
:10065000CD57DF4F8883C358D0402FCE82E00E9411
:100660008523209166072195CD57DF4F2883C358F6
:10067000D040222423941BCE80E20E948523222492
:10068000CD57DF4F1882C358D040FF24CF57DF4FDC
:100690001882C158D04003CE84E20E941B243CCD76
:1006A0008BE00E94852322240E94CB598CE00E947B
:1006B000721F882309F482CB8EE00E9485232224B6
:1006C000239433243A9466248CE00E94881F882364
:1006D00009F47ACB8EE00E941B248EE00E94721FE8
:1006E000882309F477CB84E00E9485232224239475
:1006F000A0E13A2EFFEE6F2E8FE00E94721F88233A
:1007000009F46ECB83E00E94852322242394E0E247
:100710003E2E7FED672E84E10E94721F882309F42C
:1007200065CB88E00E9485232224239460E8362E3E
:100730005FE7652E85E10E94721F882309F45CCB78
:1007400081E00E9485232224239440E4342E3FEB51
:10075000632E88E00E94721F882309F453CB84E241
:100760000E948523222423942FE0322E90EF692EBD
:100770008EE00E94881F882309F44ACB84E00E94FF
:100780001B248FE00E94881F882309F447CB83E055
:100790000E941B2484E10E94881F882309F444CB13
:1007A00088E00E941B2485E10E94881F882309F4A9
:1007B00041CB81E00E941B2488E00E94881F88238F
:1007C00009F43ECB84E20E941B243ACB0E9462577C
:1007D000882309F4C8CA10E0D3CA81E00E943459C2
:1007E000BDCA80E00E941B2480E00E94881F8823ED
:1007F00009F480CB82E20E941B248EE00E94721FCB
:10080000882309F47DCB84E00E94852374E0272EA1
:1008100060E1362E5FEE652E8FE00E94721F882306
:1008200009F474CB83E00E94852344E0242E30E257
:10083000332E2FED622E84E10E94721F882309F46B
:100840006BCB88E00E94852394E0292E80E8382E27
:100850000FE7602E85E10E94721F882309F462CBA6
:1008600081E00E94852314E0212EB0E43B2EAFEB03
:100870006A2E88E00E94721F882309F459CB84E213
:100880000E948523F4E02F2EEFE03E2E70EF672EBE
:100890008EE00E94881F882309F450CB84E00E94D8
:1008A0001B248FE00E94881F882309F44DCB83E02E
:1008B0000E941B2484E10E94881F882309F44ACBEC
:1008C00088E00E941B2485E10E94881F882309F488
:1008D00047CB81E00E941B2488E00E94881F882368
:1008E00009F444CB84E20E941B2440CB8EE00E949A
:1008F0001B24F4CA82E20E948523E3E02E2EE8CA7C
:1009000080E00E948523F2E02F2EDCCA8EE00E9458
:10091000852322242394D0CA89E10E94852322249E
:10092000CD57DF4F1882C358D040BECA81E00E9425
:100930001B24ECCB88E00E941B24E2CBCD57DF4F79
:10094000A881C358D040AA2309F0E5CC96C9CD5759
:10095000DF4FE881C358D040EE2309F48EC92092BE
:10096000F705772089F03E2F370DD50120E0822F43
:10097000830F672D0E943B87F201E90FF11D8D91D6
:1009800080832F5F271598F31091F0071123F1F062
:1009900020E040E050E060E070E0FA01E858F74FF6
:1009A00030813F703F5FDB01AC5CB74F90E0F201FC
:1009B000E20FF11D80818D939F5F2F5F9317B8F336
:1009C0004F5F5F4F605F7F4F411738F32090F00714
:1009D000222009F4C4CD7724EE24CC24DD248824FD
:1009E000992484010C5C174FC8010E94F858F60145
:1009F000E858F74F808320812F702F5FD80190E057
:100A00008D91F501EE0DF11D80839F5FE3949217A8
:100A1000B8F3720E0894C11CD11C80E190E0880EDE
:100A2000991EC214F0F2222428C984E00E9434598D
:100A30002ACC0E94922482E20E94852310933306DE
:100A400081E060E042E00E94B65781E20E941B24F0
:100A50008091EA076091F007409163072091F107C8
:100A60000091EA07E09061070E945B2B8091F705F7
:100A7000882309F4C4C082E00E94A12381E00E947F
:100A80002703F2CB83E00E941B2434CB88E00E9432
:100A90008523E1E02E2A20E8322E9FE7692E85E1AA
:100AA0000E94721F882309F413CB81E00E948523E2
:100AB000F1E02F2A80E4382E0FEB602E88E00E94B0
:100AC000721F882309F40ACB84E20E94852321E067
:100AD000222A1FE0312EB0EF6B2E8EE00E94881F7D
:100AE000882309F401CB84E00E941B24FDCA83E023
:100AF0000E948523B1E02B2A40E2342E3FED632E85
:100B0000DBCA84E00E948523A1E02A2A60E1362E18
:100B10005FEE652ECBCA8EE00E941B24C1CA8EE018
:100B20000E94852391E0292A33243A946624B2CA8C
:100B30008CE00E9485232224A5CAF7EFFF2226CB52
:100B4000E7EFFE228F2D90E08F7090701CCBF7EFB7
:100B5000FF22E8CCE7EFFE228F2D90E08F7090709F
:100B6000DECC672D6695D9F0972D915040E050E08E
:100B7000A92FB0E09201240F351FF501EA0FFB1FEA
:100B80008081F9018083A40DB51DF501E40FF51FE7
:100B900080818C9391504F5F5F4F461748F37720C9
:100BA00009F419CA81E040E050E0672D0E943B87BC
:100BB000D501A40FB51FF201E90FF11D20812074AA
:100BC000F201E40FF51F80818F7B282B2C93892F56
:100BD0008F5F4F5F5F4F471540F3FDC9F394A1E06E
:100BE000FA228DE00E941B24FF2009F003C1CE579A
:100BF000DF4F1882C258D0400E94A72480CB82E0E9
:100C00000E941B243BCF60E0EDCC82E00E941B24BD
:100C100080918D086091CE084091EA072091F007FD
:100C200004E318E00E94715BA091F007CB57DF4FFF
:100C3000A883C558D040AA2309F4FBC07724EE242A
:100C4000CC24DD248824992484010C5C174FC8012E
:100C50000E94F858F601E858F74F808320812F70E2
:100C60002F5FD80190E08D91F501EE0DF11D80838D
:100C70009F5FE3949217B8F3720E0894C11CD11CC5
:100C8000E0E1F0E08E0E9F1ECB57DF4FF881C55894
:100C9000D040CF16C8F24DC882E00E941B2480913C
:100CA0008D086091CE084091EA072091F00704E397
:100CB00018E00E94C95B33C877240C94067E6091CB
:100CC000F00784E398E0A50128E637E00E94C95CBC
:100CD000E82E882311F1850106C00F5F1F4F802F7A
:100CE0008A198E15D0F40E940402F82EBFE3B817BB
:100CF000A0F30E940402F80120816E2D0E943B8720
:100D0000F501E90FF11D8081D8018C9320830F5FDD
:100D10001F4F802F8A198E1530F36091F00784E3FE
:100D200098E0A50128E637E00E9442597090F0074C
:100D3000772009F450C9EE24CC24DD24882499249A
:100D400084010C5C174FC8010E94F858F601E8585E
:100D5000F74F808320812F702F5FD80190E08D9115
:100D6000F501EE0DF11D80839F5FE3949217B8F3B8
:100D70000894C11CD11CE0E1F0E08E0E9F1EC71448
:100D8000F8F229C9772009F426C9850107C00F5F49
:100D90001F4F802F8A19871508F01DC90E94040271
:100DA000F82E2FE3281798F30E940402D8012C9103
:100DB000672D0E943B87F501E90FF11D808183219A
:100DC000962D9223892B8C93808186212321822B3F
:100DD0008083DDCF8DE00E9485238AEA97E0B2010F
:100DE0004091F1050E94B479CE57DF4F8883C258F5
:100DF000D040B1CB8DE00E9485238AEA97E0B20112
:100E00004091F1050E94B479CE57DF4F8883C258D4
:100E1000D0404091F00784E398E0B5010E94B47996
:100E2000782EA3E02A2ECD57DF4F1882C358D0402A
:100E3000E3CE77240C94997E629FD001739FF001DA
:100E4000829FE00DF11D649FE00DF11D929FF00D5A
:100E5000839FF00D749FF00D659FF00D9927729F91
:100E6000B00DE11DF91F639FB00DE11DF91FBD011C
:100E7000CF0111240895991B79E004C0991F96179A
:100E800008F0961B881F7A95C9F780950895AA1BCC
:100E9000BB1B51E107C0AA1FBB1FA617B70710F065
:100EA000A61BB70B881F991F5A95A9F78095909597
:100EB000BC01CD01089597FB092E07260AD077FDC6
:100EC00004D0E5DF06D000201AF4709561957F4FBD
:100ED0000895F6F7909581959F4F0895A1E21A2EF7
:100EE000AA1BBB1BFD010DC0AA1FBB1FEE1FFF1FCE
:100EF000A217B307E407F50720F0A21BB30BE40B1E
:100F0000F50B661F771F881F991F1A9469F7609564
:100F10007095809590959B01AC01BD01CF0108951E
:040F2000F894FFCF73
:100F240001FFFFFFFFFFFFFFFF808D5B0000060C4A
:100F340012000A101A0001020D0002030E0002043E
:100F44000E0003050F0003060F0004071000040839
:100F5400100005091100050A1100060B1200060C09
:100F64001200070D1300070E1300080F14000810D9
:100F7400140009111500091215000A1316000A14A9
:100F840016000B1517000B16170A0A0410080101A6
:100F9400020106000100010001000100010001003E
:100FA40001000100010001000100010001C00080F6
:100FB4000040007F20640130480405060711121028
:100FC400130F04050607111210130E0409050A066F
:100FD400070B110C120D1013252123262724222080
:100FE4001D1E1B191F1C1A1012180F110C130E0BA7
:100FF400140D0A1516091704050803060107000253
:1010040013141516170506070003040D0E0F1C1BF9
:101014002423212220191A180C0B0A0908010200A2
:1010240007060517161514131112101F1E1D272667
:1010340023241B1C0F0E0D040300020108090A0BD4
:101044000C181A192022212326271D1E1F101211E5
:10105400201B191C1A180F0C0E0B0D0A090320195A
:101064001A180C0B0A0904080120191A180C0B0A87
:10107400092221252320191A18241B1C0F0E0D04E4
:10108400030A0C0B090801020026271D1E1F10125B
:101094001113141516170506076E306E7830780094
:1010A4000A4D324443206D69737365733A20000A14
:1010B4004C45442073656D692D6C69743A20003485
:1010C4004D487A00324D487A000A5350493A20007C
:1010D4002900202F20002028000A5348464C3A209B
:1010E400000A4D3244433A20000A5853796E633A59
:1010F40020000A54656D706F436F6566663A200080
:101104003A000A4D54524947206F66667365743A33
:1011140020000A42414E4B4C45443A20000A4D57A8
:101124005241503A20000A42504D3A20002F000A02
:101134004D49444920492F4F206368616E3A20008D
:101144000A53796E633A20000100070E091C1B1232
:1011540015383F363124232A2D70777E796C6B62E3
:1011640065484F464154535A5DE0E7EEE9FCFBF213
:10117400F5D8DFD6D1C4C3CACD90979E998C8B8203
:1011840085A8AFA6A1B4B3BABDC7C0C9CEDBDCD5B0
:10119400D2FFF8F1F6E3E4EDEAB7B0B9BEABACA523
:1011A400A28F88818693949D9A2720292E3B3C35D3
:1011B400321F18111603040D0A5750595E4B4C4543
:1011C400426F68616673747D7A898E878095929B7D
:1011D4009CB1B6BFB8ADAAA3A4F9FEF7F0E5E2EB63
:1011E400ECC1C6CFC8DDDAD3D4696E676075727B93
:1011F4007C51565F584D4A4344191E171005020B83
:101204000C21262F283D3A33344E49404752555C31
:101214005B7671787F6A6D64633E39303722252CA2
:101224002B0601080F1A1D1413AEA9A0A7B2B5BC52
:10123400BB9691989F8A8D8483DED9D0D7C2C5CCC2
:10124400CBE6E1E8EFFAFDF4F30409050A06070B1F
:10125400110C120D10130001000100010001000126
:101264000001000100010001000100010001000172
:10127400C00080004000010C011718191A1B1C1D26
:101284001E1F202122233F3F3F0B0C0D0E0F101178
:101294001213141516173F3F3F2324252627282908
:1012A4002A2B2C2D2E2F3F3F3F0B0C0D0E0F101110
:0C12B4001213141516173F3F3F150000E1
:00000001FF
